:020000040801F1
:1000000000000220952B01087F1F01089B1F01089B
:10001000B71F0108D31F0108EF1F010800000000EF
:100020000000000000000000000000000B2001089C
:1000300019200108000000002720010835200108D0
:10004000E52B0108E52B0108E52B0108E52B01084C
:10005000E52B0108E52B0108E52B0108E52B01083C
:10006000E52B0108E52B0108E52B0108E52B01082C
:10007000E52B0108E52B0108E52B0108E52B01081C
:10008000E52B0108E52B0108E52B010845200108B7
:1000900059200108E52B0108E52B01086D20010816
:1000A0008D200108B1200108D5200108E52B0108A9
:1000B000E52B0108E52B0108E52B0108E52B0108DC
:1000C000E52B0108E52B0108E52B0108E52B0108CC
:1000D000E52B0108F9200108E52B0108E52B0108B3
:1000E00005210108E52B0108E52B01082521010860
:1000F0004921010885210108E52B0108E52B0108AC
:10010000E52B0108E52B0108E52B0108E52B01088B
:10011000E52B0108E52B0108E52B0108E52B01087B
:10012000E52B0108E52B0108E52B0108E52B01086B
:10013000E52B01080000000000000000E52B01088D
:10014000E52B0108E52B0108E52B0108E52B01084B
:10015000E52B0108E52B0108E52B0108A921010881
:10016000E52B0108E52B0108E52B0108E52B01082B
:10017000E52B0108E52B0108E52B01080000000034
:1001800000000000E52B0108000000000000000056
:10019000E52B01080000000000000000E52B01082D
:1001A000000000000000000000000000E52B010836
:1001B000E52B0108E52B0108E52B0108E52B0108DB
:0401C000E52B010822
:1001D00010B5054C237833B9044B13B10448AFF381
:1001E00000800123237010BDF00E002000000000ED
:1001F000A87A030808B5034B1BB103490348AFF3C2
:10020000008008BD00000000F40E0020A87A03085A
:1002100010F8012B11F8013B012A28BF9A42F7D0B0
:10022000D01A7047034613F8012B002AFBD1181A85
:1002300001387047000000000000000000000000CE
:1002400001F0FF01102A2BDB10F0070F08D010F887
:10025000013B013A8B422DD010F0070F42B3F6D18B
:10026000F0B441EA012141EA014122F007047FF0A4
:1002700000070023F0E80256083C85EA010586EAFB
:10028000010685FA47F5A3FA87F586FA47F6A5FA37
:1002900087F68EB9EED1F0BC01F0FF0102F0070243
:1002A00032B110F8013B013A83EA010313B1F8D1EE
:1002B0000020704701387047002D06BF35460338CF
:1002C000073815F0010F07D1013015F4807F02BF08
:1002D000013015F4C03F0130F0BC0138704700BF59
:1002E00081F0004102E000BF83F0004330B54FEAE7
:1002F00041044FEA430594EA050F08BF90EA020F54
:100300001FBF54EA000C55EA020C7FEA645C7FEAE6
:10031000655C00F0E2804FEA5454D4EB5555B8BF09
:100320006D420CDD2C4480EA020281EA030382EA7A
:10033000000083EA010180EA020281EA0303362D0C
:1003400088BF30BD11F0004F4FEA01314FF4801CDF
:100350004CEA113102D0404261EB410113F0004FF1
:100360004FEA03334CEA133302D0524263EB4303A8
:1003700094EA050F00F0A780A4F10104D5F1200E46
:100380000DDB02FA0EFC22FA05F2801841F10001A1
:1003900003FA0EF2801843FA05F359410EE0A5F175
:1003A00020050EF1200E012A03FA0EFC28BF4CF0A6
:1003B000020C43FA05F3C01851EBE37101F000455C
:1003C00007D54FF0000EDCF1000C7EEB00006EEB69
:1003D0000101B1F5801F1BD3B1F5001F0CD34908F3
:1003E0005FEA30004FEA3C0C04F101044FEA44524A
:1003F00012F5800F80F09A80BCF1004F08BF5FEAD1
:10040000500C50F1000041EB045141EA050130BDB0
:100410005FEA4C0C404141EB0101013C28BFB1F5C2
:10042000801FE9D291F0000F04BF01460020B1FA0D
:1004300081F308BF2033A3F10B03B3F120020CDAE0
:100440000C3208DD02F1140CC2F10C0201FA0CF0BE
:1004500021FA02F10CE002F11402D8BFC2F1200C23
:1004600001FA02F120FA0CFCDCBF41EA0C019040D9
:10047000E41AA2BF01EB0451294330BD6FEA040422
:100480001F3C1CDA0C340EDC04F11404C4F120020D
:1004900020FA04F001FA02F340EA030021FA04F31F
:1004A00045EA030130BDC4F10C04C4F1200220FA76
:1004B00002F001FA04F340EA0300294630BD21FAB4
:1004C00004F0294630BD94F0000F83F4801306BF7A
:1004D00081F480110134013D4EE77FEA645C18BF6E
:1004E0007FEA655C29D094EA050F08BF90EA020F05
:1004F00005D054EA000C04BF1946104630BD91EAFD
:10050000030F1EBF0021002030BD5FEA545C05D1FF
:100510004000494128BF41F0004130BD14F580043E
:100520003CBF01F5801130BD01F0004545F0FE41B2
:1005300041F470014FF0000030BD7FEA645C1ABFE7
:10054000194610467FEA655C1CBF0B46024650EA1E
:10055000013406BF52EA033591EA030F41F400214A
:1005600030BD00BF90F0000F04BF0021704730B5D0
:100570004FF4806404F132044FF000054FF00001A5
:1005800050E700BF90F0000F04BF0021704730B566
:100590004FF4806404F1320410F0004548BF40423B
:1005A0004FF000013EE700BF42004FEAE2014FEA90
:1005B00031014FEA02701FBF12F07F4393F07F4F6B
:1005C00081F06051704732F07F4208BF704793F06E
:1005D0007F4F04BF41F40021704730B54FF4607481
:1005E00001F0004521F000411CE700BF50EA010284
:1005F00008BF704730B54FF000050AE050EA01022D
:1006000008BF704730B511F0004502D5404261EB9C
:1006100041014FF4806404F132045FEA915C3FF4DD
:10062000D8AE4FF003025FEADC0C18BF03325FEA7A
:10063000DC0C18BF033202EBDC02C2F1200300FA2B
:1006400003FC20FA02F001FA03FE40EA0E0021FA50
:1006500002F11444BDE600BF70B54FF0FF0C4CF43E
:10066000E06C1CEA11541DBF1CEA135594EA0C0FF0
:1006700095EA0C0F00F0DEF82C4481EA030621EA2B
:100680004C5123EA4C5350EA013518BF52EA033566
:1006900041F4801143F4801338D0A0FB02CE4FF018
:1006A0000005E1FB02E506F00042E0FB03E54FF048
:1006B0000006E1FB03569CF0000F18BF4EF0010E40
:1006C000A4F1FF04B6F5007F64F5407404D25FEA3C
:1006D0004E0E6D4146EB060642EAC62141EA5551EF
:1006E0004FEAC52040EA5E504FEACE2EB4F1FD0C31
:1006F00088BFBCF5E06F1ED8BEF1004F08BF5FEAAF
:10070000500E50F1000041EB045170BD06F0004660
:1007100046EA010140EA020081EA0301B4EB5C040D
:10072000C2BFD4EB0C0541EA045170BD41F4801105
:100730004FF0000E013C00F3AB8014F1360FDEBF2A
:10074000002001F0004170BDC4F10004203C35DA06
:100750000C341BDC04F11404C4F1200500FA05F389
:1007600020FA04F001FA05F240EA020001F000422A
:1007700021F0004110EBD37021FA04F642EB0601A0
:100780005EEA430E08BF20EAD37070BDC4F10C04CA
:10079000C4F1200500FA04F320FA05F001FA04F28E
:1007A00040EA020001F0004110EBD37041F100017A
:1007B0005EEA430E08BF20EAD37070BDC4F1200585
:1007C00000FA05F24EEA020E20FA04F301FA05F2ED
:1007D00043EA020321FA04F001F0004121FA04F295
:1007E00020EA020000EBD3705EEA430E08BF20EA65
:1007F000D37070BD94F0000F0FD101F0004640009F
:1008000041EB010111F4801F08BF013CF7D041EA20
:10081000060195F0000F18BF704703F00046520024
:1008200043EB030313F4801F08BF013DF7D043EAF5
:100830000603704794EA0C0F0CEA135518BF95EAAB
:100840000C0F0CD050EA410618BF52EA4306D1D132
:1008500081EA030101F000414FF0000070BD50EA51
:10086000410606BF1046194652EA430619D094EADB
:100870000C0F02D150EA013613D195EA0C0F05D1C5
:1008800052EA03361CBF104619460AD181EA030119
:1008900001F0004141F0FE4141F470014FF00000D1
:1008A00070BD41F0FE4141F4780170BD70B54FF06C
:1008B000FF0C4CF4E06C1CEA11541DBF1CEA1355EC
:1008C00094EA0C0F95EA0C0F00F0A7F8A4EB0504CE
:1008D00081EA030E52EA03354FEA013100F08880C5
:1008E0004FEA03334FF0805545EA131343EA12638E
:1008F0004FEA022245EA111545EA10654FEA002643
:100900000EF000419D4208BF964244F1FD0404F5FB
:10091000407402D25B084FEA3202B61A65EB030557
:100920005B084FEA32024FF480104FF4002CB6EB14
:10093000020E75EB030E22BFB61A754640EA0C0094
:100940005B084FEA3202B6EB020E75EB030E22BFD4
:10095000B61A754640EA5C005B084FEA3202B6EB15
:10096000020E75EB030E22BFB61A754640EA9C00D4
:100970005B084FEA3202B6EB020E75EB030E22BFA4
:10098000B61A754640EADC0055EA060E18D04FEA62
:10099000051545EA16754FEA06164FEAC30343EA02
:1009A00052734FEAC2025FEA1C1CC0D111F4801FCF
:1009B0000BD141EA00014FF000004FF0004CB6E7C8
:1009C00011F4801F04BF01430020B4F1FD0C88BF67
:1009D000BCF5E06F3FF6AFAEB5EB030C04BFB6EB72
:1009E000020C5FEA500C50F1000041EB045170BD65
:1009F0000EF0004E4EEA113114EB5C04C2BFD4EB92
:100A00000C0541EA045170BD41F480114FF0000E15
:100A1000013C90E645EA060E8DE60CEA135594EA91
:100A20000C0F08BF95EA0C0F3FF43BAF94EA0C0F94
:100A30000AD150EA01347FF434AF95EA0C0F7FF409
:100A400025AF104619462CE795EA0C0F06D152EA5D
:100A500003353FF4FDAE1046194622E750EA410641
:100A600018BF52EA43067FF4C5AE50EA41047FF452
:100A70000DAF52EA43057FF4EBAE12E74FF0FF3CB7
:100A800006E000BF4FF0010C02E000BF4FF0010C88
:100A90004DF804CD4FEA410C7FEA6C5C4FEA430C01
:100AA00018BF7FEA6C5C1BD001B050EA410C0CBF50
:100AB00052EA430C91EA030F02BF90EA020F0020B2
:100AC000704710F1000F91EA030F58BF994208BF19
:100AD00090422CBFD8176FEAE37040F001007047D6
:100AE0004FEA410C7FEA6C5C02D150EA013C07D12D
:100AF0004FEA430C7FEA6C5CD6D152EA033CD3D078
:100B00005DF8040B704700BF8446104662468C4671
:100B10001946634600E000BF01B5FFF7B7FF0028A4
:100B200048BF10F1000F01BD4DF808EDFFF7F4FFCD
:100B30000CBF012000205DF808FB00BF4DF808ED58
:100B4000FFF7EAFF34BF012000205DF808FB00BF7B
:100B50004DF808EDFFF7E0FF94BF012000205DF89D
:100B600008FB00BF4DF808EDFFF7CEFF94BF012052
:100B700000205DF808FB00BF4DF808EDFFF7C4FF4B
:100B800034BF012000205DF808FB00BF4FEA410C94
:100B90007FEA6C5C02D150EA013C0AD14FEA430C77
:100BA0007FEA6C5C02D152EA033C02D14FF00000B4
:100BB00070474FF0010070474FEA410212F50012F2
:100BC00015D211D56FF47873B3EB625212D94FEA94
:100BD000C12343F0004343EA505311F0004F23FA7E
:100BE00002F018BF404270474FF00000704750EAD3
:100BF000013005D111F0004008BF6FF00040704790
:100C00004FF00000704700BF4A0011D212F50012E9
:100C100011D20DD56FF47873B3EB62520ED44FEA54
:100C2000C12343F0004343EA505323FA02F07047D4
:100C30004FF00000704750EA013002D14FF0FF3012
:100C400070474FF00000704753B94AB9002908BFF8
:100C500000281CBF4FF0FF314FF0FF3000F074B997
:100C6000ADF1080C6DE904CE00F006F8DDF804E003
:100C7000DDE9022304B070472DE9F047089D0446E2
:100C80008E46002B4DD18A42944669D9B2FA82F23F
:100C900052B101FA02F3C2F1200120FA01F10CFA7B
:100CA00002FC41EA030E94404FEA1C48210CBEFBB3
:100CB000F8F61FFA8CF708FB16E341EA034306FB3C
:100CC00007F199420AD91CEB030306F1FF3080F0CB
:100CD0001F81994240F21C81023E63445B1AA4B218
:100CE000B3FBF8F008FB103344EA034400FB07F7BA
:100CF000A7420AD91CEB040400F1FF3380F00A81FB
:100D0000A74240F207816444023840EA0640E41BEF
:100D100000261DB1D4400023C5E900433146BDE89B
:100D2000F0878B4209D9002D00F0EF800026C5E93D
:100D3000000130463146BDE8F087B3FA83F6002E55
:100D40004AD18B4202D3824200F2F980841A61EBCD
:100D5000030301209E46002DE0D0C5E9004EDDE7EB
:100D600002B9FFDEB2FA82F2002A40F09280A1EBD3
:100D70000C014FEA1C471FFA8CFE0126200CB1FB28
:100D8000F7F307FB131140EA01410EFB03F0884221
:100D900008D91CEB010103F1FF3802D2884200F2AE
:100DA000CB804346091AA4B2B1FBF7F007FB101140
:100DB00044EA01440EFB00FEA64508D91CEB0404DE
:100DC00000F1FF3102D2A64500F2BB800846A4EB39
:100DD0000E0440EA03409CE7C6F12007B34022FA24
:100DE00007FC4CEA030C20FA07F401FA06F31C4353
:100DF000F9404FEA1C4900FA06F3B1FBF9F8200C60
:100E00001FFA8CFE09FB181140EA014108FB0EF0A5
:100E1000884202FA06F20BD91CEB010108F1FF3AF5
:100E200080F08880884240F28580A8F10208614401
:100E3000091AA4B2B1FBF9F009FB101144EA01410F
:100E400000FB0EFE8E4508D91CEB010100F1FF34BA
:100E50006CD28E456AD90238614440EA0840A0FB52
:100E60000294A1EB0E01A142C846A64656D353D028
:100E70005DB1B3EB080261EB0E0101FA07F722FA4C
:100E800006F3F1401F43C5E9007100263146BDE875
:100E9000F087C2F12003D8400CFA02FC21FA03F3D8
:100EA000914001434FEA1C471FFA8CFEB3FBF7F059
:100EB00007FB10360B0C43EA064300FB0EF69E427E
:100EC00004FA02F408D91CEB030300F1FF382FD217
:100ED0009E422DD9023863449B1B89B2B3FBF7F6BF
:100EE00007FB163341EA034106FB0EF38B4208D998
:100EF0001CEB010106F1FF3816D28B4214D9023ED9
:100F00006144C91A46EA004638E72E46284605E7F6
:100F10000646E3E61846F8E64B45A9D2B9EB0208C7
:100F200064EB0C0E0138A3E74646EAE7204694E757
:100F30004046D1E7D0467BE7023B614432E730468A
:100F400009E76444023842E7704700BF80B500AF4C
:100F5000184B194A1A60174B05225A60154B00228C
:100F60009A60144B4FF08072DA60124B4FF45022AB
:100F70001A61104B4FF400125A610E4B00221A7680
:100F80000C4B01225A760B4B00229A76094B012218
:100F9000DA76084B00221A77064B00225A7705486A
:100FA00001F094FE0346002B01D000F0F1FD00BFDC
:100FB00080BD00BF0C0F00200064004080B58AB0E7
:100FC00000AF786007F1140300221A605A609A603B
:100FD000DA601A617B681B68214A93423CD1002386
:100FE0003B61204B1B6C1F4A43F0007313641D4B85
:100FF0001B6C03F000733B613B690023FB60194BE2
:101000001B6B184A43F002031363164B1B6B03F070
:101010000203FB60FB684FF440737B610223BB61FA
:101020000023FB6103233B6209237B6207F1140366
:1010300019460D4802F0DCFD00220021132002F0C9
:10104000A0FD132002F0B9FD00220021142002F0BF
:1010500098FD142002F0B1FD00BF2837BD4680BDC9
:1010600000640040003802400004024080B58EB0A9
:1010700000AF07F11C0300221A605A609A60DA6020
:101080001A615A619A613B4600221A605A609A605E
:10109000DA601A615A619A61664B4FF020421A6019
:1010A000644B654A5A60634B00229A60614B002290
:1010B000DA60604B00221A615E4B10225A615D4B70
:1010C00000229A615B4B0022DA615A4B00225A627D
:1010D000584B4FF480529A62564B0022DA62554BBD
:1010E00000221A63534B00225A63524B00229A6328
:1010F000504B0022DA634F4B00221A644D4B002202
:101100005A640323FB610F233B6203237B620123A9
:10111000BB621023FB6211233B6300237B6307F157
:101120001C0300221946434802F075FF0346002BBA
:1011300001D000F02DFD414B414A1A603F4B002287
:101140005A603E4B01229A603C4B0822DA603B4BCE
:1011500010221A61394B40225A61384B4FF4C07249
:101160009A61364B0022DA61344B4FF400621A6206
:10117000324B4FF480525A62304B4FF400529A6215
:1011800002233B6008237B600623BB600623FB60D1
:1011900004233B6102237B610223BB613B4619466A
:1011A000264802F0B9FE0346002B01D000F0F0FC07
:1011B000244B234A1A60234B01225A60214B0122FF
:1011C0009A60204B0822DA601E4B10221A611D4BD8
:1011D00040225A611B4B4FF4C0729A61194B002296
:1011E000DA61184B4FF400621A62164B4FF48052CA
:1011F0005A62144B4FF400529A6202233B60082358
:101200007B600623BB600623FB6004233B61022353
:101210007B610223BB613B4619460A4802F07CFE13
:101220000346002B01D000F0B3FC00BF3837BD46A9
:1012300080BD00BF340F0020040100A0840F0020F7
:10124000400100A0B80F002080B586B000AF3B1D64
:1012500000221A605A609A60DA601A613B4B1B6880
:10126000002B6FD1394B01221A6000233B60384BB1
:101270009B6B374A43F001039363354B9B6B03F041
:1012800001033B603B684FF63F037B600223BB607A
:101290000023FB6003233B610C237B613B1D19464C
:1012A0002C4802F0A5FC19237B600223BB600023BD
:1012B000FB6003233B610C237B613B1D19462648E1
:1012C00002F096FC48F237137B600223BB600023D8
:1012D000FB6003233B610C237B613B1D19461F48C8
:1012E00002F086FC4FF683737B600223BB60002311
:1012F000FB6003233B610C237B613B1D19461848AF
:1013000002F076FC4CF2B3737B600223BB600023D7
:10131000FB6003233B610C237B613B1D1946114895
:1013200002F066FC60237B600223BB600023FB604D
:1013300003233B610C237B613B1D19460A4802F0E5
:1013400057FC00E000BF1837BD4680BDEC0F002001
:101350000038024000140240000802400018024019
:1013600000100240000C02400004024080B582B030
:1013700000AF7860FFF768FF00BF0837BD4680BD4B
:1013800080B582B000AF7860FFF75EFF00BF08371E
:10139000BD4680BD80B400AF044BDB681B0A03F080
:1013A00007031846BD465DF8047B704700ED00E07A
:1013B00080B483B000AF0346FB7197F90730002B70
:1013C0000BDBFB7903F01F02074997F907305B0934
:1013D000012000FA02F241F8232000BF0C37BD467D
:1013E0005DF8047B704700BF00E100E080B483B08B
:1013F00000AF03463960FB7197F90730002B0ADB19
:101400003B68DAB20C4997F907301201D2B20B44AB
:1014100083F800230AE03B68DAB20849FB7903F05D
:101420000F03043B1201D2B20B441A7600BF0C37F3
:10143000BD465DF8047B704700E100E000ED00E090
:1014400080B489B000AFF860B9607A60FB6803F0DF
:101450000703FB61FB69C3F10703042B28BF0423C7
:10146000BB61FB690433062B02D9FB69033B00E037
:1014700000237B614FF0FF32BB6902FA03F3DA43CA
:10148000BB681A407B699A404FF0FF317B6901FAD3
:1014900003F3D9437B680B40134318462437BD46FA
:1014A0005DF8047B7047000080B485B000AF7860C1
:1014B000084B1A6B07497B6813430B63054B1A6B88
:1014C0007B681340FB60FB6800BF1437BD465DF8C6
:1014D000047B70470038024080B485B000AF78606C
:1014E0003960134A3B68DBB2023352F823203B6871
:1014F0001B0CDB4302EA03013B681B0CFB60FB682F
:1015000093FAA3F3BB60BB68B3FA83F3DBB21A466A
:101510007B6803FA02F206483B68DBB20A430233F7
:1015200040F8232000BF1437BD465DF8047B7047A8
:101530000038014080B489B000AFF860B9607A60CB
:10154000FB681A68BB687B617B6993FAA3F33B6114
:101550003B69B3FA83F3DBB25B00032101FA03F3C7
:10156000DB431A40BB68FB61FB6993FAA3F3BB61E1
:10157000BB69B3FA83F3DBB25B00796801FA03F36A
:101580001A43FB681A6000BF2437BD465DF8047B30
:10159000704780B489B000AFF860B9607A60FB68CA
:1015A000DA68BB687B617B6993FAA3F33B613B69B3
:1015B000B3FA83F3DBB25B00032101FA03F3DB43ED
:1015C0001A40BB68FB61FB6993FAA3F3BB61BB697B
:1015D000B3FA83F3DBB25B00796801FA03F31A43D1
:1015E000FB68DA6000BF2437BD465DF8047B7047B6
:1015F00080B483B000AF786039607B683A689A61E4
:1016000000BF0C37BD465DF8047B704780B483B0E3
:1016100000AF786039603B681A047B689A6100BF4C
:101620000C37BD465DF8047B7047000080B588B07C
:1016300000AF07F1180300221A605A603B460022EF
:101640001A605A609A60DA601A615A610420FFF7E2
:101650002BFF2020FFF728FF8020FFF725FF012028
:10166000FFF722FF4020FFF71FFF1020FFF71CFFAE
:101670000220FFF719FF0820FFF716FF4FF4C041C3
:101680005F48FFF7B5FF48F210015E48FFF7B0FF73
:101690004FF480515C48FFF7ABFF4FF4807158481E
:1016A000FFF7B4FF4FF400533B6001237B6000233E
:1016B000BB600123FB6001233B613B461946504858
:1016C00003F052F94FF480433B6001237B60002319
:1016D000BB600023FB6001233B613B461946484841
:1016E00003F042F948F210033B6001237B600223C0
:1016F000BB600123FB6001233B613B461946414827
:1017000003F032F94FF480533B6001237B600223E6
:10171000BB600123FB6001233B613B4619463A480D
:1017200003F022F94FF480733B6001237B600223B6
:10173000BB600023FB6002233B613B4619463048F7
:1017400003F012F931490220FFF7C6FE30490320A9
:10175000FFF7C2FE4FF40043BB6101233B77002338
:101760007B770223BB7707F11803184602F030FDA0
:101770004023BB6101233B7700237B770223BB77A8
:1017800007F11803184602F023FD01224FF400412F
:101790001B48FFF7FEFE012240211E48FFF7F9FE1D
:1017A00000224FF400411648FFF7C4FE00224021FA
:1017B0001848FFF7BFFEFFF7EDFD034600220021AA
:1017C0001846FFF73DFE034619461720FFF70EFEA9
:1017D0001720FFF7EDFDFFF7DDFD03460022002196
:1017E0001846FFF72DFE034619462820FFF7FEFD99
:1017F0002820FFF7DDFD00BF2037BD4680BD00BFBC
:10180000000802400000024000040240030000F013
:101810000100000F000C024080B400AF054B1B68B4
:10182000044A43F48023136000BFBD465DF8047B87
:10183000704700BF0038024080B400AF054B1B6802
:10184000044A43F48033136000BFBD465DF8047B57
:10185000704700BF0038024080B400AF074B1B68E0
:1018600003F40033B3F5003F0CBF01230023DBB2C8
:101870001846BD465DF8047B704700BF0038024043
:1018800080B483B000AF7860064B9B6823F00302FE
:1018900004497B6813438B6000BF0C37BD465DF87D
:1018A000047B70470038024080B400AF044B9B6853
:1018B00003F00C031846BD465DF8047B704700BF7B
:1018C0000038024080B483B000AF7860064B9B685C
:1018D00023F0F00204497B6813438B6000BF0C3790
:1018E000BD465DF8047B70470038024080B483B089
:1018F00000AF7860064B9B6823F4E05204497B6894
:1019000013438B6000BF0C37BD465DF8047B704706
:101910000038024080B483B000AF7860064B9B680B
:1019200023F4604204497B6813438B6000BF0C378B
:10193000BD465DF8047B70470038024080B483B038
:1019400000AF7860074BD3F88C3023F080720549E4
:101950007B681343C1F88C3000BF0C37BD465DF87F
:10196000047B70470038024080B400AF054B1B6811
:10197000044A43F08073136000BFBD465DF8047BEA
:10198000704700BF0038024080B400AF074B1B68AF
:1019900003F00073B3F1007F0CBF01230023DBB21F
:1019A0001846BD465DF8047B704700BF0038024012
:1019B00080B485B000AFF860B9607A603B60114BCD
:1019C0005A68114B1340F968BA6811437A6892015A
:1019D0000A430C4913434B600A4B5B6823F44032C3
:1019E00008493B6813434B60064B5B6823F0E042B9
:1019F00004493B6813434B6000BF1437BD465DF894
:101A0000047B7047003802400080BFFF80B483B081
:101A100000AF7860064B1B6823F00F0204497B6817
:101A200013430B6000BF0C37BD465DF8047B704765
:101A3000003C024080B400AF044B1B6803F00F036E
:101A40001846BD465DF8047B704700BF003C02406D
:101A500080B400AF054B1B68044A43F48033136025
:101A600000BFBD465DF8047B704700BF00700040BA
:101A700080B483B000AF7860064B1B6823F440420B
:101A800004497B6813430B6000BF0C37BD465DF80B
:101A9000047B70470070004080B500AF22F05CFE10
:101AA00001F0A2F800F022F8FFF7C0FD00F0B2FF4D
:101AB00001F010F8FFF7DAFA00F0CCF8FFF746FA79
:101AC00000F030F900F082F900F018FD00F076FD2A
:101AD00000F0AEFD00F0E2FD00F016FE00F04EFE5C
:101AE00000F082FE22F054FEFEE7000080B500AF59
:101AF0000520FFF78BFF00BFFFF79CFF0346052B78
:101B0000FAD14FF44040FFF7B3FFFFF7A1FFFFF713
:101B100083FEFFF791FE00BFFFF79EFE0346012BF9
:101B2000FAD14FF000534FF4B4720C214FF48000FF
:101B3000FFF73EFFFFF718FF00BFFFF725FF034643
:101B4000012BFAD10020FFF7BDFE4FF4A050FFF7A4
:101B5000CDFE4FF40040FFF7DDFE0320FFF790FEBF
:101B600000BFFFF7A1FE03460C2BFAD1074803F094
:101B700017FD002001F05AF80346002B01D000F0B9
:101B800007F80020FFF7DAFE00BF80BD0095BA0A13
:101B900080B400AF72B600BFFEE7000080B485B02D
:101BA00000AF7860084B1A6B07497B6813430B63DF
:101BB000054B1A6B7B681340FB60FB6800BF143752
:101BC000BD465DF8047B70470038024080B485B0A4
:101BD00000AF7860084B1A6C07497B6813430B64AD
:101BE000054B1A6C7B681340FB60FB6800BF143721
:101BF000BD465DF8047B70470038024080B485B074
:101C000000AF7860084B5A6C07497B6813434B64FC
:101C1000054B5A6C7B681340FB60FB6800BF1437B0
:101C2000BD465DF8047B70470038024080B483B045
:101C300000AF786039607B685B6823F010023B6816
:101C40001A437B685A6000BF0C37BD465DF8047BC1
:101C50007047000080B590B000AF07F1180328224C
:101C60000021184622F0E6FD3B4600221A605A6029
:101C70009A60DA601A615A614FF48050FFF7BEFF34
:101C80000120FFF78BFF0220FFF788FFC0233B6096
:101C900002237B600323BB600023FB6000233B61C6
:101CA00005237B613B4619461B4802F05DFE082375
:101CB0003B6002237B600323BB600023FB600023A7
:101CC0003B6105237B613B461946144802F04CFEFC
:101CD0000023BB614FF48273FB6100233B6200234E
:101CE0007B620023BB624FF40073FB6200233B6303
:101CF00000237B630023BB630A23FB6307F1180304
:101D00001946074803F03FF800210548FFF78EFF0A
:101D100000BF4037BD4680BD0000024000040240C5
:101D20000030014080B590B000AF07F118032822C1
:101D30000021184622F07EFD3B4600221A605A60C0
:101D40009A60DA601A615A614FF48040FFF73EFFF3
:101D50000220FFF723FF4FF460433B6002237B60C8
:101D60000323BB600023FB6000233B6105237B61F1
:101D70003B461946134802F0F7FD0023BB614FF4C0
:101D80008273FB6100233B6200237B620023BB6202
:101D90004FF40073FB6200233B6300237B6300234B
:101DA000BB630A23FB6307F118031946064802F0D8
:101DB000EAFF00210448FFF739FF00BF4037BD4666
:101DC00080BD00BF000402400038004080B590B0E4
:101DD00000AF07F1180328220021184622F02AFD3F
:101DE0003B4600221A605A609A60DA601A615A61B2
:101DF0004FF40040FFF7EAFE0420FFF7CFFE022079
:101E0000FFF7CCFE4FF4A0533B6002237B6003231B
:101E1000BB600023FB6000233B6106237B613B46E4
:101E200019461C4802F0A0FD10233B6002237B6092
:101E30000323BB600023FB6000233B6106237B611F
:101E40003B461946144802F08FFD0023BB614FF456
:101E50008273FB6100233B6200237B620023BB6231
:101E60004FF40073FB6200233B6300237B6300237A
:101E7000BB630A23FB6307F118031946074802F006
:101E800082FF00210548FFF7D1FE00BF4037BD4665
:101E900080BD00BF0008024000040240003C00403A
:101EA00080B483B000AF00237B60104B5B6C0F4AA3
:101EB00043F4804353640D4B5B6C03F480437B60BD
:101EC0007B6800233B60094B1B6C084A43F080533E
:101ED0001364064B1B6C03F080533B603B6800BFF0
:101EE0000C37BD465DF8047B704700BF00380240E8
:101EF00080B483B000AF7860074B5A697B681340A9
:101F00007A689A420CBF01230023DBB218460C37D3
:101F1000BD465DF8047B7047003C014080B483B04F
:101F200000AF7860044A7B68536100BF0C37BD4640
:101F30005DF8047B704700BF003C014080B483B073
:101F400000AF78607B686FF001021A6100BF0C3748
:101F5000BD465DF8047B704780B483B000AF786005
:101F60007B681B6903F00103012B01D1012300E011
:101F7000002318460C37BD465DF8047B704780B5DA
:101F800082B000AFEFF308833B603B6810337B60A7
:101F9000796804200AF072F8FEE780B582B000AFDD
:101FA000EFF308833B603B6810337B607968002067
:101FB0000AF064F8FEE780B582B000AFEFF3088363
:101FC0003B603B6810337B60796801200AF056F86B
:101FD000FEE780B582B000AFEFF308833B603B685B
:101FE00010337B60796802200AF048F8FEE780B57C
:101FF00082B000AFEFF308833B603B6810337B6037
:10200000796803200AF03AF8FEE780B400AF00BF19
:10201000BD465DF8047B704780B400AF00BFBD468D
:102020005DF8047B704780B400AF00BFBD465DF82B
:10203000047B704780B500AF06F058F900F026FE2B
:1020400000BF80BD80B500AF024801F0C1FA00BFFB
:1020500080BD00BF0C0F002080B500AF024801F02A
:10206000B7FA00BF80BD00BF0C0F002080B500AFE5
:102070004020FFF73DFF0346002B04D04020FFF730
:102080004DFF18F093FA00BF80BD000080B500AF8F
:102090000648FFF761FF0346012B04D10348FFF711
:1020A0004DFF0AF0F1FE00BF80BD00BF00400140BF
:1020B00080B500AF0648FFF74FFF0346012B04D160
:1020C0000348FFF73BFF0BF0E7F800BF80BD00BF00
:1020D0000044014080B500AF0648FFF73DFF0346CE
:1020E000012B04D10348FFF729FF0BF0DDFA00BFF5
:1020F00080BD00BF0048014080B500AF05F0FAF98F
:1021000000BF80BD80B500AF4FF40040FFF7F0FE88
:102110000346002B03D04FF40040FFF7FFFE00BF43
:1021200080BD000080B500AF0648FFF715FF0346ED
:10213000012B04D10348FFF701FF0BF0BDFC00BFEA
:1021400080BD00BF0018004080B500AF0B48FFF70E
:1021500003FF0346012B04D10848FFF7EFFE0CF004
:1021600097FA0748FFF7F8FE0346012B04D104480D
:10217000FFF7E4FE0BF0A8FE00BF80BD00040140A5
:10218000001C004080B500AF0648FFF7E5FE03469F
:10219000012B04D10348FFF7D1FE0CF09DF800BFDE
:1021A00080BD00BF0020004080B500AF05F092FA6E
:1021B00000BF80BD80B400AF01231846BD465DF866
:1021C000047B704780B582B000AF7860396022F040
:1021D000E9FA034616221A604FF0FF331846083713
:1021E000BD4680BD80B582B000AF78604FF0FF3152
:1021F0007868FFF7E7FFFEE780B483B000AF786050
:102200004FF0FF3318460C37BD465DF8047B70472E
:1022100080B483B000AF786039603B684FF40052FF
:102220005A60002318460C37BD465DF8047B7047A2
:1022300080B483B000AF7860012318460C37BD46E8
:102240005DF8047B704780B485B000AFF860B9607A
:102250007A60002318461437BD465DF8047B70474A
:1022600080B586B000AF7860144A154BD31A7B61F5
:102270007B693B61134B1B68002B02D1114B124A47
:102280001A60104B1A687B6813443A699A4207D265
:1022900022F088FA03460C221A604FF0FF3309E05F
:1022A000084B1B68FB60074B1A687B681344054AA0
:1022B0001360FB6818461837BD4680BD0000022039
:1022C00000040000F00F0020A856002080B400AFEA
:1022D000084BD3F88830074A43F47003C2F88830BB
:1022E000044B4FF000629A6000BFBD465DF8047B6E
:1022F000704700BF00ED00E080B400AF044BDB6826
:102300001B0A03F007031846BD465DF8047B7047BF
:1023100000ED00E080B483B000AF0346FB7197F995
:102320000730002B0BDBFB7903F01F02074997F9FD
:1023300007305B09012000FA02F241F8232000BFB8
:102340000C37BD465DF8047B704700BF00E100E03C
:1023500080B483B000AF03463960FB7197F9073052
:10236000002B0ADB3B68DAB20C4997F907301201FF
:10237000D2B20B4483F800230AE03B68DAB2084982
:10238000FB7903F00F03043B1201D2B20B441A761F
:1023900000BF0C37BD465DF8047B704700E100E0EC
:1023A00000ED00E080B489B000AFF860B9607A60F9
:1023B000FB6803F00703FB61FB69C3F10703042B10
:1023C00028BF0423BB61FB690433062B02D9FB69D8
:1023D000033B00E000237B614FF0FF32BB6902FA50
:1023E00003F3DA43BB681A407B699A404FF0FF3130
:1023F0007B6901FA03F3D9437B680B40134318460A
:102400002437BD465DF8047B7047000080B485B07A
:1024100000AF7860084B1A6C07497B6813430B6464
:10242000054B1A6C7B681340FB60FB6800BF1437D8
:10243000BD465DF8047B70470038024080B485B02B
:1024400000AF7860084B5A6C07497B6813434B64B4
:10245000054B5A6C7B681340FB60FB6800BF143768
:10246000BD465DF8047B70470038024080B483B0FD
:1024700000AF78607B681B6823F080027B681A607D
:1024800000BF0C37BD465DF8047B704780B483B055
:1024900000AF786039607B689B6823F4804323F049
:1024A00007033A681A437B689A6000BF0C37BD4641
:1024B0005DF8047B704780B483B000AF786039600A
:1024C0007B685B6823F070023B681A437B685A6044
:1024D00000BF0C37BD465DF8047B704780B483B005
:1024E00000AF78607B689B6823F080027B689A600D
:1024F00000BF0C37BD465DF8047B704780B586B0E1
:1025000000AF3B1D00221A605A609A60DA601A61BF
:102510000220FFF793FFFFF7EFFE034600220021A2
:102520001846FFF73FFF034619462B20FFF710FF21
:102530002B20FFF7EFFEFFF7DFFE0346002200210E
:102540001846FFF72FFF034619462C20FFF700FF20
:102550002C20FFF7DFFEFFF7CFFE0346002200210D
:102560001846FFF71FFF034619462D20FFF7F0FE20
:102570002D20FFF7CFFEB323BB800023BB60632376
:10258000FB6000233B6100233B753B1D19460A4855
:1025900002F086FC0848FFF769FF00210648FFF7B4
:1025A00075FF00210448FFF786FF0348FFF796FFF9
:1025B00000BF1837BD4680BD0004014080B586B01D
:1025C00000AF3B1D00221A605A609A60DA601A61FF
:1025D0004FF48030FFF732FFFFF78EFE03460022F4
:1025E00000211846FFF7DEFE034619461820FFF7C4
:1025F000AFFE1820FFF78EFE40F22B13BB800023A6
:10260000BB604FF6FF73FB6000233B613B1D194627
:10261000064802F045FC0548FFF728FF0021034863
:10262000FFF734FF00BF1837BD4680BD00400140B2
:1026300080B586B000AF3B1D00221A605A609A60D8
:10264000DA601A614FF40030FFF7F8FEFFF754FE2E
:102650000346002200211846FFF7A4FE0346194650
:102660001920FFF775FE1920FFF754FE40F22B13D7
:10267000BB800023BB604FF6FF73FB6000233B6110
:102680003B1D1946044802F00BFC0348FFF7EEFE21
:1026900000BF1837BD4680BD0044014080B586B0FC
:1026A00000AF3B1D00221A605A609A60DA601A611E
:1026B0004FF48020FFF7C2FEFFF71EFE0346002204
:1026C00000211846FFF76EFE034619461A20FFF751
:1026D0003FFE1A20FFF71EFE40F22B13BB800023A3
:1026E000BB604FF6FF73FB6000233B613B1D194647
:1026F000044802F0D5FB0348FFF7B8FE00BF1837C7
:10270000BD4680BD0048014080B586B000AF3B1D8E
:1027100000221A605A609A60DA601A614020FFF75E
:1027200075FEFFF7E9FD0346002200211846FFF77A
:1027300039FE034619462B20FFF70AFE2B20FFF730
:10274000E9FD40F22B13BB800023BB604FF6FF7303
:10275000FB6000233B613B1D1946074802F0A0FBCC
:102760000548FFF783FE00210348FFF78FFE00BFF7
:102770001837BD4680BD00BF0018004080B586B048
:1027800000AF3B1D00221A605A609A60DA601A613D
:102790008020FFF73BFEFFF7AFFD0346002200213C
:1027A0001846FFF7FFFD034619462C20FFF7D0FD22
:1027B0002C20FFF7AFFD40F22B13BB800023BB6042
:1027C0004FF6FF73FB6000233B613B1D1946054834
:1027D00002F066FB0348FFF749FE00BF1837BD460D
:1027E00080BD00BF001C004080B586B000AF3B1D1F
:1027F00000221A605A609A60DA601A614FF48070A1
:10280000FFF704FEFFF778FD03460022002118467B
:10281000FFF7C8FD034619462D20FFF799FD2D202F
:10282000FFF778FD40F22B13BB800023BB604FF60F
:10283000FF73FB6000233B613B1D1946044802F017
:102840002FFB0348FFF712FE00BF1837BD4680BDBF
:102850000020004080B400AF044BDB681B0A03F08B
:1028600007031846BD465DF8047B704700ED00E0A5
:1028700080B483B000AF0346FB7197F90730002B9B
:102880000BDBFB7903F01F02074997F907305B095F
:10289000012000FA02F241F8232000BF0C37BD46A8
:1028A0005DF8047B704700BF00E100E080B483B0B6
:1028B00000AF03463960FB7197F90730002B0ADB44
:1028C0003B68DAB20C4997F907301201D2B20B44D7
:1028D00083F800230AE03B68DAB20849FB7903F089
:1028E0000F03043B1201D2B20B441A7600BF0C371F
:1028F000BD465DF8047B704700E100E000ED00E0BC
:1029000080B489B000AFF860B9607A60FB6803F00A
:102910000703FB61FB69C3F10703042B28BF0423F2
:10292000BB61FB690433062B02D9FB69033B00E062
:1029300000237B614FF0FF32BB6902FA03F3DA43F5
:10294000BB681A407B699A404FF0FF317B6901FAFE
:1029500003F3D9437B680B40134318462437BD4625
:102960005DF8047B7047000080B485B000AF7860EC
:10297000084B1A6B07497B6813430B63054B1A6BB3
:102980007B681340FB60FB6800BF1437BD465DF8F1
:10299000047B70470038024080B485B000AF786097
:1029A000084B5A6C07497B6813434B64054B5A6CC0
:1029B0007B681340FB60FB6800BF1437BD465DF8C1
:1029C000047B70470038024080B483B000AF786069
:1029D0007B68DB6843F400527B68DA6000BF0C3729
:1029E000BD465DF8047B704780B483B000AF78606B
:1029F0007B681B6923F490427B681A617B685B6982
:102A000023F02A027B685A6100BF0C37BD465DF88F
:102A1000047B704780B58EB000AF07F11C03002225
:102A20001A605A609A60DA601A615A619A613B1DB5
:102A300000221A605A609A60DA601A615A611020A6
:102A4000FFF7AAFF0120FFF78FFF4FF4C0637B6001
:102A50000223BB600323FB6000233B6100237B61F7
:102A60000723BB613B1D1946184801F07DFFFFF7A6
:102A7000F1FE0346002200211846FFF741FF0346FE
:102A800019462520FFF712FF2520FFF7F1FE4FF42E
:102A9000E133FB6100233B6200237B620023BB62C6
:102AA0000C23FB6200233B6300237B6307F11C03C1
:102AB0001946074802F0F4FC0548FFF795FF044863
:102AC000FFF782FF00BF3837BD4680BD00000240DF
:102AD0000010014080B58EB000AF07F11C0300224A
:102AE0001A605A609A60DA601A615A619A613B1DF5
:102AF00000221A605A609A60DA601A615A612020D6
:102B0000FFF74AFF0420FFF72FFFC0237B6002235B
:102B1000BB600323FB6000233B6100237B61082330
:102B2000BB613B1D1946194801F01EFFFFF792FEDD
:102B30000346002200211846FFF7E2FE034619462D
:102B40004720FFF7B3FE4720FFF792FE4FF4E13333
:102B5000FB6100233B6200237B620023BB620C23EA
:102B6000FB6200233B6300237B6307F11C031946D0
:102B7000074802F095FC0648FFF736FF0448FFF7C8
:102B800023FF00BF3837BD4680BD00BF00080240AC
:102B900000140140DFF834D0002103E00C4B5B58F7
:102BA000435004310B480C4B42189A42F6D30B4A5F
:102BB00002E0002342F8043B094B9A42F9D3FFF7A5
:102BC00085FB21F0F5FDFEF767FF7047000002204E
:102BD0009CF8030800000020F00E0020F00E0020FA
:102BE000A4560020FEE7000080B500AF0E4B1B6826
:102BF0000D4A43F4007313600B4B1B680A4A43F4FD
:102C000080631360084B1B68074A43F480731360AA
:102C1000032000F0ABFF002000F008F8FFF740F9B8
:102C20000023184680BD00BF003C024080B582B042
:102C300000AF7860124B1A68124B1B7819464FF49C
:102C40007A73B3FBF1F3B2FBF3F3184600F0C3FF62
:102C50000346002B01D001230EE07B680F2B0AD81E
:102C6000002279684FF0FF3000F08BFF064A7B6846
:102C70001360002300E0012318460837BD4680BDDD
:102C800000000020080000200400002080B400AFF5
:102C9000064B1B781A46064B1B681344044A136004
:102CA00000BFBD465DF8047B704700BF08000020F0
:102CB000F40F002080B400AF034B1B681846BD46DC
:102CC0005DF8047B704700BFF40F002080B584B02E
:102CD00000AF78607B68002B01D10123EDE07B68B9
:102CE00093F82030DBB2002B02D17868FEF766F94A
:102CF0007B681B681A687B681B6822F002021A60F6
:102D0000FFF7D8FFF86012E0FFF7D4FF0246FB6838
:102D1000D31A0A2B0BD97B685B6A43F400327B68B9
:102D20005A627B68052283F820200123C5E07B6876
:102D30001B685B6803F00203002BE5D17B681B680E
:102D40001A687B681B6842F001021A60FFF7B2FF45
:102D5000F86012E0FFF7AEFF0246FB68D31A0A2BB9
:102D60000BD97B685B6A43F400327B685A627B68EC
:102D7000052283F8202001239FE07B681B685B68A5
:102D800003F00103002BE5D07B681B7E012B08D1EB
:102D90007B681B681A687B681B6842F080021A60B7
:102DA00007E07B681B681A687B681B6822F080025A
:102DB0001A607B685B7E012B08D17B681B681A68F0
:102DC0007B681B6842F040021A6007E07B681B6862
:102DD0001A687B681B6822F040021A607B689B7E41
:102DE000012B08D17B681B681A687B681B6842F05E
:102DF00020021A6007E07B681B681A687B681B6802
:102E000022F020021A607B68DB7E012B08D17B68F0
:102E10001B681A687B681B6822F010021A6007E0C2
:102E20007B681B681A687B681B6842F010021A6096
:102E30007B681B7F012B08D17B681B681A687B6845
:102E40001B6842F008021A6007E07B681B681A687A
:102E50007B681B6822F008021A607B685B7F012B8D
:102E600008D17B681B681A687B681B6842F0040203
:102E70001A6007E07B681B681A687B681B6822F091
:102E800004021A607B689A687B68DB681A437B6877
:102E90001B691A437B685B6942EA03017B685B68D4
:102EA0005A1E7B681B680A43DA617B6800225A62FB
:102EB0007B68012283F82020002318461037BD4686
:102EC00080BD000080B487B000AF786039607B6857
:102ED0001B687B617B6893F82030FB74FB7C012BC3
:102EE00003D0FB7C022B40F0BE80654B7B617B698D
:102EF000D3F8003243F001027B69C3F800227B69FA
:102F0000D3F8003223F47C527B69C3F800227B693A
:102F1000D3F800223B685B6A1B021A437B69C3F843
:102F200000223B685B6903F01F03012202FA03F3EE
:102F3000FB607B69D3F81C22FB68DB431A407B698A
:102F4000C3F81C223B68DB69002B23D17B69D3F8D3
:102F50000C22FB68DB431A407B69C3F80C223B68F8
:102F6000DB6819043B685B689BB23A685269194395
:102F70007B69483243F832103B689B6819043B6810
:102F80001B689AB23B685B690A4379694833DB0086
:102F90000B445A603B68DB69012B22D17B69D3F873
:102FA0000C22FB681A437B69C3F80C223B681B6840
:102FB00019043B685B689BB23A68526919437B69A4
:102FC000483243F832103B689B6819043B68DB6861
:102FD0009AB23B685B690A4379694833DB000B446A
:102FE0005A603B689B69002B09D17B69D3F80422A6
:102FF000FB68DB431A407B69C3F8042207E07B6966
:10300000D3F80422FB681A437B69C3F804223B68A7
:103010001B69002B09D17B69D3F81422FB68DB43C1
:103020001A407B69C3F8142207E07B69D3F81422A5
:10303000FB681A437B69C3F814223B681B6A012BA7
:1030400007D17B69D3F81C22FB681A437B69C3F85C
:103050001C227B69D3F8003223F001027B69C3F89C
:103060000022002306E07B685B6A43F480227B68D1
:103070005A62012318461C37BD465DF8047B704731
:103080000064004080B584B000AF78607B6893F83E
:103090002030DBB2012B2ED17B68022283F8202066
:1030A0007B681B681A687B681B6822F001021A6043
:1030B000FFF700FEF86012E0FFF7FCFD0246FB6838
:1030C000D31A0A2B0BD97B685B6A43F400327B6806
:1030D0005A627B68052283F82020012312E07B6876
:1030E0001B685B6803F00103002BE5D17B680022BD
:1030F0005A62002306E07B685B6A43F400227B6827
:103100005A62012318461037BD4680BD80B489B08D
:1031100000AFF860B9607A603B60FB6893F82030DC
:10312000FB77FB681B689B68BB61FB7F012B03D0AF
:10313000FB7F022B40F0B880BB6903F08063002B5B
:103140000AD1BB6903F00063002B05D1BB6903F012
:103150008053002B00F0A080BB691B0E03F003031B
:103160007B617B69022B07D9FB685B6A43F4000231
:10317000FB685A6201239EE001227B699A403B680A
:103180001A60BB689B68002B0DD1BB681B685A0591
:10319000BB68DB68F96809681A437B6918331B014F
:1031A0000B441A600FE0BB685B68DA00BB689B6881
:1031B0001A43BB68DB68F96809681A437B691833EE
:1031C0001B010B441A60FB681968BB681A697B69AC
:1031D00018331B010B4404331A60BB681B7D012BA1
:1031E00011D1FB681A687B6918331B01134404333F
:1031F0001B68FA68116843F480727B6918331B01FD
:103200000B4404331A607B6807331B781A067B680B
:1032100006331B781B041A437B6805331B781B029B
:1032200013437A68043212781046FA68116843EA48
:1032300000027B691B010B4403F5C6731A607B68AF
:1032400003331B781A067B6802331B781B041A436E
:103250007B6801331B781B0213437A68127810468F
:10326000FA68116843EA00027B691B010B4403F50D
:10327000C4731A60FB681A687B6918331B01134416
:103280001B68FA68116843F001027B6918331B015F
:103290000B441A6000230EE0FB685B6A43F40012E3
:1032A000FB685A62012306E0FB685B6A43F48022F4
:1032B000FB685A62012318462437BD465DF8047B3B
:1032C000704780B487B000AFF860B9607A603B6047
:1032D000FB6893F82030FB75FB7D012B03D0FB7D51
:1032E000022B40F0F380BB68002B0ED1FB681B68FB
:1032F000DB6803F00303002B16D1FB685B6A43F421
:103300000012FB685A620123E7E0FB681B681B6937
:1033100003F00303002B07D1FB685B6A43F4001240
:10332000FB685A620123D8E0FB681A68BB681B334C
:103330001B0113441B6803F004027B689A607B68DE
:103340009B68002B0CD1FB681A68BB681B331B0100
:1033500013441B685B0DC3F30A027B681A600BE021
:10336000FB681A68BB681B331B0113441B68DB082E
:1033700023F060427B685A60FB681A68BB681B33A5
:103380001B0113441B6803F002027B68DA60FB68D0
:103390001A68BB681B331B01134404331B6803F01A
:1033A0000F027B681A61FB681A68BB681B331B013C
:1033B000134404331B681B0ADAB27B689A61FB680A
:1033C0001A68BB681B331B01134404331B681B0CB6
:1033D0009AB27B685A61FB681A68BB681B01134488
:1033E00003F5DC731B68DAB23B681A70FB681A6875
:1033F000BB681B01134403F5DC731B681A0A3B68A6
:103400000133D2B21A70FB681A68BB681B011344FF
:1034100003F5DC731B681A0C3B680233D2B21A70D6
:10342000FB681A68BB681B01134403F5DC731B6857
:103430001A0E3B680333D2B21A70FB681A68BB6875
:103440001B01134403F5DE731A683B680433D2B2E0
:103450001A70FB681A68BB681B01134403F5DE731E
:103460001B681A0A3B680533D2B21A70FB681A68E7
:10347000BB681B01134403F5DE731B681A0C3B6821
:103480000633D2B21A70FB681A68BB681B0113447A
:1034900003F5DE731B681A0E3B680733D2B21A704D
:1034A000BB68002B08D1FB681B68DA68FB681B68E7
:1034B00042F02002DA6007E0FB681B681A69FB68CB
:1034C0001B6842F020021A61002306E0FB685B6A79
:1034D00043F48022FB685A62012318461C37BD461C
:1034E0005DF8047B704780B485B000AF78603960C8
:1034F0000023FB607B6893F82030FB72FB7A012B82
:1035000002D0FB7A022B0FD13B68002B06D17B68DF
:103510001B68DB6803F00303FB6005E07B681B6846
:103520001B6903F00303FB60FB6818461437BD46B4
:103530005DF8047B704780B485B000AF7860396077
:103540007B6893F82030FB73FB7B012B02D0FB7B65
:10355000022B09D17B681B6859697B681B683A6834
:103560000A435A61002306E07B685B6A43F48022C9
:103570007B685A62012318461437BD465DF8047B08
:10358000704780B485B000AF786039607B6893F88D
:103590002030FB73FB7B012B02D0FB7B022B0AD17B
:1035A0007B681B6859693B68DA437B681B680A4083
:1035B0005A61002306E07B685B6A43F480227B68E3
:1035C0005A62012318461437BD465DF8047B7047E4
:1035D00080B58AB000AF786000237B627B681B688F
:1035E0005B693B627B681B685B68FB617B681B688F
:1035F0009B68BB617B681B68DB687B617B681B68C1
:103600001B693B617B681B689B69FB603B6A03F03D
:103610000103002B7CD0BB6903F00103002B23D0F6
:103620007B681B6801229A60BB6903F00203002BD0
:1036300003D0786802F050FD16E0BB6903F0040384
:10364000002B04D07B6A43F400637B620CE0BB690F
:1036500003F00803002B04D07B6A43F480537B62A1
:1036600002E0786800F06BF9BB6903F48073002B0B
:1036700024D07B681B684FF480729A60BB6903F4A6
:103680000073002B03D0786802F030FD16E0BB69B0
:1036900003F48063002B04D07B6A43F400537B6205
:1036A0000CE0BB6903F40063002B04D07B6A43F495
:1036B00080437B6202E0786800F04BF9BB6903F459
:1036C0008033002B24D07B681B684FF480329A60D3
:1036D000BB6903F40033002B03D0786802F010FDBF
:1036E00016E0BB6903F48023002B04D07B6A43F40B
:1036F00000437B620CE0BB6903F40023002B04D081
:103700007B6A43F480337B6202E0786800F02BF937
:103710003B6A03F00803002B0CD07B6903F0100315
:10372000002B07D07B6A43F400737B627B681B68C5
:103730001022DA603B6A03F00403002B0BD07B6994
:1037400003F00803002B06D07B681B680822DA60B0
:10375000786802F0E9FC3B6A03F00203002B09D011
:103760007B681B68DB6803F00303002B02D07868DA
:1037700002F0D0FC3B6A03F04003002B0CD03B6905
:1037800003F01003002B07D07B6A43F480637B6255
:103790007B681B6810221A613B6A03F02003002B30
:1037A0000BD03B6903F00803002B06D07B681B6835
:1037B00008221A61786800F0EAF83B6A03F0100307
:1037C000002B09D07B681B681B6903F00303002BE7
:1037D00002D0786800F0D1F83B6A03F40033002B84
:1037E0000BD0FB6903F01003002B06D07B681B682D
:1037F00010225A60786800F0D4F83B6A03F48033F2
:10380000002B0BD0FB6903F00803002B06D07B686C
:103810001B6808225A60786800F0CDF83B6A03F410
:103820000043002B7BD0FB6903F00403002B72D014
:103830003B6A03F48073002B08D0FB6803F001039C
:10384000002B03D07B6A43F001037B623B6A03F4E5
:103850000073002B08D0FB6803F00203002B03D099
:103860007B6A43F002037B623B6A03F48063002BB4
:1038700008D0FB6803F00403002B03D07B6A43F0FD
:1038800004037B623B6A03F40063002B43D0FB68B4
:1038900003F07003002B3ED0FB6803F07003602B35
:1038A0002BD0602B2ED8502B22D0502B2AD8402B37
:1038B00019D0402B26D8302B10D0302B22D8102BEB
:1038C00002D0202B05D01DE07B6A43F008037B6209
:1038D00019E07B6A43F010037B6214E07B6A43F0DB
:1038E00020037B620FE07B6A43F040037B620AE0C7
:1038F0007B6A43F080037B6205E07B6A43F480735C
:103900007B6200E000BF7B681B689A697B681B686C
:1039100022F070029A617B681B6804225A607B6AFD
:10392000002B08D07B685A6A7B6A1A437B685A620C
:10393000786802F007FC00BF2837BD4680BD80B420
:1039400083B000AF786000BF0C37BD465DF8047BE4
:10395000704780B483B000AF786000BF0C37BD46BD
:103960005DF8047B704780B483B000AF786000BF1F
:103970000C37BD465DF8047B704780B483B000AF60
:10398000786000BF0C37BD465DF8047B704780B49B
:1039900083B000AF786000BF0C37BD465DF8047B94
:1039A000704780B483B000AF786000BF0C37BD466D
:1039B0005DF8047B704780B483B000AF786000BFCF
:1039C0000C37BD465DF8047B7047000080B485B0BD
:1039D00000AF78607B6803F00703FB600C4BDB688B
:1039E000BB60BA684FF6FF031340BB60FB681A0266
:1039F000BB68134343F0BF6343F40033BB60044A26
:103A0000BB68D36000BF1437BD465DF8047B7047C8
:103A100000ED00E080B400AF044BDB681B0A03F04C
:103A200007031846BD465DF8047B704700ED00E0D3
:103A300080B483B000AF0346FB7197F90730002BC9
:103A40000BDBFB7903F01F02074997F907305B098D
:103A5000012000FA02F241F8232000BF0C37BD46D6
:103A60005DF8047B704700BF00E100E080B483B0E4
:103A700000AF03463960FB7197F90730002B0ADB72
:103A80003B68DAB20C4997F907301201D2B20B4405
:103A900083F800230AE03B68DAB20849FB7903F0B7
:103AA0000F03043B1201D2B20B441A7600BF0C374D
:103AB000BD465DF8047B704700E100E000ED00E0EA
:103AC00080B489B000AFF860B9607A60FB6803F039
:103AD0000703FB61FB69C3F10703042B28BF042321
:103AE000BB61FB690433062B02D9FB69033B00E091
:103AF00000237B614FF0FF32BB6902FA03F3DA4324
:103B0000BB681A407B699A404FF0FF317B6901FA2C
:103B100003F3D9437B680B40134318462437BD4653
:103B20005DF8047B7047000080B582B000AF78601C
:103B30007B68013BB3F1807F01D301230FE00A4A88
:103B40007B68013B53600F214FF0FF30FFF78EFF82
:103B5000054B00229A60044B07221A600023184686
:103B60000837BD4680BD00BF10E000E080B582B0E0
:103B700000AF78607868FFF729FF00BF0837BD46BF
:103B800080BD80B586B000AF0346B9607A60FB7334
:103B900000237B61FFF73EFF78617A68B968786936
:103BA000FFF78EFF024697F90F3011461846FFF7D0
:103BB0005DFF00BF1837BD4680BD80B582B000AF45
:103BC0000346FB7197F907301846FFF731FF00BF36
:103BD0000837BD4680BD80B582B000AF7860786898
:103BE000FFF7A2FF034618460837BD4680BD000018
:103BF00080B489B000AF7860396000237B61002316
:103C00003B610023BB610023FB6165E10122FB698D
:103C100002FA03F37B613B681B687A6913403B61DE
:103C20003A697B699A4240F054813B685B68012B9A
:103C30000BD03B685B68022B07D03B685B68112B9D
:103C400003D03B685B68122B30D17B689B68BB61FB
:103C5000FB695B00032202FA03F3DB43BA691340FA
:103C6000BB613B68DA68FB695B0002FA03F3BA697F
:103C70001343BB617B68BA699A607B685B68BB6110
:103C80000122FB6902FA03F3DB43BA691340BB610B
:103C90003B685B681B0903F00102FB6902FA03F34E
:103CA000BA691343BB617B68BA695A607B68DB6899
:103CB000BB61FB695B00032202FA03F3DB43BA69D1
:103CC0001340BB613B689A68FB695B0002FA03F32F
:103CD000BA691343BB617B68BA69DA603B685B68A9
:103CE000022B03D03B685B68122B23D1FB69DA08F7
:103CF0007B68083253F82230BB61FB6903F007038D
:103D00009B000F2202FA03F3DB43BA691340BB6145
:103D10003B681A69FB6903F007039B0002FA03F38F
:103D2000BA691343BB61FB69DA087B680832B96979
:103D300043F822107B681B68BB61FB695B000322B0
:103D400002FA03F3DB43BA691340BB613B685B686B
:103D500003F00302FB695B0002FA03F3BA69134341
:103D6000BB617B68BA691A603B685B6803F080538B
:103D7000002B00F0AE800023FB605D4B5B6C5C4A67
:103D800043F4804353645A4B5B6C03F48043FB6001
:103D9000FB68584AFB699B08023352F82330BB6129
:103DA000FB6903F003039B000F2202FA03F3DB43DA
:103DB000BA691340BB617B684F4A934225D07B6848
:103DC0004E4A93421FD07B684D4A934219D07B687C
:103DD0004C4A934213D07B684B4A93420DD07B6888
:103DE0004A4A934207D07B68494A934201D106234D
:103DF0000CE007230AE0052308E0042306E0032380
:103E000004E0022302E0012300E00023FA6902F04B
:103E1000030292009340BA691343BB613549FB69C1
:103E20009B080233BA6941F823203A4B1B68BB61F7
:103E30003B69DB43BA691340BB613B685B6803F4D1
:103E40008033002B03D0BA693B691343BB61314A0D
:103E5000BB6913602F4B5B68BB613B69DB43BA698D
:103E60001340BB613B685B6803F40033002B03D055
:103E7000BA693B691343BB61264ABB695360254B52
:103E80009B68BB613B69DB43BA691340BB613B681C
:103E90005B6803F48013002B03D0BA693B691343BA
:103EA000BB611C4ABB6993601A4BDB68BB613B6911
:103EB000DB43BA691340BB613B685B6803F40013E2
:103EC000002B03D0BA693B691343BB61114ABB693C
:103ED000D360FB690133FB61FB690F2B7FF696AE64
:103EE00000BF00BF2437BD465DF8047B704700BFAC
:103EF0000038024000380140000002400004024047
:103F000000080240000C0240001002400014024071
:103F100000180240003C014080B582B000AF7860DC
:103F200039607B68002B01D1012325E07B6893F881
:103F30002C30DBB2002B06D17B68002283F82D20C9
:103F40007868FDF71DFA7B68022283F82C207B68D5
:103F50001A687B6804331946104600F0BFFA7B6884
:103F600018687B685B681A46396800F02AFB7B6832
:103F7000012283F82C20002318460837BD4680BD57
:103F800080B584B000AFF860B9607A60FB6893F8E0
:103F90002C30DBB2022B01D1022318E0FB68022295
:103FA00083F82C20FB681B687A68B968184600F013
:103FB00087FBBB681B68022B04D1FB68052283F8D2
:103FC0002C2003E0FB68012283F82C2000231846F4
:103FD0001037BD4680BD80B582B000AF78603960D3
:103FE0007B6893F82C30DBB2022B01D102230EE068
:103FF0007B68022283F82C207B681B68396818468E
:1040000000F09AFB7B68012283F82C2000231846DD
:104010000837BD4680BD80B584B000AFF860B96098
:104020007A60FB68002B01D1012334E0FB6893F830
:104030004930DBB2002B06D1FB68002283F8482010
:10404000F868FDF793F9FB681A68FB6808331946AE
:10405000104600F03FF9FB681868FB689B681A4639
:10406000B96800F0A7F9FB685868FB689A68FB68B4
:104070001B6B796800F0F2F9FB681B68FA689268BC
:1040800053F82210FB681B68FA68926841F001013E
:1040900043F82210002318461037BD4680BD0000AB
:1040A00080B483B000AF7860054B1A6804497B6820
:1040B00013430B6000BF0C37BD465DF8047B7047AF
:1040C000003C014080B483B000AF7860064B1A68B2
:1040D0007B68DB43044913400B6000BF0C37BD46CF
:1040E0005DF8047B704700BF003C014080B483B0A2
:1040F00000AF7860054B5A6804497B6813434B60F6
:1041000000BF0C37BD465DF8047B7047003C0140A2
:1041100080B483B000AF7860064B5A687B68DB439D
:10412000044913404B6000BF0C37BD465DF8047B6B
:10413000704700BF003C014080B483B000AF78609E
:10414000054B9A6804497B6813438B6000BF0C37AA
:10415000BD465DF8047B7047003C014080B483B0ED
:1041600000AF7860064B9A687B68DB4304491340D4
:104170008B6000BF0C37BD465DF8047B704700BF05
:10418000003C014080B483B000AF7860054BDA6832
:1041900004497B681343CB6000BF0C37BD465DF814
:1041A000047B7047003C014080B483B000AF78606E
:1041B000064BDA687B68DB4304491340CB6000BFE1
:1041C0000C37BD465DF8047B704700BF003C0140E2
:1041D00080B584B000AF78600023FB737B681B79E7
:1041E000002B65D07B681B68002B6CD07B685B79EB
:1041F000022B1CD0022B25DC002B02D0012B0BD074
:1042000020E07B681B681846FFF782FF7B681B680D
:104210001846FFF745FF18E07B681B681846FFF754
:1042200051FF7B681B681846FFF760FF0DE07B6855
:104230001B681846FFF734FF7B681B681846FFF7BA
:1042400055FF02E00123FB7300BF7B689B79002BC5
:1042500039D07B689B79032B1CD0032B25DC012BE9
:1042600002D0022B0BD020E07B681B681846FFF7BA
:104270009BFF7B681B681846FFF75EFF24E07B68A6
:104280001B681846FFF76AFF7B681B681846FFF734
:1042900079FF19E07B681B681846FFF74DFF7B68C4
:1042A0001B681846FFF76EFF0EE00123FB730BE05F
:1042B0007B681B681846FFF705FF7B681B6818467C
:1042C000FFF726FF00E000BFFB7B18461037BD4616
:1042D00080BD000080B485B000AF786039600023F5
:1042E000FB603B681A687B6853F82230FB60FA6811
:1042F0002F4B1340FB603B685A683B689B681A432E
:104300003B68DB681A433B681B691A433B685B697F
:104310001A433B68DB691A433B681B6A1A433B68D4
:104320005B6A1A433B689B6A1A433B68DB6A1A4321
:104330003B681B6B1A433B685B6B1A433B68DB6B48
:104340001A433B689B6B1343FA681343FB603B685B
:104350009B68082B03D1FB6843F04003FB603B687C
:104360001A687B68F96843F822103B685B6BB3F509
:10437000801F0AD13B681B68002B06D07B681A6837
:104380003B685B6B1A437B681A603B681B68002BB9
:1043900006D07B681A683B689B6B1A437B681A607F
:1043A000002318461437BD465DF8047B704700BFF4
:1043B0008004C0FF80B487B000AFF860B9607A6055
:1043C00000237B617B685A1CFB6853F822307B61B9
:1043D0007B6903F040437B61BB681A68BB685B681C
:1043E0001B011A43BB689B681B021A43BB68DB684E
:1043F0001B041A43BB681B69013B1B051A43BB68BE
:104400005B69023B1B061A43BB689B6913437A69CD
:1044100013437B617B685A1CFB68796943F822105F
:10442000FB681B6803F48013B3F5801F0ED1FB6893
:104430005B6823F470037B61BB681B69013B1B0550
:104440007A6913437B61FB687A695A6000231846D6
:104450001C37BD465DF8047B7047000080B487B010
:1044600000AFF860B9607A603B6000237B613B6815
:10447000B3F5804F22D1FB687A6853F822307B6114
:104480007A69154B13407B61BB681A68BB685B682F
:104490001B011A43BB689B681B021A43BB68DB689D
:1044A0001B041A43BB689B6913437A6913437B61FE
:1044B000FB687A68796943F8221005E0FB687A683E
:1044C0006FF0704143F82210002318461C37BD4698
:1044D0005DF8047B704700BF0000F0CF80B485B06A
:1044E00000AF786039600023FB600023BB603B684D
:1044F0001B68012B29D07B681B68FB60FB6823F4D9
:10450000FF4323F07F03FB603B685A683B689B686E
:104510001A433B68DB681A433B681B691A433B68D4
:104520005B691A433B689B691A433B68DB691A4322
:104530003B681B6A1A433B685B6A1343FA68134380
:10454000FB607B68FA681A6034E07B681B68FB607C
:10455000FB6823F4F843FB603B68DA693B681B6A3D
:104560001A433B685B6A1343FA681343FB607B683A
:104570005B68BB60BB6823F4FF4323F07F03BB6031
:104580003B685A683B689B681A433B68DB681A4380
:104590003B681B691A433B685B691A433B689B692C
:1045A0001343BA681343BB607B68FA681A607B6880
:1045B000BA685A60002318461437BD465DF8047B7C
:1045C000704780B487B000AFF860B9607A600023AC
:1045D0007B6100233B617B68012B2ED0FB689B68CD
:1045E0007B617B6903F070437B61BB681B685A1E6B
:1045F000BB685B68013B1B011A43BB689B68013BBE
:104600001B021A43BB68DB68013B1B031A43BB68F0
:104610001B69013B1B041A43BB685B69013B1B051B
:104620001A43BB689B69013B1B0613437A6913431A
:104630007B61FB687A699A603BE0FB689B687B6101
:104640007B6923F4700323F470437B61BB68DB68F0
:10465000013B1A03BB685B69013B1B0513437A6985
:1046600013437B61FB68DB683B613B6903F070438C
:104670003B61BB681B685A1EBB685B68013B1B0142
:104680001A43BB689B68013B1B021A43BB681B694A
:10469000013B1B041A43BB689B69013B1B06134388
:1046A0003A6913433B61FB687A699A60FB683A692F
:1046B000DA60002318461C37BD465DF8047B70475E
:1046C00080B586B000AFF860B9607A6000233B61C6
:1046D00000237B61BB681A68BB685B681A43BB68D0
:1046E0009B68013B5B011A43BB68DB685B021343B9
:1046F0003B613A69FB681A61FEF7DCFA786110E009
:104700007B68B3F1FF3F0CD07B68002B07D0FEF72E
:10471000D1FA02467B69D31A7A689A4201D20323FE
:1047200006E0FB689B6903F02003202BE8D0002300
:1047300018461837BD4680BD80B483B000AF78609E
:1047400039607B685A693B685B001A437B685A6131
:10475000002318460C37BD465DF8047B704780B4D3
:1047600089B000AFF860B9607A60FB681A68BB680E
:104770007B617B6993FAA3F33B613B69B3FA83F3F3
:10478000DBB25B00032101FA03F3DB431A40BB6891
:10479000FB61FB6993FAA3F3BB61BB69B3FA83F3D3
:1047A000DBB25B00796801FA03F31A43FB681A6015
:1047B00000BF2437BD465DF8047B704780B485B0E8
:1047C00000AFF860B9607A60FB685A68BB68DB4389
:1047D0001A40BB68796801FB03F31A43FB685A600F
:1047E00000BF1437BD465DF8047B704780B489B0C4
:1047F00000AFF860B9607A60FB689A68BB687B615B
:104800007B6993FAA3F33B613B69B3FA83F3DBB2B1
:104810005B00032101FA03F3DB431A40BB68FB6131
:10482000FB6993FAA3F3BB61BB69B3FA83F3DBB211
:104830005B00796801FA03F31A43FB689A6000BFD2
:104840002437BD465DF8047B704780B489B000AF63
:10485000F860B9607A60FB68DA68BB687B617B6985
:1048600093FAA3F33B613B69B3FA83F3DBB25B00DA
:10487000032101FA03F3DB431A40BB68FB61FB69C8
:1048800093FAA3F3BB61BB69B3FA83F3DBB25B00BA
:10489000796801FA03F31A43FB68DA6000BF243732
:1048A000BD465DF8047B704780B489B000AFF86006
:1048B000B9607A60FB681A6ABB687B617B6993FAAE
:1048C000A3F33B613B69B3FA83F3DBB29B000F2197
:1048D00001FA03F3DB431A40BB68FB61FB6993FAFF
:1048E000A3F3BB61BB69B3FA83F3DBB29B007968C6
:1048F00001FA03F31A43FB681A6200BF2437BD466E
:104900005DF8047B704780B489B000AFF860B9608F
:104910007A60FB685A6ABB681B0A7B617B6993FA01
:10492000A3F33B613B69B3FA83F3DBB29B000F2136
:1049300001FA03F3DB431A40BB681B0AFB61FB6906
:1049400093FAA3F3BB61BB69B3FA83F3DBB29B00B9
:10495000796801FA03F31A43FB685A6200BF2437EF
:10496000BD465DF8047B704780B588B000AF7860C5
:1049700039600023FB610023BB613B681B687B61DE
:104980007B6993FAA3F33B613B69B3FA83F3DBB230
:10499000FB6150E03B681A680121FB6901FA03F3EF
:1049A0001340BB61BB69002B42D03B685B68012BA5
:1049B00003D03B685B68022B0DD13B689B681A46AD
:1049C000B9697868FFF712FF3B68DB681A46B96976
:1049D0007868FFF7F3FE3B681B691A46B969786887
:1049E000FFF733FF3B685B68022B1AD1BB69FB60A2
:1049F000FB6893FAA3F3BB60BB68B3FA83F3DBB243
:104A0000072B07D83B685B691A46B9697868FFF7D6
:104A10004BFF06E03B685B691A46B9697868FFF7A7
:104A200072FF3B685B681A46B9697868FFF797FEC2
:104A3000FB690133FB613B681A68FB6922FA03F3E7
:104A4000002BA7D1002318462037BD4680BD0000AB
:104A500080B400AF044B9B6803F00C031846BD46BE
:104A60005DF8047B704700BF0038024080B400AF9F
:104A7000044B9B6803F0F0031846BD465DF8047BC9
:104A8000704700BF0038024080B400AF044B9B6801
:104A900003F4E0531846BD465DF8047B704700BF41
:104AA0000038024080B400AF044B9B6803F46043BD
:104AB0001846BD465DF8047B704700BF00380240D1
:104AC00080B400AF044B5B6803F480031846BD4616
:104AD0005DF8047B704700BF0038024080B400AF2F
:104AE000044B5B689B09C3F308031846BD465DF899
:104AF000047B70470038024080B400AF044B5B6811
:104B000003F440331846BD465DF8047B704700BF90
:104B10000038024080B400AF044B5B6803F0E04310
:104B20001846BD465DF8047B704700BF0038024060
:104B300080B400AF044B5B6803F03F031846BD46EA
:104B40005DF8047B704700BF0038024080B582B03A
:104B500000AF786000F020F802467B681A607B683E
:104B60001B68184600F05CF802467B685A607B6858
:104B70005B68184600F06AF802467B689A607B68BA
:104B80005B68184600F076F802467B68DA6000BF82
:104B90000837BD4680BD000080B582B000AF00235D
:104BA0007B60FFF755FF03460C2B2DD801A252F86E
:104BB00023F000BFE94B0108094C0108094C01082A
:104BC000094C0108EF4B0108094C0108094C010888
:104BD000094C0108F54B0108094C0108094C010872
:104BE000094C0108FF4B01080B4B7B600FE00B4B9E
:104BF0007B600CE0082000F051F8786007E00C20A2
:104C000000F04CF8786002E0034B7B6000BF7B68EB
:104C100018460837BD4680BD0024F400001BB700CD
:104C200080B582B000AF7860FFF720FF03461B0914
:104C300003F00F03044AD35C1A467B68D34018463E
:104C40000837BD4680BD00BF84CA030880B582B066
:104C500000AF7860FFF718FF03469B0A044AD35C55
:104C60001A467B68D34018460837BD4680BD00BF52
:104C700094CA030880B582B000AF7860FFF712FFD6
:104C800003465B0B044AD35C1A467B68D340184644
:104C90000837BD4680BD00BF94CA030890B587B0F1
:104CA00000AF786000237B610023FB6000233B6141
:104CB000FFF706FFF860FB68002B04D0FB68B3F534
:104CC000800F03D005E01C4B7B6105E01B4B7B6133
:104CD00002E0194B7B6100BF7B68082B14D1FFF702
:104CE00027FF02467B69B3FBF2F4FFF7F7FE0346AA
:104CF00003FB04F4FFF700FF03461B0C01335B00CA
:104D0000B4FBF3F33B6111E0FFF712FF02467B694E
:104D1000B3FBF2F4FFF7E2FE034603FB04F4FFF7F4
:104D2000F9FE03461B0FB4FBF3F33B613B691846E6
:104D30001C37BD4690BD00BF0024F400001BB70027
:104D400080B483B000AF78607B681B6803F04003D9
:104D5000402B01D1012300E0002318460C37BD464B
:104D60005DF8047B704780B483B000AF7860396031
:104D70003B689BB21A467B681A6100BF0C37BD4680
:104D80005DF8047B704780B584B000AF786039600F
:104D90000123FB737868FFF7D3FF0346002B39D15B
:104DA0007B681B6823F47F4323F0BF033A681168D4
:104DB0003A68526811433A68926811433A68D26877
:104DC00011433A68126911433A68526911433A68CB
:104DD000926911433A68D26911433A68126A0A43E8
:104DE0001A437B681A607B685B6823F004023B68A7
:104DF0005B691B0C1A437B685A603B681B6AB3F5FE
:104E0000005F05D13B685B6A19467868FFF7ABFF26
:104E10000023FB737B68DB6923F400627B68DA6143
:104E2000FB7B18461037BD4680BD80B483B000AF11
:104E3000786039607B683A689A6200BF0C37BD467B
:104E40005DF8047B704780B483B000AF7860396050
:104E50007B683A68DA6200BF0C37BD465DF8047BB8
:104E6000704780B483B000AF786039607B683A687F
:104E70001A6300BF0C37BD465DF8047B704780B4F1
:104E800083B000AF78607B685B6943F001027B68A8
:104E90005A6100BF0C37BD465DF8047B70470000C7
:104EA00080B584B000AF786039607B681B68FB60B8
:104EB0007B683D4A934213D07B68B3F1804F0FD09B
:104EC0007B683A4A93420BD07B68394A934207D0B9
:104ED0007B68384A934203D07B68374A934206D1B5
:104EE000FB6823F070023B685B681343FB607B68E0
:104EF0002D4A93422BD07B68B3F1804F27D07B683B
:104F00002A4A934223D07B68294A93421FD07B6868
:104F1000284A93421BD07B68274A934217D07B686C
:104F2000264A934213D07B68254A93420FD07B6870
:104F3000244A93420BD07B68234A934207D07B6874
:104F4000224A934203D07B68214A934206D1FB68F0
:104F500023F440723B68DB681343FB607B68FA68AC
:104F60001A603B689B6819467868FFF76CFF3B68DE
:104F70001B8819467868FFF758FF7B680A4A9342F6
:104F800003D07B680C4A934205D13B681B7C1946D1
:104F90007868FFF766FF7868FFF771FF002318460F
:104FA0001037BD4680BD00BF000001400004004036
:104FB00000080040000C0040000401400040014097
:104FC000004401400048014000180040001C00401F
:104FD0000020004080B483B000AF78607B68DB685D
:104FE00003F40053B3F5005F0CBF01230023DBB2D1
:104FF00018460C37BD465DF8047B704780B483B01B
:1050000000AF786039607B681B6923F440523B68CD
:105010001A437B681A6100BF0C37BD465DF8047BFC
:10502000704780B483B000AF786039607B685B699B
:1050300023F440723B681A437B685A6100BF0C3707
:10504000BD465DF8047B70472DE9B04FC0B000AF9E
:10505000C7F8FC00C7F8F810C7F8F420C7F8F0301C
:10506000D7F8F430B3F5004F40F00C81D7F8F830A2
:105070000022C7F8E830C7F8EC20D7E93A452246C5
:105080002B46911839665B417B66D7E91823214688
:1050900012EB0108294643EB01094FF000024FF0E3
:1050A00000034FEAC90343EA58734FEAC802904627
:1050B0009946234618EB0303C7F8E0302B4649EB2B
:1050C0000303C7F8E430D7F8F03000229A4693463D
:1050D0001AEB0A03BB654BEB0B03FB65D7E9162301
:1050E000D7E93801FBF7B0FD02460B46644BA3FB42
:1050F00002235B099BB21B019CB2D7F8F830002257
:10510000C7F8D830C7F8DC20D7E9368942464B4685
:10511000911839655B417B65D7E9142341465118E5
:10512000B96449464B41FB644FF000024FF0000365
:10513000D7E912AB5946CB00514643EA5173514669
:10514000CA0010461946034642469B18C7F8D0309D
:105150004B460A4642EB0303C7F8D430D7F8F03089
:105160000022C7F8C830C7F8CC20D7E932120B4666
:10517000DB183B64134642EB03037B64D7E910233F
:10518000D7E93401FBF760FD02460B4611463C4B64
:10519000A3FB01235B09642202FB03F3CB1ADB00B0
:1051A00003F13202364BA3FB02235B099BB25B0087
:1051B0009BB203F4F8739BB223449CB2D7F8F83047
:1051C0000022C7F8C030C7F8C420D7E9308942466A
:1051D0004B469118B9635B41FB63D7E90E23414607
:1051E0005118396349464B417B634FF000024FF041
:1051F0000003D7E90CAB5946CB00514643EA517343
:105200005146CA0010461946034642469B18C7F845
:10521000B8304B460A4642EB0303C7F8BC30D7F818
:10522000F0300022C7F8B030C7F8B420D7E92C120C
:105230000B46DB18BB62134642EB0303FB62D7E964
:105240000A23D7E92E01FBF7FFFC02460B460C4B65
:10525000A3FB02135B09642101FB03F3D31ADB00F8
:105260003233074AA2FB03235B099BB203F0070317
:105270009BB223449BB21A46D7F8FC309A6007E1F0
:105280001F85EB51D7F8F8300022C7F8A830C7F8CF
:10529000AC20D7E92A8942464B46911839625B41D6
:1052A0007B62D7E9082341465418494643EB010580
:1052B0004FF000024FF00003EB0043EA5473E200AA
:1052C00014461D464346E318C7F8A0304B4645EB4D
:1052D0000303C7F8A430D7F8F0300022C7F898309D
:1052E000C7F89C204FF000024FF00003D7E9264595
:1052F00029468B00214643EA917321468A00D7E96B
:105300002801FBF7A1FC02460B46644BA3FB0223DA
:105310005B099BB21B019CB2D7F8F8300022C7F89A
:105320009030C7F89420D7E9248942464B4691181B
:10533000B9615B41FB61D7E90623414651183961E8
:1053400049464B417B614FF000024FF00003D7E923
:1053500004AB5946CB00514643EA51735146CA004B
:1053600010461946034642469B18C7F888304B46FC
:105370000A4642EB0303C7F88C30D7F8F03000221E
:10538000C7F88030C7F884204FF000024FF00003C8
:10539000D7E9208949468B00414643EA917341464B
:1053A0008A00D7E92201FBF74FFC02460B463B4B34
:1053B000A3FB02135B09642101FB03F3D31A1B0156
:1053C0003233364AA2FB03235B099BB203F0F0039E
:1053D0009BB223449CB2D7F8F8300022BB67FA672F
:1053E000D7E91E8942464B469118B9605B41FB6084
:1053F000D7E9022341465118396049464B417B6049
:105400004FF000024FF00003D7E900AB5946CB0044
:10541000514643EA51735146CA00104619460346A5
:1054200042469B183B674B460A4642EB03037B67A9
:10543000D7F8F0300022BB66FA664FF000024FF05A
:105440000003D7E91A8949468B00414643EA917324
:1054500041468A00D7E91C01FBF7F6FB02460B46E2
:105460000E4BA3FB02135B09642101FB03F3D31A68
:105470001B013233094AA2FB03235B099BB203F0F1
:105480000F039BB223449BB21A46D7F8FC309A60B4
:1054900000BF07F58077BD46BDE8B08F1F85EB5193
:1054A00080B588B000AF786039600123FB770023B6
:1054B000BB617868FFF78EFD0346002B5ED17B68E9
:1054C000DB6823F4164323F00C033A6851683A680A
:1054D000D26811433A68126911433A6892690A43E3
:1054E0001A437B68DA603B689B6819467868FFF767
:1054F00085FD3B685B6919467868FFF792FD07F107
:1055000008031846FFF722FB7B681F4A934202D12B
:105510007B69BB6121E07B681C4A934202D13B69F5
:10552000BB611AE07B681A4A934202D13B69BB61B6
:1055300013E07B68174A934202D17B69BB610CE0A0
:105540007B68154A934202D13B69BB6105E07B68E9
:10555000124A934201D13B69BB61BB69002B0DD05C
:105560003B681B68002B09D00023FB773B689A69D6
:105570003B681B68B9697868FFF766FDFB7F1846D2
:105580002037BD4680BD00BF0010014000440040F0
:105590000048004000140140004C00400050004012
:1055A00080B483B000AF7860044A7B68136000BFAA
:1055B0000C37BD465DF8047B704700BF000000203B
:1055C00080B582B000AF184B0022C3F8F020164B14
:1055D0000022C3F8F420144B4FF0FF32C3F8F82038
:1055E000F022002110481FF025F900237B600BE01A
:1055F0000D497A6813465B001344DB000B4400221C
:105600001A607B6801337B607B68092BF0DD064BF9
:105610000022C3F80421002204490A2002F090FD70
:1056200000BF0837BD4680BDF80F00204557010870
:1056300080B584B000AFF8607A603B600B46FB72C7
:10564000FB68002B70D07B68002B08D13B68002BD7
:1056500005D1BB69002B02D1FB69002B64D0374B0D
:10566000D3F8F030092B5FDC344BD3F8F02013462D
:105670005B001344DB00314A134418220021184612
:105680001FF0D8F82D4BD3F8F0202C4913465B00BF
:105690001344DB000B44FA681A60284BD3F8F0205F
:1056A000264913465B001344DB000B440433FA7AAB
:1056B0001A70224BD3F8F020204913465B001344A4
:1056C000DB000B4408337A681A601C4BD3F8F020D7
:1056D0001A4913465B001344DB000B4410333A684D
:1056E0001A60164BD3F8F020144913465B0013449C
:1056F000DB000B440C33BA691A60104BD3F8F0206E
:105700000E4913465B001344DB000B441433FA6963
:105710001A600A4BD3F8F0300133084AC2F8F0306F
:10572000064BD3F8F03004E005481FF091FD4FF030
:10573000FF3318461037BD4680BD00BFF80F00206C
:10574000C07A030880B584B000AF9F4BD3F8F8301F
:10575000B3F1FF3F3CD10023BB6032E0BA6813468F
:105760005B001344DB00984A13447B607B681B6832
:10577000002B22D07B681B6898470346FB707B6830
:105780001B79FA789A4219D18F4ABB68C2F8F8306F
:105790008D4B002283F802218B4B0022A3F8FE20C0
:1057A000894B0022A3F8FC207B681B79DB43022293
:1057B000194686481FF03EF803E100BFBB6801337D
:1057C000BB60814BD3F8F030BA689A42C6DBF8E090
:1057D0007D4BD3F8F8207C4BD3F8F0309A4280F21E
:1057E000F080794BD3F8F82013465B001344DB00BC
:1057F000754A13447B607B681B68002B00F0E180D6
:105800007B681B6898470346FB700123FB736E4B54
:1058100093F802315A1CD1B26B4A82F802111A462F
:10582000694B1344FA7883F80021674B93F80231EF
:1058300003F00103DAB2644B83F802210023BB605A
:1058400013E0614ABB68134403F580731A78BB68A0
:1058500001335D490B4493F800319A4202D0002392
:10586000FB7305E0BB680133BB60BB68002BE8DD60
:10587000554BB3F8FC30002B1FD17B681B79FA78AD
:105880009A4278D1FB7B012B75D14F4B0122A3F8B3
:10589000FC207B685B69002B02D07B685B699847C2
:1058A0007B68DB68002B66D0474B0122C3F8F420ED
:1058B000454B3222A3F8FE205DE0434BD3F8F43091
:1058C000032B58D07B681B79FA789A4227D13E4B3C
:1058D000B3F8FC30312B08D83B4BB3F8FC30013324
:1058E0009AB2394BA3F8FC2045E0374BB3F8FC30B3
:1058F000322B40D17B689B68002B07D0324B322281
:10590000A3F8FE20304B0222C3F8F4202E4BB3F84C
:10591000FC3001339AB22C4BA3F8FC202BE0FB7B2C
:10592000012B28D17B681B69002B08D0264B322223
:10593000A3F8FE20244B0322C3F8F4201BE07B686D
:10594000DB68002B07D17B689B68002B03D17B6849
:105950001B69002B05D01C4BD3F8F430B3F1FF3F8B
:1059600009D1194B0022C3F8F420174B4FF0FF3236
:10597000C3F8F82025E0144BD3F8F430002B20DDD9
:10598000114BB3F8FE30002B1BD00F4BB3F8FE3099
:10599000013B9AB20C4BA3F8FE200B4BB3F8FE3040
:1059A000002B0ED1084BD3F8F430032B04D1064B57
:1059B0004FF0FF32C3F8F820034B4FF0FF32C3F82B
:1059C000F4201037BD4680BDF80F0020F8100020ED
:1059D00080B586B000AF0023FB6002F0DFFCB8604A
:1059E00000233B6100237B611CE07A6913465B0066
:1059F0001344DB00264A13443B603B681B68002BC2
:105A00000CD03B681B68984703461A463B681B79D5
:105A10009A4204D03B6901333B6100E000BF7B69DF
:105A200001337B611A4BD3F8F0307A699A42DCDBA0
:105A3000174BD3F8F0303A699A4219D0FFF782FE3B
:105A4000134BD3F80431002B04D0114BD3F804319D
:105A50000120984702F0A2FC78607A68BB68D31AEC
:105A600041F288329342BBD94FF0FF33FB6000E034
:105A700000BF074B0022C3F8F420054B4FF0FF3264
:105A8000C3F8F820FB6818461837BD4680BD00BF34
:105A9000F80F002080B483B000AF7860044A7B68C0
:105AA000C2F8043100BF0C37BD465DF8047B704777
:105AB000F80F002080B400AF064B0022C3F8F4209A
:105AC000044B4FF0FF32C3F8F82000BFBD465DF82D
:105AD000047B7047F80F002080B584B000AF544BB2
:105AE000D3F80831002B40F09F80514BD3F8083198
:105AF00001334F4AC2F808314D4BD3F8F430002B34
:105B000040F38D804A4BD3F8F830002BC0F28780E9
:105B10000023BB600023FB602EE0FA6813465B00A5
:105B20001344DB00424A13447B607B681B68002BF4
:105B30001ED07B681B6898470346FB707B681B7907
:105B4000FA789A4215D13A4BD3F8F830FA689A426B
:105B500003D1BB680133BB600BE0BB68013BBB609A
:105B6000334BD3F8F830194632481FF0D5FA00E02D
:105B700000BFFB680133FB602D4BD3F8F030FA68AF
:105B80009A42CADB2A4BD3F8F430032B02D0BB680D
:105B9000012B07D0264BD3F8F430032B3AD1BB6846
:105BA000002B37D1224BD3F8F82013465B00134467
:105BB000DB001F4A13447B607B68002B2AD01C4B00
:105BC000D3F8F430012B08D17B68DB68002B21D09F
:105BD0007B68DB689847B8601CE0154BD3F8F4305D
:105BE000022B08D17B689B68002B13D07B689B68D5
:105BF0009847B8600EE00E4BD3F8F430032B09D170
:105C00007B681B69002B05D07B681B699847B860CF
:105C1000FFF750FF064B4FF0FF32C3F8F420044B60
:105C20000022C3F8082100E000BF1037BD4680BD48
:105C3000F80F0020E07A030880B58EB000AF03466D
:105C4000FB7100233B6200237B620123BB620023C4
:105C5000FB6000233B6100237B610023BB61FB7978
:105C6000FB610E233B630123FB6207F10C03194622
:105C70000848FDF727F9034687F83730FB7997F88E
:105C80003720194604481FF047FA00BF3837BD4691
:105C900080BD00BF0C0F0020F87A030880B483B0E9
:105CA00000AF78607B68044A136000BF0C37BD46C4
:105CB0005DF8047B704700BF0C00002080B582B007
:105CC00000AF00F047F81D4B1B68002B03D01B4BA7
:105CD0001B680020984702211948FDF72CFC034659
:105CE000FB71FB79002B02D016481FF0B1FA04219A
:105CF0001348FDF720FC0346FB71FB79002B02D013
:105D000011481FF0A5FA01210D48FDF73AFC0346A2
:105D1000FB71FB79002B02D00C481FF099FA084860
:105D2000FDF7B0F90346FB71FB79002B02D0084860
:105D30001FF08EFA00BF0837BD4680BD0C00002062
:105D40000C0F0020207B03086C7B0308B07B03084A
:105D5000F87B030880B500AF4FF4047200211348AC
:105D60001EF068FD4FF41372002111481EF062FD11
:105D70000E4B0E4AC3F800220C4B0C4AC3F8042207
:105D80000A4B0022C3F80822084B0022C3F80C2259
:105D9000074B074AC3F84022054B054AC3F8442283
:105DA000034B0022C3F8482200BF80BD50130020DF
:105DB0000411002080B582B000AF204BD3F8083228
:105DC000002B01DC012335E01C4BD3F804321946CB
:105DD0001A4BD3F8043203F118023B461848FDF77A
:105DE00095F90346FB71FB79002B1DD101F0D4F826
:105DF000124BD3F80832013B104AC2F808320F4B5D
:105E0000D3F8043220330D4AC2F804320B4BD3F8D6
:105E100004320C4A934203D9084B084AC3F80422BF
:105E200001F0CEF8002305E0FB79194606481FF083
:105E300073F9022318460837BD4680BD5013002071
:105E40000C0F002030150020107C030880B58AB0AC
:105E500000AF3B461C333A4600212048FDF731FA9B
:105E6000034687F8273097F82730002B2AD11C4BA0
:105E7000D3F848320E2B21DC194BD3F84032394687
:105E8000242218461EF0C8FC154BD3F848320133C3
:105E9000134AC2F84832124BD3F840322433104A26
:105EA000C2F840320E4BD3F840320E4A934203D927
:105EB0000B4B0B4AC3F8402200230AE00A481FF0AC
:105EC000C7F905E097F82730194608481FF024F96C
:105ED000012318462837BD4680BD00BF0C0F0020A7
:105EE00004110020201300203C7C0308587C030888
:105EF00080B584B000AF78607B68002B05D1324854
:105F00001FF0A6F94FF0FF3359E0304BD3F80832B9
:105F10000F2B4EDC2D4BD3F8003220227968184627
:105F20001EF07AFC01F038F8284BD3F80832013320
:105F3000264AC2F80832254BD3F800322033234AD0
:105F4000C2F80032214BD3F80032214A934203D9E0
:105F50001E4B1E4AC3F8002201F032F81B4BD3F847
:105F60000C32002B1ED1FFF725FFF860FB68002BD9
:105F700008D1164B0122C3F80C2201211548FDF768
:105F8000DAFA13E0FB68012B08D1104B0022C3F8AA
:105F90000C2201210F48FDF7F4FA07E00E481FF02C
:105FA00057F903E001210B48FDF7C5FA0023FB6018
:105FB00004E00A481FF04CF90123FB60FB68184617
:105FC0001037BD4680BD00BF847C030850130020FD
:105FD000301500200C0F0020A47C0308C87C0308A7
:105FE00080B584B000AF78607B68002B02D14FF0A1
:105FF000FF332EE0194BD3F84832002B26DD174B28
:10600000D3F844322422194678681EF005FC00F0CB
:10601000C3FF124BD3F84832013B104AC2F8483252
:106020000E4BD3F8443224330C4AC2F844320B4BA3
:10603000D3F844320A4A934203D9084B074AC3F8BB
:10604000442200F0BDFF0023FB6001E00123FB6060
:10605000FB6818461037BD4680BD00BF0411002004
:106060002013002080B582B000AFFFF7A3FE786058
:106070007B68002B0ED07B68012B08D1074B0022D8
:10608000C3F80C2201210648FDF77BFA02E005481F
:106090001FF0DEF800BF0837BD4680BD501300205A
:1060A0000C0F0020E07C030880B582B000AF002117
:1060B0000848FDF718FA786004E0FFF7C7FE7B6830
:1060C000013B7B607B68002BF7D100BF00BF083726
:1060D000BD4680BD0C0F002080B582B000AF786057
:1060E000FFF7C0FF00BF0837BD4680BD80B582B056
:1060F00000AF7860FFF7B6FF00BF0837BD4680BD30
:1061000080B582B000AF7860FFF7ACFF00BF083702
:10611000BD4680BD80B582B000AF7860FFF7C4FF98
:1061200000BF0837BD4680BD80B582B000AF786043
:1061300003481FF08DF800BF0837BD4680BD00BF83
:10614000F47C030880B582B000AF786003481FF08C
:106150007FF800BF0837BD4680BD00BF087D03083B
:1061600080B483B000AF78607B68002B03D0064B0F
:1061700001221A6002E0044B00221A6000BF0C37B3
:10618000BD465DF8047B70471000002080B582B0EA
:1061900000AF78603960094B1B68012B05D1396865
:1061A000786801F0CFF8034604E03968786801F0B8
:1061B00033FA034618460837BD4680BD100000205C
:1061C00080B582B000AF78603960094B1B68012B45
:1061D00005D13968786801F02BF9034604E0396885
:1061E000786801F045FA034618460837BD4680BD79
:1061F0001000002080B584B000AF78607B68DBB20F
:10620000FB7307F10F0301211846FFF7BFFF7B68FF
:1062100018461037BD4680BD80B582B000AFFB1C6C
:1062200001211846FFF7CCFF78607B68012B03D172
:10623000FB787B607B6800E0002318460837BD468A
:1062400080BD80B586B000AFF860B9607A607968CB
:10625000B868FFF7B5FF78617B6918461837BD4607
:1062600080BD80B584B000AFF860B9607A607968AD
:10627000B868FFF78BFF7B6818461037BD4680BDB6
:1062800080B582B000AF78607868FFF7B3FF03464F
:1062900018460837BD4680BD80B400AF034B5B682D
:1062A0001846BD465DF8047B704700BF60150020AE
:1062B00080B584B000AF786000F06EFE0A4BDB6CF6
:1062C000FB60094B01229A60074B00225A6000F0E4
:1062D00077FEFB681A46054978681EF09DFAFB6850
:1062E00018461037BD4680BD60150020701500208F
:1062F00080B400AF034B00229A6000BFBD465DF83A
:10630000047B70476015002080B500AF0A4B002267
:106310001A600A4B00221A60094B4FF0FF321A60D4
:10632000084B00221A604FF4FA72002106481EF052
:1063300081FA00BF80BD00BFD8170020DC17002005
:1063400014000020E0170020E415002080B588B07C
:1063500000AF78607B68002B00F0B6800023FB6103
:1063600080E0FB69322202FB03F3594A1344796847
:106370001846F9F74DFF0346002B70D1554B1B68AB
:10638000FA699A4208DB544B1A68524B1B68F96948
:10639000CB1AD31A3B6104E04E4B1A68FB69D31A3F
:1063A0003B613B69013B3B610023FB6052E0FA69C2
:1063B000FB681344BB61BB6901337B61464B1B68BF
:1063C000BA699A4204DB444B1B68BA69D31ABB61B1
:1063D000414B1B687A699A4204DB3F4B1B687A6920
:1063E000D31A7B61BB69322202FB03F3384A1344A0
:1063F0003222002118461EF01DFABB69322202FB30
:1064000003F3334A1A447B69322101FB03F3304919
:106410000B44194610461EF043FF3B69013BFA68E6
:106420009A4214D17B69322202FB03F3284A1344B7
:106430003222002118461EF0FDF97B69322202FB50
:1064400003F3234A1344796818461EF029FFFB68BA
:106450000133FB60FA683B699A42A8DB34E0FB69D0
:106460000133FB611C4B1B68FA699A42FFF679AF56
:10647000184B1B68092B02DD164B00221A60154BC6
:106480001B68322202FB03F3114A1344322200211B
:1064900018461EF0CFF90F4B1B68322202FB03F3A4
:1064A0000B4A1344796818461EF0FAFE094B1B6824
:1064B0000133084A1360084B1B68092B04DC064BA8
:1064C0001B680133044A13602037BD4680BD00BFFE
:1064D000E4150020D8170020DC17002080B582B01A
:1064E00000AF364B1B68002B64DD344B1B68013B4F
:1064F000324A1360324B1B68013B314A1360304B08
:106500001B68002B13DA2F4B1B68013B2C4A1360CE
:106510000DE00820FFF76EFE2020FFF76BFE08203D
:10652000FFF768FE284B9B6C013B274A9364264B80
:106530009B6C002BEDD1244B9B68002B32D1224B5E
:106540005B68002B2ED100237B6027E01C4B1B686F
:106550001E4A322101FB03F31A447B6813441B7863
:10656000FB70FB781F2B16D9FB787E2B13D8164BAC
:106570009B6C302B0FDCFB781846FFF73BFE124B71
:106580009B6C114A1344FA7883F850200E4B9B6C95
:1065900001330D4A93647B6801337B607B68312B48
:1065A000D4DD08E0084B00229A64074B002283F8F0
:1065B000502000E000BF0837BD4680BDE017002036
:1065C00014000020DC17002060150020E4150020D6
:1065D00080B582B000AF444B1A68444B1B689A42A6
:1065E0007EDA414B1B6801333F4A1360404B1B6806
:1065F00001333F4A13603C4B1A683C4B1B689A427C
:1066000013D10DE00820FFF7F5FD2020FFF7F2FD84
:106610000820FFF7EFFD374B9B6C013B354A936435
:10662000344B9B6C002BEDD15BE0314B1A682F4B48
:106630001B689A4211DB2E4B00221A600DE00820E5
:10664000FFF7D8FD2020FFF7D5FD0820FFF7D2FD8A
:10665000284B9B6C013B274A9364264B9B6C002B79
:10666000EDD1244B9B68002B32D1224B5B68002B71
:106670002ED100237B6027E01D4B1B681E4A322170
:1066800001FB03F31A447B6813441B78FB70FB780F
:106690001F2B16D9FB787E2B13D8164B9B6C302BF7
:1066A0000FDCFB781846FFF7A5FD124B9B6C114AD7
:1066B0001344FA7883F850200E4B9B6C01330D4A3B
:1066C00093647B6801337B607B68312BD4DD08E009
:1066D000084B00229A64074B002283F8502000E008
:1066E00000BF0837BD4680BDE0170020DC17002042
:1066F0001400002060150020E415002080B500AFD4
:106700000E4B00229A640D4B0022DA640D20FFF735
:1067100071FD0A20FFF76EFD4320FFF76BFD4D2052
:10672000FFF768FD4420FFF765FD3A20FFF762FDA3
:106730003E20FFF75FFD00BF80BD00BF6015002059
:1067400080B500AF01F0C6FC31234E2238214FF452
:10675000E13000F097FD00220C490A2001F0F0FC26
:106760000C201EF0F1FC0A481EF0D6FC0C201EF096
:10677000EBFC8422002107481EF05CF8064B012246
:106780001A60FFF7C1FD00BF80BD00BF9D67010813
:10679000147D0308601500201000002080B582B031
:1067A00000AFC64B1B68002B40F00283FFF734FD9F
:1067B00078607B68002B03DAC04B00225A64FAE24F
:1067C0007B687F2B00F2718101A252F823F000BF99
:1067D000AB6A0108AB6A0108AB6A0108D16901081C
:1067E000AB6A0108AB6A0108AB6A0108AB6A010831
:1067F000E5690108AB6A0108AB6A0108AB6A0108E8
:10680000AB6A01080B6A0108AB6A0108AB6A0108B0
:10681000AB6A0108AB6A0108AB6A0108AB6A010800
:10682000AB6A0108AB6A0108AB6A0108AB6A0108F0
:10683000AB6A0108AB6A0108AB6A01086B6A010820
:10684000AB6A0108AB6A0108AB6A0108AB6A0108D0
:10685000AB6A0108AB6A0108AB6A0108AB6A0108C0
:10686000AB6A0108AB6A0108AB6A0108AB6A0108B0
:10687000AB6A0108AB6A0108AB6A0108AB6A0108A0
:10688000AB6A0108AB6A0108AB6A0108AB6A010890
:10689000AB6A0108AB6A0108AB6A0108AB6A010880
:1068A000AB6A0108AB6A0108AB6A0108AB6A010870
:1068B000AB6A0108AB6A0108AB6A0108AB6A010860
:1068C000AB6A0108AB6A0108AB6A0108AB6A010850
:1068D000AB6A0108AB6A0108AB6A0108AB6A010840
:1068E000AB6A0108AB6A0108AB6A0108AB6A010830
:1068F000AB6A0108AB6A0108AB6A0108AB6A010820
:10690000AB6A0108AB6A0108AB6A0108AB6A01080F
:10691000AB6A0108AB6A0108AB6A0108AB6A0108FF
:10692000AB6A0108AB6A0108AB6A0108AB6A0108EF
:10693000AB6A0108AB6A0108AB6A0108AB6A0108DF
:10694000AB6A0108AB6A0108AB6A0108AB6A0108CF
:10695000AB6A0108AB6A0108AB6A0108AB6A0108BF
:10696000AB6A0108AB6A0108AB6A0108AB6A0108AF
:10697000AB6A0108AB6A0108AB6A0108AB6A01089F
:10698000AB6A0108AB6A0108AB6A0108AB6A01088F
:10699000AB6A0108AB6A0108AB6A0108AB6A01087F
:1069A000AB6A0108AB6A0108AB6A0108AB6A01086F
:1069B000AB6A0108AB6A0108AB6A0108AB6A01085F
:1069C000AB6A0108AB6A0108AB6A0108736A010887
:1069D0003A4B9B68012B6AD1FFF790FE374B01229F
:1069E000DA6064E0354B9B6C002B62D00820FFF727
:1069F00001FC2020FFF7FEFB0820FFF7FBFB2F4BDD
:106A00009B6C013B2D4A936453E02C4B5B68002B3D
:106A100051D12A4B9B68002B4DD10D20FFF7EAFB8B
:106A20000A20FFF7E7FB254B9B6C244A1344002206
:106A300083F85020214B9B6C204AD3642049214885
:106A40001EF02EFC1D4BDB6C002B02D01C48FFF708
:106A50007DFC1D4B1B681D4A13601D4B1B681D4AA6
:106A60001360164B01225A6025E0144B01225A6430
:106A700033E0124B9B6C002B2ED00820FFF7BAFBA3
:106A80002020FFF7B7FB0820FFF7B4FB0B4B9B6CF4
:106A9000013B0A4A9364094BDB6C002B1CD0074B6B
:106AA000DB6C013B054AD36416E000BF15E000BF74
:106AB00013E000BF11E000BF0FE000BF6015002031
:106AC000B015002070150020D817002014000020F9
:106AD000DC170020E017002000BF7B681B2B00F0B4
:106AE0003B81964B5B6C002B00F03681934B5B6CCB
:106AF000012B40F025817B685B2B40F02181FFF763
:106B00008BFB78607B68313B132B00F2068101A27E
:106B100052F823F0856B0108616C0108D36C010801
:106B2000E56C0108F76C0108096D01081B6D01088F
:106B30001B6D01081B6D01081B6D01081B6D010811
:106B40001B6D01081B6D01081B6D01081B6D010801
:106B50001B6D0108656B01086F6B0108796B0108FB
:106B60007F6B010875237B60FFF7B8FCE4E06423CA
:106B70007B60FFF72DFDDFE072237B60DCE06C23A0
:106B80007B60D9E0FFF748FB78607B687E2B02D101
:106B900068237B60C5E07B68312B09D1FFF73CFBA4
:106BA00078607B687E2B40F0BC8031237B60B8E04E
:106BB0007B68322B09D1FFF72FFB78607B687E2B37
:106BC00040F0AF8032237B60ABE07B68332B09D190
:106BD000FFF722FB78607B687E2B40F0A280332396
:106BE0007B609EE07B68342B09D1FFF715FB786052
:106BF0007B687E2B40F0958034237B6091E07B683E
:106C0000352B09D1FFF708FB78607B687E2B40F0BD
:106C1000888035237B6084E07B68372B08D1FFF7C1
:106C2000FBFA78607B687E2B7BD136237B6078E033
:106C30007B68382B08D1FFF7EFFA78607B687E2BF2
:106C40006FD137237B606CE07B68392B69D1FFF70C
:106C5000E3FA78607B687E2B63D138237B6060E049
:106C6000FFF7DAFA78607B687E2B02D169237B60BC
:106C700059E07B68302B08D1FFF7CEFA78607B684B
:106C80007E2B50D139237B604DE07B68312B08D1BE
:106C9000FFF7C2FA78607B687E2B44D161237B606A
:106CA00041E07B68332B08D1FFF7B6FA78607B6848
:106CB0007E2B38D162237B6035E07B68342B32D168
:106CC000FFF7AAFA78607B687E2B2CD163237B6068
:106CD00029E0FFF7A1FA78607B687E2B25D1642339
:106CE0007B6022E0FFF798FA78607B687E2B1ED1EC
:106CF00065237B601BE0FFF78FFA78607B687E2B53
:106D000017D175237B6014E0FFF786FA78607B6803
:106D10007E2B10D164237B600DE0084B00225A6467
:106D20000AE000BF0FE000BF0DE000BF0BE000BFB6
:106D300009E000BF07E000BF05E000BF60150020CC
:106D40001E4B00225A641D4B5B6C002B04D00023A9
:106D50007B601A4B00225A64184B9B68002B1FD192
:106D6000164B5B68002B1BD17B681F2B22DD7B68D9
:106D70007E2B1FDC114B9B6C302B1BDC7868FFF7E4
:106D800039FA0E4B9B6C7A68D1B20C4A13440A460E
:106D900083F85020094B9B6C0133084A936409E047
:106DA000064B00229A64054B002283F8502002E033
:106DB00000BF00E000BF0837BD4680BD6015002061
:106DC00080B483B000AF064BDB687B60044B0022CD
:106DD000DA607B6818460C37BD465DF8047B704767
:106DE0006015002080B400AFBFF34F8F00BF064B8B
:106DF000DB6803F4E0620449044B1343CB60BFF348
:106E00004F8F00BF00BFFDE700ED00E00400FA0572
:106E100090B58FB000AF78605D4B1A685D4BA3FBF7
:106E20000213D21A520813449B083B627B68002B62
:106E300000F0A5803A6A1346DB009B1A3B62544B74
:106E40001968544BA3FB0123CA1A520813449A0829
:106E50001346DB009B1ACA1A3B6A13443B623B6A27
:106E60003B6300237B630DE03B6B1B78BB777A6849
:106E70007B6B1344BA7F1A703B6B01333B637B6BB4
:106E800001337B637B6B0B2BEEDD7B680C2118469B
:106E900001F0C2FD02467B68DA603BA3D3E9002320
:106EA000C7E90A237B6807F10C04186859689A68D7
:106EB000DB680FC400237B6321E007F10C027B6BCE
:106EC00013441B78BB7797F8283003F00F0387F83B
:106ED0002730D7E90A014FF000024FF00003020902
:106EE00042EA01720B09C7E90A2397F82730BA7FF3
:106EF000D243D1B27A68D1547B6B01337B637B6B15
:106F00000F2BDADD002387F8273034E07B681B780D
:106F1000FB7701237B6326E07B6B013B7A68D35CC4
:106F2000BB77BB7F5B08BB777B6B102B03D1FB7FF1
:106F300087F8263005E07A687B6B13441B7887F866
:106F4000263097F82630DB0187F82630BA7F97F88D
:106F500026301343BB777B6B013B7A68B97FD154F2
:106F60007B6B01337B637B6B102BD5DD97F8273070
:106F7000013387F8273097F82730002BC6D000BFA1
:106F80003C37BD4690BD00BFB8369A1F5EC7D240A1
:106F9000180000202549922480B400AF074B1B68DD
:106FA000002B01D172B600BF044B1B680133034AAA
:106FB000136000BFBD465DF8047B7047E4170020F6
:106FC00080B400AF094B1B68002B04D0074B1B6833
:106FD000013B064A1360054B1B68002B01D162B6CA
:106FE00000BF00BFBD465DF8047B7047E41700207A
:106FF00080B500AF03481EF02BF972B600BFFFF753
:10700000F1FE00BF207D030880B584B000AF78603A
:1070100001F094F9F86001F091F9B860BA68FB6882
:10702000D31A7A689A4200D3F5E700BF00BF103741
:10703000BD4680BD80B586B000AF786001F07EF9B6
:1070400078617B684FF47A7202FB03F33B6101F0D5
:1070500075F9F860FA687B69D31A3A699A4200D3E5
:10706000F5E700BF00BF1837BD4680BD80B58AB0C8
:1070700000AF00237B620823BB613B1D1846FFF76E
:10708000C7FE00233B620023FB6127E0184A3B6AEE
:1070900052F823307B61FB69BA6993FBF2F2B9695C
:1070A00001FB02F29B1AFB61FB695B0028333B4446
:1070B00033F8242C7B691B889A4209D07B691B8892
:1070C0004FF6FF72934203D03B6A01337B620AE0C2
:1070D0003B6A01333B62FB690133FB61054B1B6873
:1070E0003A6A9A42D2DB7B6A18462837BD4680BD91
:1070F000EC170020E817002080B483B000AF0346EF
:10710000FB80FB8841F69812934206D8FB881A460A
:10711000920013445B00FB8002E04FF6FF73FB809C
:1071200000BF0C37BD465DF8047B704780B400AFEC
:1071300000BFBD465DF8047B704780B483B000AFEC
:1071400078607B68DB6843F400527B68DA6000BFDC
:107150000C37BD465DF8047B704780B483B000AF48
:1071600078607B681B6803F02003202B0CBF012391
:107170000023DBB218460C37BD465DF8047B704730
:1071800080B483B000AF78607B681B6803F0400375
:10719000402B0CBF01230023DBB218460C37BD4641
:1071A0005DF8047B704780B483B000AF78607B6883
:1071B0001B6803F08003802B0CBF01230023DBB28C
:1071C00018460C37BD465DF8047B704780B483B029
:1071D00000AF78607B68DB6843F020027B68DA6090
:1071E00000BF0C37BD465DF8047B704780B483B0A8
:1071F00000AF78607B68DB6843F080027B68DA6010
:1072000000BF0C37BD465DF8047B704780B483B087
:1072100000AF78607B68DB6823F020027B68DA606F
:1072200000BF0C37BD465DF8047B704780B483B067
:1072300000AF78607B68DB6823F080027B68DA60EF
:1072400000BF0C37BD465DF8047B704780B483B047
:1072500000AF78607B685B68DBB218460C37BD46D0
:107260005DF8047B704780B483B000AF78600B4654
:10727000FB70FA787B685A6000BF0C37BD465DF83A
:10728000047B704780B582B000AF78600846114635
:107290001A460346FB700B46BB7013467B703822C0
:1072A000002124481DF0C6FA224B234A1A61214BC3
:1072B0004FF4C062DA601F4B204A5A621D4B4FF4F4
:1072C00000721A621B4B1E4A5A601A4A7B6893600E
:1072D000184B1B69174A5361164B5B69154A93613A
:1072E000144B00229A83134B0022DA83114B5B6A02
:1072F000104A93620F4B9B6A0E4AD3620D4B0022D9
:107300001A860C4B01225A860A4B45F2AA521A8061
:10731000084B00225A630A48FFF798FF0848FFF716
:1073200055FF0748FFF709FF002318460837BD46F9
:1073300080BD00BF6C2000206C1800206C1E002057
:107340000010014080B584B000AF786039607B6880
:10735000002B02D03B68002B02DA4FF0FF3361E0D4
:10736000324B1B8845F2AA52934202D06FF00103C0
:1073700058E0FFF711FE2D4B9B8B1A463B681A44D1
:107380002A4BDB689A4201DD00233B60274B9B6957
:10739000BB60FFF715FE3B68002B02DA6FF00203BB
:1073A00040E00023FB6016E07A68531C7B60BB68FA
:1073B000591CB96012781A701C4B1A691B4BDB6898
:1073C000013B1344BA689A4202D9184B1B69BB604F
:1073D000FB680133FB60FA683B689A42E4DB3B6878
:1073E000002B1ED0FFF7D8FD104ABB6893610F4BEE
:1073F0009A8B3B689BB213449AB20C4B9A830B4B0B
:10740000DB8B012B0BD0094B9B8B002B07D0074B41
:107410000122DA83054B5B681846FFF7E7FEFFF7AA
:10742000CFFD3B6818461037BD4680BD6C2000205C
:1074300080B586B000AF786039607B68002B02D0E1
:107440003B68002B02DA4FF0FF334DE0284B1B88DE
:1074500045F2AA52934202D06FF0010344E0FFF7D5
:107460009BFD234B9B6A3B61214B1B8EFB60FFF70F
:10747000A7FDFB68002B02DA6FF0020334E03A68E4
:10748000FB689A4201DD00232EE000237B6117E0B8
:107490007B685A1C7A603A6912781A703B6901332A
:1074A0003B61134B5A6A124B1B6A013B13443A6906
:1074B0009A4202D90E4B5B6A3B617B6901337B6167
:1074C0007A693B689A42E3DBFFF766FD084A3B694D
:1074D0009362074B1A8E3B689BB2D31A9AB2044B45
:1074E0001A86FFF76DFD3B6818461837BD4680BD0C
:1074F0006C20002080B582B000AF464B5B68184618
:10750000FFF72BFE0346002B39D0424B5B68184631
:10751000FFF79CFE0346FB713E4B1B8845F2AA52C7
:10752000934273D13B4B1B8E1A463A4B1B6A9A42CD
:107530001CDA384BDB6AFA791A70364BDB6A013396
:10754000344AD362334BDA6A324B596A314B1B6A85
:10755000013B0B449A4203D92E4B5B6A2D4AD362FE
:107560002C4B1B8E01339AB22A4B1A86294B5B6B2C
:10757000002B04D0274B5B6BFA7910469847254BBC
:107580005B681846FFF70FFE0346002B3FD0214BE8
:107590001B8845F2AA52934205D01E4B5B681846E1
:1075A000FFF744FE33E01B4B9B8B002B25D0194B80
:1075B0005A68184B5B691B7819461046FFF753FE53
:1075C000144B5B690133134A5361124B5A69114BD7
:1075D0001969104BDB68013B0B449A4203D90D4BF0
:1075E0001B690C4A53610B4B9B8B013B9AB2094BB5
:1075F0009A83084B0122DA8309E0064B0022DA83E2
:10760000044B5B681846FFF711FE00E000BF083727
:10761000BD4680BD6C20002080B582B000AF786090
:107620003960124B5B681846FFF700FE16E000BF9A
:107630000E4B5B681846FFF7A3FD0346002BF7D0FF
:107640000A4B5A687B681B7819461046FFF70BFEF9
:107650007B6801337B603B68013B3B603B68002BF0
:10766000E5D13B6818460837BD4680BD6C20002038
:1076700080B584B000AF786039600023FB60144BA4
:107680005B681846FFF7C2FD1AE000BF104B5B684D
:107690001846FFF775FD0346002BF7D00C4B5B68CF
:1076A0001846FFF7D3FD03461A467B681A707B68BD
:1076B00001337B603B68013B3B60FB680133FB604F
:1076C0003B68002BE1D1FB6818461037BD4680BDF2
:1076D0006C20002080B582B000AF464B5B68184636
:1076E000FFF73BFD0346002B39D0424B5B68184641
:1076F000FFF7ACFD0346FB713E4B1B8845F2AA52D7
:10770000934273D13B4B1B8E1A463A4B1B6A9A42EB
:107710001CDA384BDB6AFA791A70364BDB6A0133B4
:10772000344AD362334BDA6A324B596A314B1B6AA3
:10773000013B0B449A4203D92E4B5B6A2D4AD3621C
:107740002C4B1B8E01339AB22A4B1A86294B5B6B4A
:10775000002B04D0274B5B6BFA7910469847254BDA
:107760005B681846FFF71FFD0346002B3FD0214BF7
:107770001B8845F2AA52934205D01E4B5B681846FF
:10778000FFF754FD33E01B4B9B8B002B25D0194B8F
:107790005A68184B5B691B7819461046FFF763FD62
:1077A000144B5B690133134A5361124B5A69114BF5
:1077B0001969104BDB68013B0B449A4203D90D4B0E
:1077C0001B690C4A53610B4B9B8B013B9AB2094BD3
:1077D0009A83084B0122DA8309E0064B0022DA8300
:1077E000044B5B681846FFF721FD00E000BF083737
:1077F000BD4680BDA420002080B485B000AF786075
:1078000014E07B681B78FB73FB7B002B12D0FB7BA7
:10781000602B08D9FB7B7A2B05D8FB7B203BFB73C5
:107820007B68FA7B1A707B6801337B607B68002B76
:10783000E7D100E000BF00BF1437BD465DF8047B10
:107840007047000080B584B000AFF860B9607A601E
:10785000314B1B681F2B53DCF868F8F7E3FC034639
:107860000B2B18D92C4B1A6813469B0013449B0012
:107870002A4A13440B22F96818461CF0CDFF264B08
:107880001A68264913469B0013449B000B440B3394
:1078900000221A700BE0204B1A6813469B00134419
:1078A0009B001E4A1344F96818461DF0F9FC1A4B58
:1078B0001A6813469B0013449B00184A1344184649
:1078C000FFF79AFF144B1A68144913469B001344A0
:1078D0009B000B440C33BA681A600F4B1A680F49AF
:1078E00013469B0013449B000B4410337A681A60C4
:1078F000094B1B680133084A1360074B1B6807E0FC
:10790000054B1B68194606481DF006FC4FF0FF3377
:1079100018461037BD4680BD5C230020DC200020C7
:10792000347D030880B5BCB000AFFEF7B5FC03465C
:10793000002B02D14FF0FF33B4E107F19C0318464E
:10794000FEF7B6FCC7F8D0000023C7F8E0300023EC
:10795000C7F8DC300023C7F8D8300023C7F8D4308C
:10796000002387F86830002387F8343000233B7009
:107970000023C7F8EC30A3E007F19C02D7F8EC3005
:1079800013441B7887F8CF30D7F8E030002B2DD187
:10799000D7F8DC30002B04D197F8CF30202B00F043
:1079A0008580D7F8DC30002B0ED097F8CF30202B15
:1079B0000AD107F16802D7F8DC30134400221A70AC
:1079C0000123C7F8E03076E0D7F8DC30302B72DCEA
:1079D00007F16802D7F8DC30134497F8CF201A700B
:1079E000D7F8DC300133C7F8DC3064E0D7F8E0309A
:1079F000012B2CD1D7F8D830002B03D197F8CF30FA
:107A0000202B55D0D7F8D830002B0ED097F8CF3098
:107A1000202B0AD107F13402D7F8D83013440022C2
:107A20001A700223C7F8E03045E0D7F8D830302B81
:107A300041DC07F13402D7F8D830134497F8CF204F
:107A40001A70D7F8D8300133C7F8D83033E0D7F8F8
:107A5000E030022B3CD1D7F8D430002B03D197F87B
:107A6000CF30202B26D0D7F8D430002B0DD097F86C
:107A7000CF30202B09D13A46D7F8D4301344002216
:107A80001A700323C7F8E03015E0D7F8D430302B54
:107A900011DC3A46D7F8D430134497F8CF201A7047
:107AA000D7F8D4300133C7F8D43004E000BF02E087
:107AB00000BF00E000BFD7F8EC300133C7F8EC306E
:107AC000D7F8EC20D7F8D0309A42FFF655AF00E057
:107AD00000BF07F16802D7F8DC30134400221A70A7
:107AE00007F13402D7F8D830134400221A703A460E
:107AF000D7F8D430134400221A7007F168031846EF
:107B0000FFF77AFE07F134031846FFF775FE3B4690
:107B10001846FFF771FE0023C7F8EC3031E0D7F8C4
:107B2000EC2013469B0013449B00604A134407F16A
:107B3000680211461846F8F76BFB0346002B1BD171
:107B40005A49D7F8EC2013469B0013449B000B4482
:107B500010331B68002B1BD05449D7F8EC20134678
:107B60009B0013449B000B4410331B68394607F1FC
:107B70003402104698470BE0D7F8EC300133C7F8D1
:107B8000EC304B4B1B68D7F8EC209A42C7DB00E087
:107B900000BF474B1B68D7F8EC209A427DDB4FF0C3
:107BA000FF33C7F8E4300023C7F8EC3050E000237F
:107BB000C7F8E83030E007F16802D7F8E83013443E
:107BC0001B7887F8CF303949D7F8EC2013469B0053
:107BD00013449B00CA18D7F8E83013441B7887F881
:107BE000CE3097F8CF30202B1ED097F8CF30002B17
:107BF0001AD097F8CE30202B16D097F8CE30002B25
:107C000012D097F8CF2097F8CE309A420BD1D7F800
:107C1000E8300133C7F8E830D7F8E820D7F8DC308F
:107C20009A42C8DB00E000BFD7F8E820D7F8DC3084
:107C30009A4208D1D7F8DC30002B04D0D7F8EC30CA
:107C4000C7F8E4300AE0D7F8EC300133C7F8EC307D
:107C5000174B1B68D7F8EC209A42A8DBD7F8E43022
:107C6000002B1ADB1149D7F8E42013469B0013447C
:107C70009B000B4410331B68002B0ED00B49D7F828
:107C8000E42013469B0013449B000B4410331B68F5
:107C9000394607F1340210469847FEF72FFDFEF7EC
:107CA00027FB00231846F037BD4680BDDC200020AE
:107CB0005C23002080B590B000AF7860396007F198
:107CC0000C03184611F04EFC002387F83C3007F1F6
:107CD0000C03194608481DF01FFA07F10C0318465B
:107CE00011F0AEFC07F10C03194604481DF014FA1C
:107CF00000BF4037BD4680BD587D0308707D030836
:107D000080B584B000AF786039600023FB601AE072
:107D1000FA6813469B0013449B00104A134419460B
:107D20000F481DF0F9F90D49FA6813469B001344FA
:107D30009B000B440C331B6819460A481DF0ECF9F4
:107D4000FB680133FB60084B1B68FA689A42DFDB73
:107D500000BF00BF1037BD4680BD00BFDC20002043
:107D6000787D0308807D03085C23002080B582B005
:107D700000AF78603960FFF73BF900BF0837BD46B8
:107D800080BD000080B500AFFEF7DAFC4FF4207232
:107D900000210B481CF04EFD0A4B00221A600A4AD3
:107DA0000A490B48FFF74EFD0A4A0B490B48FFF7FB
:107DB00049FD0B4A0B490C48FFF744FD00BF80BD4D
:107DC000DC2000205C230020017D0108AC7D03083D
:107DD000C07D0308B57C0108C87D0308E07D030869
:107DE0006D7D0108E87D0308F87D030880B483B049
:107DF00000AF78607B681B6843F040027B681A60C4
:107E000000BF0C37BD465DF8047B704780B483B07B
:107E100000AF78607B689B6803F00103012B01D100
:107E2000012300E0002318460C37BD465DF8047BB3
:107E3000704780B483B000AF78607B689B6803F0C4
:107E40000203022B01D1012300E0002318460C3766
:107E5000BD465DF8047B704780B483B000AF7860A6
:107E60007B68DB68DBB218460C37BD465DF8047BE7
:107E7000704780B485B000AF78600B46FB707B68BC
:107E80000C33FB60FB68FA781A7000BF1437BD46EC
:107E90005DF8047B7047000080B500AF0348FFF732
:107EA000A5FF034B01221A7000BF80BD00300140C6
:107EB0006023002080B582B000AF0346FB7100BF95
:107EC0000C48FFF7B6FF0346002BF9D0FB791946A3
:107ED0000848FFF7CEFF00BF0648FFF797FF0346AD
:107EE000002BF9D00348FFF7B7FF034618460837C1
:107EF000BD4680BD0030014080B582B000AF034672
:107F0000FB71FB791846FFF7D5FF00BF0837BD4668
:107F100080BD80B500AFFF20FFF7CCFF03461846B9
:107F200080BD000080B500AF0348FFF75FFF034B43
:107F300001221A7000BF80BD00380040612300207C
:107F400080B582B000AF0346FB7100BF0C48FFF75D
:107F500070FF0346002BF9D0FB7919460848FFF75C
:107F600088FF00BF0648FFF751FF0346002BF9D0FA
:107F70000348FFF771FF034618460837BD4680BD2A
:107F80000038004080B582B000AF0346FB71FB793A
:107F90001846FFF7D5FF00BF0837BD4680BD80B546
:107FA00000AFFF20FFF7CCFF0346184680BD00005E
:107FB00080B500AF0348FFF719FF034B01221A7089
:107FC00000BF80BD003C00406223002080B582B02D
:107FD00000AF0346FB7100BF0C48FFF72AFF0346C2
:107FE000002BF9D0FB7919460848FFF742FF00BF84
:107FF0000648FFF70BFF0346002BF9D00348FFF7B5
:108000002BFF034618460837BD4680BD003C0040A4
:1080100080B582B000AF0346FB71FB791846FFF7CD
:10802000D5FF00BF0837BD4680BD80B500AFFF203B
:10803000FFF7CCFF0346184680BD000080B483B034
:1080400000AF03463960FB7197F90730002B0ADB5C
:108050003B68DAB20C4997F907301201D2B20B44EF
:1080600083F800230AE03B68DAB20849FB7903F0A1
:108070000F03043B1201D2B20B441A7600BF0C3737
:10808000BD465DF8047B704700E100E000ED00E0D4
:1080900080B582B000AF78607B68013BB3F1807F30
:1080A00001D301230FE00A4A7B68013B53600F2193
:1080B0004FF0FF30FFF7C2FF054B00229A60044BE0
:1080C00007221A60002318460837BD4680BD00BF4E
:1080D00010E000E080B500AF124B1B68002B1FD1F1
:1080E0001148FFF7D5FF00214FF0FF30FFF7A6FF43
:1080F0000E4B00221A600E4B00221A60A0220021B3
:108100000C481CF097FB0C4B00221A600B4B002212
:108110001A60044B01221A604FF47A70FEF7ECFFEC
:1081200000BF80BD1424002020BF02006423002073
:10813000682300206C2300200C2400201024002041
:1081400080B586B000AFF860B9607A60FB68002B3C
:1081500001DC0123FB601D4B1B68002B26D01C4B50
:108160001B68092B22DCFB68002B1FD0184B1B68F7
:10817000FA6818491B010B441A60154B1B68154A15
:108180001B0113440433BA681A60114B1B68114A6F
:108190001B0113440C337A681A600D4B1B687B611A
:1081A0000B4B1B6801330A4A13600AE0074B19683E
:1081B000074B1A68FB6808481CF0AEFF4FF0FF330E
:1081C0007B617B6918461837BD4680BD14240020AA
:1081D000682300206C230020007E030880B582B055
:1081E00000AF214B1B68002B3AD000237B6032E0AC
:1081F0001E4B1B681A461E497B681B010B441B68FB
:10820000B2FBF3F101FB03F3D31A002B20D1184A80
:108210007B681B01134404331B68002B06D0144AEF
:108220007B681B01134404331B689847104A7B6822
:108230001B0113440C331B68002B09D00C4A7B68CC
:108240001B011344083301221A600A4B01221A60F1
:108250007B6801337B60084B1B687A689A42C7DBF6
:1082600000BF0837BD4680BD1424002064230020D1
:108270006C230020102400206823002080B582B0E9
:1082800000AF164B1B68002B24D0154B1B68002B2E
:1082900020D000237B6018E0124A7B681B01134446
:1082A00008331B68002B0DD00E4A7B681B0113445A
:1082B000083300221A600B4A7B681B0113440C33FD
:1082C0001B6898477B6801337B60074B1B687A68A3
:1082D0009A42E1DB00BF0837BD4680BD1424002070
:1082E000102400206C2300206823002080B500AFFC
:1082F0000F4B1B6801330E4A1360FFF76FFF0C4BE7
:1083000019680C4B83FB01239A10CB17D21A134622
:108310009B0013445B00CA1A002A06D1064B1B6857
:108320000133054A1360FEF701FF00BF80BD00BFA7
:1083300064230020676666660C24002080B485B044
:1083400000AF134B1B68BB60124B9B68FB60104B6C
:108350001B687B60BA687B689A4204D00D4B9B68AF
:10836000FB607B68BB60BB6801334FF47A7203FB30
:1083700002F2FB6801339B080749A1FB03139B082A
:10838000D31A18461437BD465DF8047B704700BF0A
:108390006423002010E000E0176CC11680B400AF29
:1083A000034B1B681846BD465DF8047B704700BF51
:1083B0006423002080B58AB000AF78607B689B683A
:1083C0009847786219E07B6A0F2B02DC7B6A3B627C
:1083D00001E010233B627B685B6807F10C02396A9D
:1083E00010469847F861FB69002B02DC0023FB6113
:1083F00006E07A6AFB69D31A7B627B6A002BE2DCB7
:108400007B6A18462837BD4680BD000080B590B015
:1084100000AF7860396007F10803BB627B68002B0E
:1084200002D03B68002B02D14FF0FF33A7E1954B00
:108430001B68B3F5826F33DA7B689B689847786274
:108440007B6A002B03DC6FF00203FB6328E08D4B9B
:108450001A687B6A134440F2DC5293420BDC7B685F
:108460005B68884A126887490A440432796A104670
:108470009847F8630EE07B685A68824B1B68814915
:108480000B44181D7F4B1B68C3F5BB6304331946AF
:108490009047F8637B4B1A68FB6B1344794A13606F
:1084A000784B1B687B627B6A0F2B04DC6FF0020346
:1084B000FB63FB6B63E10023BB630023FB620023D0
:1084C0007B6300233B630023FB6380E07B6B002B1B
:1084D00006D1BB6B102B03DD6FF00303FB637AE067
:1084E000684B1B68BA6B9A4213DA664ABB6B13443B
:1084F00004331B7887F82330BB6B0133BB63BA6A44
:108500007B6B134497F823201A707B6B032B5BDC87
:1085100003E06FF00203FB635DE07B6B002B1ED179
:10852000462297F82330934205D1BB6B013BFB6297
:1085300001233B6348E0562297F82330934205D14C
:10854000BB6B013BFB6202233B633DE0BB6BFB6209
:1085500000233B6300237B630023FB6337E03B6B1B
:10856000012B10D1484A7B6B13441B7897F82320CA
:108570009A4229D00023FB6200233B6300237B63E4
:108580000023FB6323E03B6B022B10D13F4A7B6B44
:1085900013441B7897F823209A4215D00023FB62DE
:1085A00000233B6300237B630023FB630FE0002376
:1085B000FB6200233B6300237B636FF00703FB63D5
:1085C00033481CF045FE06E07B6B01337B637B6B1D
:1085D0000F2B7FF77BAF7B6B0F2B1DDDBB6A04334B
:1085E0000A21184600F0BEF903463B84BB6ADB89CA
:1085F0009BB23A8C9A4207D11022B96A38681CF0B3
:108600000BF91023FB6307E0BB6BFB6221481CF0F6
:108610001FFE6FF00103FB63FB6B102B76D13B68F1
:1086200004221A4918461CF0E7F80346002B6AD1C9
:108630003B68DB889BB2FB61FB69B3F5806F0CDDA7
:10864000FB691033FA6A1344FB62F96912481CF0A3
:1086500063FD6FF00503FB6358E0FB69002B05D158
:10866000FB6A1033FB621023FB634FE0FB6903F1ED
:108670000F02044B1B689A4210DB6FF00203FB638E
:1086800044E000BF182400209CCA0308A0CA0308C5
:10869000507E0308787E03089C7E0308BB6B3A4A31
:1086A00013440433F969184600F05CF903467B83F0
:1086B000BB6A1B899BB27A8B9A4218D13B6803F143
:1086C0001000BB6B304A13440433FA6919461CF09E
:1086D000A3F8FB69B3F5806F05DA3A68FB691344C8
:1086E000103300221A70FB691033FB6305E0274842
:1086F0001CF0AEFD6FF00103FB63FB691033FA6AF7
:108700001344FB6202E0FB6A1033FB62FB6A002B3E
:108710001EDD1D4B1B68FA6A9A4219DC1A4B1B6856
:10872000FA6A9A420BDAFB6A174A1344191D164B70
:108730001A68FB6AD31A1A4615481CF06DF8124BDA
:108740001A68FB6AD31A104A13600023FB6215E013
:10875000FB6A002B03DA0F481CF07AFD0EE00A4B8F
:108760001B68FA6A9A4209DD074B00221A60064B21
:108770001B681A46F96A08481CF0CEFCFB6B1846C9
:108780004037BD4680BD00BF18240020B87E0308D6
:108790001C240020DC7E0308EC7E030880B588B032
:1087A00000AFF860B9607A60BB68002B02D14FF06F
:1087B000FF335AE0BB6804222E4918461CF01CF80F
:1087C0000346002B02D11023BB6114E0BB680422D6
:1087D000294918461CF010F80346002B05D1BB6848
:1087E000DB889BB21033BB6105E024481CF030FDF0
:1087F0004FF0FF3339E00023FB61FB68DB689847EB
:1088000078617B69002B03DC6FF00103FB6116E0EC
:108810007A69BB699A4211DA7B68013B7B607B68AD
:10882000002B02DC0123FB6109E0FB681B69002BC4
:10883000E3D0FB681B6901209847DEE700BFFB69B6
:10884000002B11D1FB681B68BA68B96910469847BC
:10885000F861FA69BB699A4206D0F96908481CF0C8
:108860005BFC6FF0010300E0002318462037BD4693
:1088700080BD00BF9CCA0308A0CA0308247F030868
:10888000487F030880B584B000AFF860B960134634
:10889000FB80FB68002B02D14FF0FF332EE0BB685A
:1088A000002B01D10023FB80FB68164A106818607A
:1088B000FB68FA88DA80FB881946B86800F052F83D
:1088C00003461A46FB681A81FB6804330A211846DE
:1088D00000F048F803461A46FB68DA81FB88002B53
:1088E0000BD0FB681033BA689A4206D0FB6810338D
:1088F000FA88B96818461BF08FFF00231846103716
:10890000BD4680BDA0CA030880B582B000AF7860C4
:108910007B68002B04D05822002178681BF08AFF66
:1089200000BF0837BD4680BD80B483B000AF0346AA
:108930000A46FB8013467B71FB881B0A9AB2F988B2
:108940007B794B40DBB2064931F813305340FB8052
:10895000FB8818460C37BD465DF8047B704700BFA6
:10896000A4CA030880B584B000AF786039600023E2
:108970007B810023FB600DE0FB687A6813441A7862
:108980007B8911461846FFF7CFFF03467B81FB68C2
:108990000133FB60FA683B689A42EDDB7B8918463D
:1089A0001037BD4680BD80B485B000AF78603960B7
:1089B0000023BB600023FB600AE0FB687A68134475
:1089C0001B781A46BB681344BB60FB680133FB602D
:1089D000FA683B689A42F0DBBB6818461437BD461C
:1089E0005DF8047B7047000080B483B000AF78600E
:1089F0000B46FB707B681A0AF9787B684B40DBB248
:108A0000044951F82330534018460C37BD465DF8F1
:108A1000047B7047A4CC030880B584B000AF7860B5
:108A200039604FF0FF33BB600023FB600BE0FB6855
:108A30007A6813441B781946B868FFF7D5FFB86009
:108A4000FB680133FB60FA683B689A42EFDBBB6866
:108A500018461037BD4680BD80B485B000AF786041
:108A600039600023FB730FE07B681A78FB7B53406F
:108A7000DBB21A46094B9B5CDB43FB737B6801331B
:108A80007B603B68013B3B603B68002BECD1FB7B90
:108A900018461437BD465DF8047B7047A4D0030820
:108AA00080B500AF00F066F800BF80BD80B58AB029
:108AB00000AFF860B9607A603B60BB68012B02D1FF
:108AC00010237B6207E0BB68022B02D108237B6284
:108AD00001E018237B62FB687B617B6ABB617B687A
:108AE000FB613B683B6207F114034FF48052194667
:108AF0000648FBF745FA0346002B01D1012300E0AD
:108B0000002318462837BD4680BD00BF840F0020D3
:108B100080B58AB000AFF860B9607A603B60BB682E
:108B2000012B02D110237B6207E0BB68022B02D12C
:108B300008237B6201E018237B62FB687B617B6A10
:108B4000BB617B68FB613B683B6207F114034FF438
:108B5000805219460648FBF713FA0346002B01D151
:108B6000012300E0002318462837BD4680BD00BF22
:108B7000B80F002080B582B000AF00230122012190
:108B80000120FFF793FF4FF4FA70FEF73DFA002340
:108B9000012201210220FFF789FF00230822012181
:108BA0000320FFF783FF4FF40C737B607B68012287
:108BB00001210420FFF77AFF40F2AB211548FBF7B3
:108BC0000AFA0023012202210120FFF7A1FF4FF43E
:108BD000FA70FEF719FA0023012202210220FFF7A2
:108BE00097FF0023082202210320FFF791FF4FF493
:108BF0000C737B607B68012202210420FFF788FF51
:108C000040F2AB210448FBF7E6F900BF0837BD4648
:108C100080BD00BF840F0020B80F002080B483B057
:108C200000AF78600B467B807B687A881A8000BF33
:108C30000C37BD465DF8047B704780B483B000AF4D
:108C400078607B681B889BB218460C37BD465DF880
:108C5000047B704780B485B000AFF860B9607A607B
:108C600008E0BB689A1CBA60FA681B8813807B68AE
:108C7000013B7B607B68002BF3D100BF00BF143742
:108C8000BD465DF8047B704780B500AFFFF790F9F3
:108C900000BF80BD90B585B000AF03463960FB8052
:108CA0001346BB80BB88002B28D03B68002B25D007
:108CB00011F074FE0320FFF7ABF9FB881B0A9BB28F
:108CC000DBB21846FFF7A4F9FB88DBB21846FFF7C2
:108CD0009FF90023FB6009E03C68631C3B60FFF7E1
:108CE000A4F903462370FB680133FB60BB88FA6874
:108CF0009A42F1DB11F05EFEBB8800E000231846CB
:108D00001437BD4690BD80B584B000AF03463960CE
:108D1000FB801346BB80BB88002B2FD03B68002B09
:108D20002CD011F03BFE0620FFF772F911F042FE45
:108D300011F034FE0220FFF76BF9FB881B0A9BB28F
:108D4000DBB21846FFF764F9FB88DBB21846FFF781
:108D50005FF90023FB6009E03B685A1C3A601B780E
:108D60001846FFF755F9FB680133FB60BB88FA68CA
:108D70009A42F1DB11F01EFEBB8800E0002318468A
:108D80001037BD4680BD80B500AF00F016F8FFF784
:108D900083F800F019F800F0C3F800F002F800BF03
:108DA00080BD80B500AF00F081F900F067FC00F0F5
:108DB0008BFC00F039FA00BF80BD80B400AF00BF6B
:108DC000BD465DF8047B704780B500AF0449054897
:108DD00002F036F80449054802F058F800BF80BD9B
:108DE00059A9020845A90208F97E0108137F010864
:108DF00080B485B000AFF860B9607A603B60FB6812
:108E0000DAB2284B9A71FB681B0ADAB2254BDA7189
:108E1000FB681B0CDAB2234B1A72FB681B0EDAB22A
:108E2000204B5A72BB68DAB21E4B9A72BB681B0A9F
:108E3000DAB21C4BDA72BB681B0CDAB2194B1A732C
:108E4000BB681B0EDAB2174B5A737B68DAB2154B4C
:108E50009A737B681B0ADAB2124BDA737B681B0CBD
:108E6000DAB2104B1A747B681B0EDAB20D4B5A74CF
:108E70003B68DAB20B4B9A743B681B0ADAB2094BB7
:108E8000DA743B681B0CDAB2064B1A753B681B0E92
:108E9000DAB2044B5A7500BF1437BD465DF8047B47
:108EA000704700BF082A002080B588B000AF786006
:108EB00007F10C031846FDF7ABFF07F10C03102177
:108EC0001846FFF74FFD0346FB8307F10C03102103
:108ED0001846FFF768FD03467B777B68002B1AD0A6
:108EE0007B6852221A707B68013350221A707B68AB
:108EF00002334E221A70FB8B1B0A9AB27B68033333
:108F0000D2B21A707B680433FA8BD2B21A707B68C3
:108F100005337A7F1A7000BF2037BD4680BD000040
:108F200080B500AF184B01221A70174B00225A70FF
:108F3000154B01229A70144B0122DA701348FFF787
:108F4000B3FF134B134A1A60134B6FF07F421A6042
:108F5000124B134A1A60134B114A1A600C4B1868D3
:108F60000D4B19680D4B1A680E4B1B68FFF740FF3D
:108F7000064B01229A750C4B03221A700A4B4FF4D0
:108F8000FA625A8000BF80BD202A0020082A0020F3
:108F9000282A0020C0A810FD2C2A0020302A0020FA
:108FA000C0A81001342A0020242A002080B500AF78
:108FB00030490B2001F096FF2F481CF049F92D4B4A
:108FC0001B78012B03D12D481CF042F90DE0294BF1
:108FD0001B78002B03D12A481CF03AF905E0254BF9
:108FE0001B78194627481CF097F8224B5B78012B19
:108FF00003D125481CF02CF90DE01E4B5B78002BAB
:1090000003D122481CF024F905E01A4B5B7819467D
:109010001F481CF081F8174B9B78012B03D11D488A
:109020001CF016F90DE0134B9B78002B03D11A4866
:109030001CF00EF905E00F4B9B78194617481CF001
:109040006BF80C4BDB78012B03D115481CF000F9B1
:109050000DE0084BDB78002B03D112481CF0F8F828
:1090600005E0044BDB7819460F481CF055F800BFAB
:1090700080BD00BF202A0020707F0308947F030872
:10908000AC7F0308C47F0308D47F0308F07F030884
:109090000C8003081C8003083880030850800308F4
:1090A000608003087C80030898800308B0B58CB00A
:1090B00004AF544B3C460FCB84E80F000021002046
:1090C00001F010FF0A20FDF7B5FF0021092001F093
:1090D00009FF0A20FDF7AEFF4B490A2001F002FF0D
:1090E0000A20FDF7A7FF0021092001F0FBFE0A205E
:1090F000FDF7A0FFFFF75AFF3B461946012001F09C
:10910000F1FE0346FB61FB69B3F1FF3F05D13F4828
:109110001CF09EF84FF0FF3370E007F11B03194677
:109120000E2001F0DFFEFB7E194639481BF0F4FFEC
:10913000F0233B8307F118031946042001F0D2FE07
:1091400007F118031946052001F0CCFE07F11803BA
:109150001946022001F0C6FE4FF6F0733B8307F17B
:1091600018031946032001F0BDFE19233B8307F1C4
:1091700018031946062001F0B5FE07F11803194639
:10918000072001F0AFFE3B8B194622481BF0C4FFBD
:1091900007F110031946082001F0A4FE3B7C184695
:1091A0007B7C1C46BB7C1D46FB7C3A7D797D029115
:1091B000019200932B462246014617481BF0ACFF54
:1091C00007F11B0319460F2001F08CFE0346FB61DB
:1091D000FB69B3F1FF3F03D110481CF039F80CE0F4
:1091E000FB7E012B03D10E481CF032F805E0FB7E1C
:1091F000002B02D10B481CF02BF8FB6918462037D6
:10920000BD46B0BD48810308202A0020A88003087D
:10921000C4800308D8800308EC8003080C8103088D
:109220002881030838810308B0B586B004AF002355
:10923000FB71FB1D1946022001F036FF4449002056
:1092400001F032FF0A20FDF7F5FE4149012001F04F
:109250002BFF3B461946082001F044FE3B461946C9
:109260003C481BF059FF3A4B1B781846384B5B784B
:109270001C46374B9B781D46354BDB781A46344BE2
:109280001B791946324B5B790293019100922B4670
:109290002246014630481BF03FFF2D4B9B79194673
:1092A0002B4BDB791A462A4B1B7A1846284B5B7AE4
:1092B0000093034629481BF02FFF254B9B7B194643
:1092C000234BDB7B1A46224B1B7C1846204B5B7CD6
:1092D0000093034622481BF01FFF1D4B9B7A194643
:1092E0001B4BDB7A1A461A4B1B7B1846184B5B7BD1
:1092F000009303461B481BF00FFF154B9B7C194640
:10930000134BDB7C1A46124B1B7D1846104B5B7DC2
:109310000093034614481BF0FFFE0D4B9B7D012B71
:1093200003D112481BF094FF06E0094B9B7D022BF2
:1093300002D10F481BF08CFF0E481BF089FF0E492D
:10934000042001F0B1FE00BF0837BD46B0BD00BF2C
:10935000082A002058810308708103088C810308C3
:10936000A0810308B4810308C8810308DC810308D5
:10937000F081030804820308242A002080B584B009
:1093800000AF78600023FB607B68012B00F3A880AE
:109390007B6813F10F0F0ADA7B686FF47A729342DD
:1093A00000F097807B6813F57A7F33D098E07B6874
:1093B0000F33102B00F2948001A252F823F000BF6B
:1093C000C5940108B7940108A99401089B94010869
:1093D0008D9401087F940108E1940108E19401084B
:1093E0007194010863940108559401084794010899
:1093F000399401082B9401081D9401080D9401086B
:10940000059401083B481BF023FF6CE03A481BF031
:109410001FFF68E039481BF01BFF64E038481BF071
:1094200017FF4FF0FF33FB605DE036481BF010FF85
:109430004FF0FF33FB6056E033481BF009FF4FF05D
:10944000FF33FB604FE031481BF002FF4FF0FF336A
:10945000FB6048E02E481BF0FBFE4FF0FF33FB6043
:1094600041E02C481BF0F4FE4FF0FF33FB603AE084
:1094700029481BF0EDFE4FF0FF33FB6033E0274837
:109480001BF0E6FE4FF0FF33FB602CE024481BF09E
:10949000DFFE4FF0FF33FB6025E022481BF0D8FED3
:1094A0004FF0FF33FB601EE01F481BF0D1FE4FF072
:1094B000FF33FB6017E01D481BF0CAFE4FF0FF337F
:1094C000FB6010E01A481BF0C3FE4FF0FF33FB6057
:1094D00009E018481BF0BCFE4FF0FF33FB6002E0D0
:1094E0007B68FB6000BF00F0C2F8FB6818461037CD
:1094F000BD4680BD6C82030890820308DC820308AD
:109500000C830308248303083C8303088483030833
:10951000A4830308D0830308E8830308188403089E
:109520002C84030844840308588403086C840308CB
:10953000A4840308DC84030880B586B000AFF8601B
:10954000B9607A6000237B61FB681B68012B03D044
:10955000FB681B68022B14D1FB685B68022B0DD1E2
:10956000FB681B7A7A6892B2B968184601F054F821
:1095700038613869FFF702FF786102E003481BF0A9
:1095800067FE7B6918461837BD4680BD0485030811
:1095900080B586B000AFF860B9607A6000237B6167
:1095A000FB681B68012B03D0FB681B68022B14D1DE
:1095B000FB685B68022B0DD1FB681B7A7A6892B25C
:1095C000B968184601F022F938613869FFF7D6FE0C
:1095D000786102E003481BF03BFE7B6918461837B0
:1095E000BD4680BD0485030880B582B000AF7860B9
:1095F0007B685B68022B06D17B681B7A184600F0FB
:10960000B4FC034601E04FF0FF3318460837BD466F
:1096100080BD80B582B000AF78607B685B68022B4C
:1096200006D17B681B7A184600F054FC034601E023
:109630004FF0FF3318460837BD4680BD80B582B075
:1096400000AF78607B68002B04DA786800F0DCFA01
:10965000034608E07B68002B04DC786800F0BEFA63
:10966000034600E0002318460837BD4680BD80B59C
:1096700000AF00F055F800BF80BD000080B483B09B
:1096800000AF00237B6009E00C4A7B685B01134458
:10969000043301221A607B6801337B607B68002BF6
:1096A000F2DD074B00221A60064B00221A6000BF51
:1096B0000C37BD465DF8047B704700BF1C000020DE
:1096C000382A00203C2A002080B582B000AF012358
:1096D000FB7000237B6017E00F4A7B685B0113443B
:1096E00008331B78FA1C0721184601F045F90A4A8D
:1096F0007B685B01134408331B78194607481BF04D
:109700000BFD7B6801337B607B68002BE4DD00BFD1
:1097100000BF0837BD4680BD1C0000201885030827
:10972000B0B590B004AF0023BB6207F10F03194638
:109730000F2001F0D7FB0346FB610A237B6207F190
:109740000E0319460F2001F0CDFB0346BB61FA69F9
:10975000BB699A4204D0B9699C481BF0DDFC11E05A
:10976000BA7BFB7B9A4207D0BB7B1946FB7B1A4630
:1097700097481BF0D1FC05E07B6A013B7B627B6A6A
:10978000002BDCDC7B6A002B40F00C82FB69B3F120
:10979000FF3F06D18F4B00221A608F481BF058FD07
:1097A00003E2FB7B012B0FD18A4B1B68012B52D0AC
:1097B0000123BB62874B01221A6088481BF048FDD9
:1097C000874B00221A6046E0FB7B002B3FD1814B88
:1097D0001B68002B03D07F4B1B68012B16D17D4BE0
:1097E0001B68002B08D10223BB627A4B03221A604C
:1097F0007C481BF02DFD2EE0794B00221A60754B42
:1098000002221A6078481BF023FD24E0714B1B688C
:10981000022B14D175481BF01BFD714B1B680133E3
:109820006F4A13606E4B1B680A2B14DD0223BB6268
:10983000684B03221A606B481BF00AFD0BE0654B76
:109840001B68032B07D06A481BF002FD03E0694840
:109850001BF0FEFCA9E15F4B1B68032B37D1BB6AF1
:10986000022B34D10023FB622DE0634AFB6A5B01CB
:10987000134404331B68012B22D05F4AFB6A5B014F
:109880001344043301221A605B4AFB6A5B011344F0
:1098900008331B78194659481BF03EFC564AFB6AB0
:1098A0005B01134408331B78184600F03FFE524A10
:1098B000FB6A5B01134408331B78184600F06EFD09
:1098C000FB6A0133FB62FB6A002BCEDD6DE10023F6
:1098D000FB6262E1484AFB6A5B01134408331B7870
:1098E000FB75454AFB6A5B01134410331B88BB823E
:1098F000FB7D9B000133DB0003F54073184600F04D
:109900008FF90346FB730A233B62FB7D9B00013307
:10991000DB0003F54073184600F082F90346FB7440
:10992000FB7BFA7C9A4206D0F97DFA7CFB7B3448BB
:109930001BF0F2FB05E03B6A013B3B623B6A002BFC
:10994000E3DC3B6A002B40F02F81FB7B1C2B00F2F9
:10995000118101A252F823F0CB9A0108759B0108EE
:10996000759B0108759B0108759B0108759B010893
:10997000759B0108759B0108759B0108759B010883
:10998000759B0108759B0108759B0108759B010873
:10999000759B0108759B0108759B0108759B010863
:1099A000759B0108199B0108879B0108759B01089D
:1099B000759B0108059A0108759B0108759B0108B4
:1099C000759B0108759B01089B9A01083C8503085B
:1099D00054850308382A00207885030894850308F5
:1099E0003C2A0020A4850308B8850308CC85030819
:1099F000E0850308F48503081C000020088603089E
:109A000038860308FB7D9B000133DB0003F5007300
:109A1000184600F005F903469BB203F01F033B8292
:109A20003B8A03F00103002B00F0AF80604AFB6A21
:109A30005B011344043302221A6007F10802FB7D24
:109A40000421184601F098F8BA1DFB7D052118463F
:109A500001F092F8F97DBB68DBB21C46BB681B0ABB
:109A6000DBB21D46BB681B0CDBB21A46BB681B0E83
:109A7000DBB2F8880290019300922B4622464D48B3
:109A80001BF04AFBFB7D9B000133DB0003F50073F9
:109A90000121184600F010F977E0FB7D184600F030
:109AA00045FD0346FB61FB7D184600F077FCFB7D1E
:109AB000FA69194640481BF02FFB3D4AFB6A5B01DF
:109AC0001344043301221A6064E0FB7D19463B48CD
:109AD0001BF022FBBA8AF87D0123012100F048FB2C
:109AE0000346FB61FB7DFA699A4205D1FB7D19466D
:109AF00033481BF011FB4AE0FB7DFA6919463148F7
:109B00001BF00AFBFB6913F1030F40D12E481BF039
:109B10009FFBFFF746F93AE0FB7D184600F0ACFCEE
:109B20000346FB61FB69012B1DD1214AFB6A5B01E6
:109B30001344043303221A60F97D244B9B791C469D
:109B4000224BDB791D46214B1B7A1A461F4B5B7A51
:109B50001846BB8A0293019000922B4622461C486D
:109B60001BF0DAFA16E0FB7DFA69194619481BF07A
:109B7000D3FA0FE0FB7B002B0BD0FB7B194616487A
:109B80001BF0CAFA05E000BF04E000BF02E000BF1E
:109B900000E000BFFB6A0133FB62FB6A002B7FF72A
:109BA00099AE02E000BF00E000BF3037BD46B0BD57
:109BB0001C0000205C860308A8860308D4860308DE
:109BC0000C8703083487030864870308082A0020E9
:109BD00078870308C4870308F487030880B483B038
:109BE00000AF78607B68002B04DC7B685B01054A72
:109BF000134400E0002318460C37BD465DF8047B93
:109C0000704700BF1C00002080B483B000AF7860B4
:109C1000002318460C37BD465DF8047B70470000F2
:109C200080B584B000AF7860224BDB689847214B49
:109C30005B6998471F4B5B6A002B03D01D4B9B6AE7
:109C4000002B14D11B4B1B6A7A68120CD2B210463F
:109C50009847184B1B6A7A68120AD2B21046984786
:109C6000144B1B6A7A68D2B21046984711E07B68A1
:109C70001B0CDBB23B737B681B0ADBB27B737B681C
:109C8000DBB2BB730B4B9B6A07F10C02032110463E
:109C90009847084BDB6998470346FB73054B9B6964
:109CA0009847044B1B699847FB7B18461037BD4605
:109CB00080BD00BF4000002080B584B000AF786058
:109CC0000B46FB70224BDB689847214B5B6998473A
:109CD0007B6843F004037B601D4B9B6A002B19D10A
:109CE0001B4B1B6A7A68120CD2B210469847184B6D
:109CF0001B6A7A68120AD2B210469847144B1B6A44
:109D00007A68D2B210469847114B1B6AFA7810460F
:109D1000984713E07B681B0CDBB23B737B681B0A24
:109D2000DBB27B737B68DBB2BB73FB78FB73084BE6
:109D30009B6A07F10C02042110469847044B9B696B
:109D40009847034B1B69984700BF1037BD4680BD3D
:109D50004000002090B587B000AFF860B9601346AE
:109D6000FB802B4BDB689847294B5B699847284B56
:109D70005B6A002B03D0264B9B6A002B26D1244B19
:109D80001B6AFA68120CD2B210469847204B1B6A25
:109D9000FA68120AD2B2104698471D4B1B6AFA683D
:109DA000D2B2104698470023FB820AE0184BDB69C9
:109DB000FA8AB9688C18984703462370FB8A0133E6
:109DC000FB82FA8AFB889A42F0D317E0FB681B0CEF
:109DD000DBB23B74FB681B0ADBB27B74FB68DBB253
:109DE000BB740B4B9B6A07F1100203211046984786
:109DF000074B5B6AFA881146B8689847044B9B6921
:109E00009847034B1B69984700BF1C37BD4690BD60
:109E10004000002080B586B000AFF860B9601346FE
:109E2000FB802B4BDB689847294B5B699847FB68A5
:109E300043F00403FB60264B9B6A002B26D1244B86
:109E40001B6AFA68120CD2B210469847204B1B6A64
:109E5000FA68120AD2B2104698471D4B1B6AFA687C
:109E6000D2B2104698470023FB820AE0184B1B6AC7
:109E7000FA8AB9680A44127810469847FB8A013377
:109E8000FB82FA8AFB889A42F0D317E0FB681B0C2E
:109E9000DBB23B74FB681B0ADBB27B74FB68DBB292
:109EA000BB740B4B9B6A07F11002032110469847C5
:109EB000074B9B6AFA881146B8689847044B9B6920
:109EC0009847034B1B69984700BF1837BD4680BDB4
:109ED0004000002090B585B000AF0346FB71002321
:109EE000FB810023BB81FB799B000133DB0003F581
:109EF00000531846FFF794FE0346BB81BB891B0243
:109F00009CB2FB799B000133DB0003F50453184638
:109F1000FFF786FE03469BB22344BB81BB89002B1F
:109F20001AD0FB799B000133DB0003F50053184680
:109F3000FFF776FE0346FB81FB891B029CB2FB798F
:109F40009B000133DB0003F504531846FFF768FE5E
:109F500003469BB22344FB81FA89BB899A42C2D152
:109F6000FB8918461437BD4690BD90B585B000AF4B
:109F70000346FB710023FB810023BB81FB799B001F
:109F80000133DB0003F518531846FFF749FE03467B
:109F9000BB81BB891B029CB2FB799B000133DB00B8
:109FA00003F51C531846FFF73BFE03469BB22344C0
:109FB000BB81BB89002B1AD0FB799B000133DB00EE
:109FC00003F518531846FFF72BFE0346FB81FB8968
:109FD0001B029CB2FB799B000133DB0003F51C5391
:109FE0001846FFF71DFE03469BB22344FB81FA8906
:109FF000BB899A42C2D1FB8918461437BD4690BD31
:10A0000090B585B000AF03463960FB711346BB8045
:10A010000023FB810023BB60BB88002B48D0FB7969
:10A020009B000133DB0003F510531846FFF7F8FDE2
:10A0300003469BB21B029CB2FB799B000133DB0001
:10A0400003F514531846FFF7EBFD03469BB2234478
:10A05000FB81FB891B02FA7992000232D200134481
:10A06000BB60BB881A463968B868FFF7D3FEFA8927
:10A07000BB881344FB81FB799B000133DB0003F5B4
:10A0800010531A46FB891B0A9BB2DBB219461046D5
:10A09000FFF712FEFB799B000133DB0003F514533D
:10A0A0001A46FB89DBB219461046FFF705FE00E0B1
:10A0B00000BF1437BD4690BD90B585B000AF0346D4
:10A0C0003960FB711346BB800023FB810023BB601A
:10A0D000BB88002B48D0FB799B000133DB0003F5E4
:10A0E00020531846FFF79CFD03469BB21B029CB20F
:10A0F000FB799B000133DB0003F524531846FFF77F
:10A100008FFD03469BB22344FB81FB891B02FA7936
:10A1100092000332D2001344BB60BB881A463968F0
:10A12000B868FFF717FEFA89BB881344FB81FB79F7
:10A130009B000133DB0003F520531A46FB891B0A01
:10A140009BB2DBB219461046FFF7B6FDFB799B00C8
:10A150000133DB0003F524531A46FB89DBB21946B1
:10A160001046FFF7A9FD00E000BF1437BD4690BDC3
:10A1700090B585B000AF0446084611461A462346FE
:10A18000FB710346BB710B46BB801346FB70FB792A
:10A19000082B02D94FF0FF33F2E0BB79012B05D039
:10A1A000002B11DD023B022B0ED811E007F10C034E
:10A1B000042219464FF47060FFF7CCFDFB68002BBA
:10A1C00005D16FF00203DBE06FF00403D8E000BFBD
:10A1D000FB7803F00403002B02D06FF00503CFE0FF
:10A1E000FB78002B25D0BB79012B02D0022B08D0A5
:10A1F00024E0FB7803F02103002B1CD16FF0050352
:10A20000BEE0FB7803F02003002B06D097F9033063
:10A21000002B02DB6FF00503B2E0FB7803F01003C4
:10A22000002B0AD097F90330002B06DB6FF00503F3
:10A23000A6E000BF02E000BF00E000BFFB791846C7
:10A2400000F0ACF8FB799B000133DB00184697F96E
:10A25000033023F00F035AB297F9063013435BB271
:10A26000DBB21946FFF728FDBB88002B10D1464B07
:10A270001B885A1C91B2444A1180BB80424B1B88F8
:10A280004FF6F072934203D13F4B4FF440421A8095
:10A29000FB799B000133DB0003F580631A46BB8822
:10A2A0001B0A9BB2DBB219461046FFF705FDFB798E
:10A2B0009B000133DB0003F5A0631A46BB88DBB2C9
:10A2C00019461046FFF7F8FCFB799B000133DB00D1
:10A2D00003F5807301211846FFF7EEFC00BFFB7900
:10A2E0009B000133DB0003F580731846FFF798FCF1
:10A2F0000346002BF3D1FB79012202FA03F31BB2D0
:10A30000DB431AB2214B1B881BB213401BB29AB21B
:10A310001E4B1A80FB7803F00102FB7902FA03F36B
:10A320001AB21A4B1B881BB213431BB29AB2174BBB
:10A330001A80FB79012202FA03F31BB2DB431AB243
:10A34000134B1B881BB213401BB29AB2104B1A80DE
:10A35000FB79104A002122F81310FB790E4A0021E4
:10A36000D15400BFFB799B000133DB0003F5407340
:10A370001846FFF755FC0346002BF3D097F907303A
:10A3800018461437BD4690BD3C000020402A0020EE
:10A39000422A0020442A0020542A002080B582B09E
:10A3A00000AF0346FB71FB79082B02D94FF0FF3356
:10A3B00055E0FB799B000133DB0003F5807310212E
:10A3C0001846FFF779FC00BFFB799B000133DB00E7
:10A3D00003F580731846FFF723FC0346002BF3D1E7
:10A3E000FB799B000133DB0003F500731F21184646
:10A3F000FFF762FCFB79012202FA03F31BB2DB4395
:10A400001AB2194B1B881BB213401BB29AB2164BDF
:10A410001A80FB79012202FA03F31BB2DB431AB262
:10A42000124B1B881BB213401BB29AB20F4B1A80FF
:10A43000FB790F4A002122F81310FB790D4A002105
:10A44000D15400BFFB799B000133DB0003F540735F
:10A450001846FFF7E5FB0346002BF3D1012318460E
:10A460000837BD4680BD00BF402A0020422A002098
:10A47000442A0020542A002080B582B000AF034651
:10A48000FB71FB79082B02D94FF0FF3349E0FB79D0
:10A490009B000133DB001846FFF7C2FB034603F0C5
:10A4A0000F03012B02D06FF004033AE0FB799B000D
:10A4B0000133DB0003F540731846FFF7B1FB034699
:10A4C000132B02D06FF002032BE0FB799B000133CA
:10A4D000DB0003F5807302211846FFF7EDFB00BF98
:10A4E000FB799B000133DB0003F580731846FFF70F
:10A4F00097FB0346002BF3D106E0FB791846FFF7E4
:10A500004DFF6FF003030CE0FB799B000133DB0090
:10A5100003F540731846FFF783FB0346142BECD179
:10A52000012318460837BD4680BD000080B582B0C3
:10A5300000AF0346FB71FB79082B02D94FF0FF33C4
:10A5400062E0FB799B000133DB001846FFF768FBF4
:10A55000034603F00F03012B02D06FF0040353E016
:10A56000FB799B000133DB0003F58073082118465B
:10A57000FFF7A2FB00BFFB799B000133DB0003F573
:10A5800080731846FFF74CFB0346002BF3D1FB7991
:10A59000012202FA03F31BB2DB431AB21C4B1B88E5
:10A5A0001BB213401BB29AB2194B1A80194B1B886D
:10A5B0001A46FB7942FA03F303F00103002B16D08D
:10A5C000002321E0FB799B000133DB0003F50073DE
:10A5D0001846FFF725FB034603F00803002B06D0BF
:10A5E000FB791846FFF7DAFE6FF00C030CE0FB79FD
:10A5F0009B000133DB0003F540731846FFF710FBA7
:10A600000346002BDED1012318460837BD4680BD26
:10A61000422A0020402A002080B584B000AF0346C3
:10A620003960FB711346BB800023FB730023BB81A1
:10A63000FB79082B02D94FF0FF33DEE0FB799B005A
:10A640000133DB001846FFF7EBFA034603F00F0374
:10A65000012B02D06FF00403CFE0BB88002B02D1A6
:10A660006FF00D03C9E0FB799B000133DB0003F5BC
:10A6700040731846FFF7D4FA0346FB73FB7B172B96
:10A6800005D0FB7B1C2B02D06FF00603B5E05D4BC1
:10A690001B881A46FB7942FA03F303F00103002BEF
:10A6A00039D0FB799B000133DB0003F500731846BA
:10A6B000FFF7B6FA034603F01F03FB73FB7B03F0BF
:10A6C0001003002B19D0FB799B000133DB0003F54D
:10A6D000007310211846FFF7EFFAFB79012202FA06
:10A6E00003F31BB2DB431AB2464B1B881BB2134069
:10A6F0001BB29AB2434B1A800DE0FB7B03F00803B8
:10A70000002B06D0FB791846FFF748FE6FF00C03CC
:10A7100073E0002371E0FB799B000133DB0003F55C
:10A72000F8531846FFF77CFA03469BB29B02BB81A5
:10A73000BA88BB899A4201D9BB89BB80FB7918468C
:10A74000FFF7C8FB0346BB81FB799B000133DB00AD
:10A7500003F540731846FFF763FA0346FB73FB7B70
:10A76000172B09D0FB7B1C2B06D0FB791846FFF773
:10A7700015FE6FF0060340E0234B1B881A46FB7959
:10A7800042FA03F303F00103002B05D0BA88BB891A
:10A790009A4201D9002330E0BA88BB899A4200D995
:10A7A000CCE700BFBA88FB7939681846FFF728FC68
:10A7B000FB799B000133DB0003F5807320211846F1
:10A7C000FFF77AFA00BFFB799B000133DB0003F54A
:10A7D00080731846FFF724FA0346002BF3D1FB7968
:10A7E000012202FA03F31AB2064B1B881BB2134371
:10A7F0001BB29AB2034B1A80BB8818461037BD466D
:10A8000080BD00BF422A0020402A002090B585B0BC
:10A8100000AF03463960FB711346BB800023FB7316
:10A820000023BB81FB79082B02D94FF0FF339CE05A
:10A83000FB799B000133DB001846FFF7F1F9034673
:10A8400003F00F03012B02D06FF004038DE0BB88EF
:10A85000002B02D16FF00D0387E0FB799B000133E1
:10A86000DB0003F5F0531846FFF7DAF903469BB215
:10A870009B02BB81BA89BB889A4201D2BB89BB804B
:10A88000FB791846FFF771FB0346BB81FB799B0000
:10A890000133DB0003F540731846FFF7C1F90346A7
:10A8A000FB73FB7B172B26D0FB7B1C2B1CD1BB899E
:10A8B000002B33D1FB791846FFF70CFB03461C46EF
:10A8C000FB799B000133DB0003F5F8531846FFF7D3
:10A8D000A7F903469B029C420DD1FB791846FFF76E
:10A8E0005DFD6FF0060340E0FB791846FFF756FD6B
:10A8F0006FF0060339E01F4B1B881A46FB7942FABA
:10A9000003F303F00103002B04D0BB89002B01D11A
:10A9100000232AE0BB89002B02D1B1E700BF00E091
:10A9200000BFBA89BB889A4201D2BB89BB80BA8872
:10A93000FB7939681846FFF7BFFBFB799B000133B1
:10A94000DB0003F5807340211846FFF7B5F900BF1F
:10A95000FB799B000133DB0003F580731846FFF79A
:10A960005FF90346002BF3D1BB8818461437BD4668
:10A9700090BD00BF402A002080B582B000AF0346E2
:10A980003A60FB710B46BB71FB79082B02D94FF083
:10A99000FF33EDE0BB79013B062B00F2E58001A21D
:10A9A00052F823F0C1A90108DDA90108F9A901089D
:10A9B00037AA01084FAA01088DAA01082FAB010888
:10A9C000FB799B000133DB0003F5B0531A463B686B
:10A9D0001B7819461046FFF76FF9C8E0FB799B001A
:10A9E0000133DB0003F5A8531A463B681B78194670
:10A9F0001046FFF761F9BAE0FB799B000133DB00F9
:10AA000003F590531A463B681B881B0A9BB2DBB2C6
:10AA100019461046FFF750F9FB799B000133DB0024
:10AA200003F598531A463B681B88DBB2194610465B
:10AA3000FFF742F99BE0FB799B000133DB0003F554
:10AA40004063042239681846FFF7E4F98FE0FB7988
:10AA50009B000133DB0003F580531A463B681B88DB
:10AA60001B0A9BB2DBB219461046FFF725F9FB79AA
:10AA70009B000133DB0003F588531A463B681B88B3
:10AA8000DBB219461046FFF717F970E0FB799B001F
:10AA90000133DB001846FFF7C3F8034603F00F034A
:10AAA000012B02D06FF0040362E0FB799B000133BD
:10AAB000DB0003F53C531846FFF7B2F80346002BC2
:10AAC00002D06FF0010353E0FB799B000133DB0000
:10AAD00003F5807322211846FFF7EEF81AE0FB79A0
:10AAE0009B000133DB0003F500731846FFF798F86D
:10AAF000034603F00803002B0CD0FB799B000133C5
:10AB0000DB0003F5007308211846FFF7D5F86FF056
:10AB10000C032DE0FB799B000133DB0003F5807310
:10AB20001846FFF77DF80346002BD8D11FE0FB79CC
:10AB30009B000133DB001846FFF772F8034603F071
:10AB40000F03012B02D06FF0040311E0FB799B008F
:10AB50000133DB0003F53C531A463B681B7819466A
:10AB60001046FFF7A9F802E06FF0090300E00123A7
:10AB700018460837BD4680BD90B583B000AF034688
:10AB80003A60FB710B46BB71FB79082B02D94FF081
:10AB9000FF3301E1BB790C2B00F2FA8001A252F8DD
:10ABA00023F000BFD9AB0108F5AB010811AC0108D7
:10ABB0002DAC010867AC01087FAC010891AD01081C
:10ABC000B9AC0108F3AC010805AD010817AD0108E7
:10ABD00033AD01086BAD0108FB799B000133DB004D
:10ABE0001846FFF71DF8034623F00F03DAB23B685F
:10ABF0001A70D0E0FB799B000133DB0003F5B05302
:10AC00001846FFF70DF803461A463B681A70C2E073
:10AC1000FB799B000133DB0003F5A8531846FEF7D0
:10AC2000FFFF03461A463B681A70B4E0FB799B00AD
:10AC30000133DB0003F590531846FEF7F1FF03469E
:10AC40009BB21B029CB2FB799B000133DB0003F536
:10AC500098531846FEF7E4FF03469BB223449AB28A
:10AC60003B681A8097E0FB799B000133DB0003F51A
:10AC70004063042239681846FFF76CF88BE0FB79D3
:10AC80009B000133DB0003F580531846FEF7C8FF35
:10AC900003469BB21B029CB2FB799B000133DB0095
:10ACA00003F588531846FEF7BBFF03469BB22344C7
:10ACB0009AB23B681A806EE0FB799B000133DB009F
:10ACC0001846FEF7ADFF034603F00F03012B02D039
:10ACD0006FF0040360E0FB799B000133DB0003F5B8
:10ACE0003C531846FEF79CFF03469AB23B681A8015
:10ACF00051E0FB791846FFF7EDF803461A463B682A
:10AD00001A8048E0FB791846FFF72FF903461A46E8
:10AD10003B681A803FE0FB799B000133DB0003F5C1
:10AD200040731846FEF77CFF03461A463B681A70CC
:10AD300031E0FB799B000133DB001846FEF770FF22
:10AD4000034603F00103002B08D0FB791846FFF7F8
:10AD50000CF903461A463B681A801CE0FB79104A3E
:10AD600032F813203B681A8015E0FB799B00013311
:10AD7000DB001846FEF754FF0346012B02D16FF0AB
:10AD8000040309E0FB79074AD25C3B681A7002E0D1
:10AD90006FF0010300E0012318460C37BD4690BD5B
:10ADA000442A0020542A002080B400AF00BFBD46D2
:10ADB0005DF8047B704780B400AF00BFBD465DF80E
:10ADC000047B704780B400AF00BFBD465DF8047BD4
:10ADD000704780B400AF00BFBD465DF8047B70478C
:10ADE00080B483B000AF78607B681B78DBB2184614
:10ADF0000C37BD465DF8047B704780B483B000AF6C
:10AE000078600B46FB707B68FA781A7000BF0C37CD
:10AE1000BD465DF8047B704780B400AF0023184640
:10AE2000BD465DF8047B704780B483B000AF034635
:10AE3000FB7100BF0C37BD465DF8047B7047000016
:10AE400080B483B000AF786039607B68002B02D09B
:10AE50003B68002B06D10A4B0A4A5A61084B0A4A42
:10AE60009A6106E0064A7B685361054A3B68936134
:10AE700000BF00BF0C37BD465DF8047B704700BFC4
:10AE800040000020C5AD0108D3AD010880B483B0F7
:10AE900000AF7860396000BF0F4B1B8803F400736C
:10AEA000002BF9D07B68002B02D03B68002B06D129
:10AEB000094B0A4ADA61084B094A1A6206E0064A57
:10AEC0007B68D361044A3B68136200BF00BF0C3744
:10AED000BD465DF8047B70474000002019AE0108B4
:10AEE00029AE010890B587B000AF03463960FB7109
:10AEF0000023FB750023FB6000233B61FB790F2BD4
:10AF000000F2C78001A252F823F000BF4DAF010844
:10AF100053AF01087FAF010873AF01088DAF01087F
:10AF200099AF0108A7AF0108CDAF0108F3AF010841
:10AF300037B001083DB0010845B0010899B00108DB
:10AF40004DB001085BB0010877B0010800F0EAF8E5
:10AF5000A3E03B68002B04D03B68FB60FB68083330
:10AF60003B61FB683A691146184600F027F9034631
:10AF700094E03B681B88184600F0ACF98DE000F0C7
:10AF8000DDF903461A463B681A8086E03B681B8859
:10AF9000184600F0F8F980E000F010FA03461A466F
:10AFA0003B681A8079E03B681B881B0A9BB2DBB2C6
:10AFB00019464FF49850FEF77FFE3B681B88DBB2C2
:10AFC00019464FF4A050FEF777FE66E04FF4985014
:10AFD000FEF726FE03469BB21B029CB24FF4A05024
:10AFE000FEF71EFE03469BB223449AB23B681A80CA
:10AFF00053E02C4B9A783B681A703B680133294A1E
:10B00000D2781A703B680233264A12791A703B686C
:10B010000333244A52791A703B680433214A9279E7
:10B020001A703B6805331F4AD2791A703B680633A1
:10B0300000221A7031E000F013FA2EE0386800F0B8
:10B0400036FA2AE0386800F074FA26E03B681B788C
:10B05000184600F0D7FA034620E000F0E8F903466E
:10B06000FB75FB7DFF2B02D14FF0FF3316E03B68F1
:10B07000FA7D1A7011E000F0C4F90346FB75FB7D00
:10B08000FF2B02D14FF0FF3308E03B68FA7D1A70C6
:10B0900003E04FF0FF3301E000BF002318461C37E8
:10B0A000BD4690BD4000002080B582B000AF034691
:10B0B0003960FB71FB79052B2CD801A252F823F0E3
:10B0C000D9B00108E1B00108E9B00108F7B0010802
:10B0D00005B101080DB10108386800F0DDFA1CE087
:10B0E000386800F019FB18E03B681B78184600F040
:10B0F00053FB034612E000F071FB03461A463B681F
:10B100001A700AE0386800F071FB06E0386800F059
:10B110008EFB02E04FF0FF3300E0002318460837B3
:10B12000BD4680BD80B586B000AF3B1D06221946E6
:10B130004FF41060FEF70EFE07F1140304221946C7
:10B140004FF48070FEF706FE07F110030422194643
:10B150004FF4A060FEF7FEFD07F10C030422194630
:10B160004FF47060FEF7F6FD80210020FEF7A4FD8D
:10B170000020FEF755FD3B1D062219464FF41060D6
:10B18000FEF748FE07F11403042219464FF48070BD
:10B19000FEF740FE07F11003042219464FF4A060A9
:10B1A000FEF738FE07F10C03042219464FF47060D5
:10B1B000FEF730FE00BF1837BD4680BD80B584B0B5
:10B1C00000AF786039600023BB73FFF7ABFF7B688B
:10B1D000002B3BD00023BB730023FB7315E097F9D2
:10B1E0000F307A6813441A78BB7B1344DBB2BB730D
:10B1F00097F90E30102B02DD4FF0FF3366E097F920
:10B200000F30DBB20133DBB2FB7397F90F30072B42
:10B21000E5DD0023FB7315E097F90F309B00013348
:10B22000DB0003F5F853184697F90F307A6813449A
:10B230001B781946FEF740FD97F90F30DBB201335A
:10B24000DBB2FB7397F90F30072BE5DD3B68002B72
:10B250003BD00023BB730023FB7315E097F90F303D
:10B260003A6813441A78BB7B1344DBB2BB7397F97B
:10B270000E30102B02DD4FF0FF3327E097F90F302F
:10B28000DBB20133DBB2FB7397F90F30072BE5DD3F
:10B290000023FB7315E097F90F309B000133DB00AF
:10B2A00003F5F053184697F90F303A6813441B78AA
:10B2B0001946FEF701FD97F90F30DBB20133DBB21F
:10B2C000FB7397F90F30072BE5DD00231846103785
:10B2D000BD4680BD80B584B000AF0346FB80FB88CF
:10B2E000FB73FB881B0A9BB2BB73FB7B23F00F0332
:10B2F000DBB219464FF4A850FEF7DEFC0023FB73C7
:10B3000014E0BA7BFB7B42FA03F303F00103002B4A
:10B3100009D0FB7B9B000133DB0003F500731F2189
:10B320001846FEF7C9FCFB7B0133FB73FB7B072B45
:10B33000E7D900BF00BF1037BD4680BD80B582B0E1
:10B3400000AF0023FB710023BB710023BB804FF4CF
:10B35000A850FEF765FC034623F00F03FB714FF482
:10B36000B850FEF75DFC0346BB71BB79BB80BB8860
:10B370001B029AB2FB799BB21344BB80BB88184670
:10B380000837BD4680BD80B584B000AF0346FB8062
:10B39000FB88FB73FB881B0A9BB2BB73FB7B1946C4
:10B3A0004FF4B050FEF788FCBB7B19464FF4C050F9
:10B3B000FEF782FC00BF1037BD4680BD80B582B06D
:10B3C00000AF0023FB710023BB710023BB804FF44F
:10B3D000B050FEF725FC0346FB714FF4C050FEF75A
:10B3E0001FFC0346BB71BB79BB80BB881B029AB2B2
:10B3F000FB799BB21344BB80BB8818460837BD4617
:10B4000080BD80B582B000AF0023FB714FF438508F
:10B41000FEF706FC034603F00103002B01D00123D5
:10B42000FB7197F9073018460837BD4680BD80B5D7
:10B4300082B000AF0023FB714FF43850FEF7F0FBF1
:10B44000034603F03803302B02D10123FB7101E0E6
:10B450000023FB7197F9073018460837BD4680BDB9
:10B4600080B582B000AF4FF43850FEF7D9FB0346E9
:10B47000FB71FB7903F07F03FB71FB7919464FF4F5
:10B480003850FEF719FC4FF43850FEF7C9FB03465D
:10B49000FB71FB7963F07F03FB71FB7919464FF475
:10B4A0003850FEF709FC00BF0837BD4680BD80B5A7
:10B4B00084B000AF78600023FB737B681B78012B9E
:10B4C00004D1FB7B43F04003FB7303E0FB7B23F0E1
:10B4D0004003FB737B685B78012B04D1FB7B43F05B
:10B4E0003803FB7319E07B68DB78012B0DD17B6897
:10B4F0009B78012B04D1FB7B43F01803FB730CE01A
:10B50000FB7B43F00803FB7307E07B689B78012B10
:10B5100003D1FB7B43F01003FB73FB7B19464FF415
:10B520003850FEF7C9FBFFF79BFF00BF1037BD4641
:10B5300080BD80B584B000AF78600023FB734FF40A
:10B540003850FEF76DFB0346FB73FB7B9B11DBB2B0
:10B5500003F00103DAB27B681A70FB7B03F0380357
:10B56000202B01D0382B03D17B6801225A7003E0D5
:10B570007B6800225A7000BFFB7B03F03803103B4E
:10B58000102B8CBF01220022D2B2002A11D101223D
:10B5900002FA03F303F0013323F08073002B14BF8E
:10B5A00001230023DBB2002B03D07B6801229A70B9
:10B5B00003E07B6800229A7000BFFB7B03F0380336
:10B5C000083B182B8CBF01220022D2B2002A11D1D5
:10B5D000012202FA03F303F0013323F48073002BFA
:10B5E00014BF01230023DBB2002B03D07B680122B0
:10B5F000DA7003E07B680022DA7000BF00BF10370A
:10B60000BD4680BD80B584B000AF0346FB7100230A
:10B61000FB734FF43850FEF703FB0346FB73FB7BD1
:10B6200003F04003002B02D14FF0FF3330E0FB7BEF
:10B6300023F03803FB73FB79012B04D1FB7B43F030
:10B640003003FB7303E0FB7B43F03803FB73FB7BAE
:10B6500019464FF43850FEF72FFBFFF701FF4FF468
:10B660003850FEF7DDFA0346FB73FB79012B06D158
:10B67000FB7B03F03003002B08D0002308E0FB7BAA
:10B6800003F03803002B01D0002301E04FF0FF331B
:10B6900018461037BD4680BD80B582B000AF7860D7
:10B6A0007B68062219464FF41060FEF7B3FB7B68F7
:10B6B0000E33042219464FF48070FEF7ABFB7B6813
:10B6C0000A33042219464FF4A060FEF7A3FB7B68FF
:10B6D0000633042219464FF47060FEF79BFB7B682B
:10B6E0009A7C0B4B1A707B68DA7C094B5A707B682A
:10B6F0001A7D074B9A707B685A7D054BDA707B6820
:10B700009A7D044B1A7000BF0837BD4680BD00BF4C
:10B710005C2A0020602A002080B582B000AF7860EB
:10B720007B68062219464FF41060FEF713FB7B6816
:10B730000E33042219464FF48070FEF70BFB7B6832
:10B740000A33042219464FF4A060FEF703FB7B681E
:10B750000633042219464FF47060FEF7FBFA0C4BD7
:10B760001A787B689A740A4B5A787B68DA74084BAB
:10B770009A787B681A75064BDA787B685A75054BA0
:10B780001A787B689A7500BF0837BD4680BD00BF38
:10B790005C2A0020602A002080B584B000AF0346F8
:10B7A000FB710023FB73FB7923F03A03002B02D0DB
:10B7B0004FF0FF330EE00020FEF732FA0346FB7332
:10B7C000FA7BFB791343FB73FB7B19460020FEF7E2
:10B7D00073FA002318461037BD4680BD80B500AF10
:10B7E0000020FEF71DFA0346184680BD80B582B0E2
:10B7F00000AF78607B681B7819464FF4D850FEF78D
:10B800005BFA7B685B881B0A9BB2DBB219464FF47C
:10B81000C850FEF751FA7B685B88DBB219464FF4DB
:10B82000D050FEF749FA00BF0837BD4680BD90B53D
:10B8300083B000AF78604FF4D850FEF7F1F90346BB
:10B840001A467B681A704FF4C850FEF7E9F90346B0
:10B850009BB21B029CB24FF4D050FEF7E1F90346B5
:10B860009BB223449AB27B685A8000BF0C37BD4616
:10B8700090BD000080B584B000AFF860B9607A6018
:10B880003B60142200211C4818F0D4FF1A4AFB68C0
:10B890005360194ABB689360174A7B68D360164AA5
:10B8A0003B681361144B5B68002B0BD0124B9B68F9
:10B8B000002B07D0104BDB68002B03D00E4B1B690D
:10B8C000002B05D10D4819F0C3FC4FF0FF330EE0FB
:10B8D000094B01221A6000F013F80021002000F04B
:10B8E0005BF8642000F088FB00F020F80023184685
:10B8F0001037BD4680BD00BF642A002018880308A9
:10B9000080B500AF084B1B68002B0AD0064B5B6864
:10B910009847054B1B6906209847034B9B6898473F
:10B9200000E000BF80BD00BF642A002080B500AFEA
:10B93000084B1B68002B0AD0064B5B689847054BE9
:10B940001B6904209847034B9B68984700E000BFA1
:10B9500080BD00BF642A002080B582B000AF0D4BCF
:10B960001B68002B01D100230FE00A4B5B6898474E
:10B97000084B1B6905209847064BDB689847034630
:10B98000FB71044B9B689847FB7918460837BD4606
:10B9900080BD00BF642A002080B582B000AF03469E
:10B9A0000A46FB711346BB710E4B1B68002B14D06B
:10B9B0000C4B5B6898470B4B1B6901209847094B60
:10B9C0001B69FA7910469847064B1B69BA791046ED
:10B9D0009847044B9B68984700E000BF0837BD4676
:10B9E00080BD00BF642A002080B582B000AFFFF7A1
:10B9F000B3FF0346FB71FB7903F00103FB71FB7995
:10BA000018460837BD4680BD90B587B000AFF860D6
:10BA1000B9607A60BB68002B06D07B68002B03DD21
:10BA20001E4B1B68002B02D14FF0FF3332E01B4B43
:10BA30005B689847194B1B6903209847174B1B6994
:10BA4000FA68120CD2B210469847144B1B69FA6878
:10BA500092B2120A92B2D2B2104698470F4B1B69AB
:10BA6000FA68D2B21046984700237B610AE00B4B7C
:10BA7000DB68BC68621CBA609847034623707B6928
:10BA800001337B617A697B689A42F0DB034B9B68E8
:10BA90009847002318461C37BD4690BD642A0020F5
:10BAA00080B584B000AF786039600023BB601F4B65
:10BAB0001B68002B01D1002333E01C4B5B689847C7
:10BAC0001A4B1B6903209847184B1B697A68120CA4
:10BAD000D2B210469847154B1B697A6892B2120A87
:10BAE00092B2D2B210469847104B1B697A68D2B214
:10BAF000104698470023FB600BE00C4BDB6898472F
:10BB00000346FF2B02D00123BB6006E0FB68013334
:10BB1000FB603B68FA689A42EFD3044B9B689847F6
:10BB2000BB6818461037BD4680BD00BF642A0020A0
:10BB300080B586B000AFF860B9607A60BB68002B52
:10BB400006D07B68002B03DD234B1B68002B02D142
:10BB50004FF0FF333BE0FFF7D3FE642000F06DFAB7
:10BB60001D4B5B6898471C4B1B69022098471A4B7A
:10BB70001B69FA68120CD2B210469847164B1B6923
:10BB8000FA6892B2120A92B2D2B210469847124B99
:10BB90001B69FA68D2B21046984700237B610AE01D
:10BBA0000D4B1A69BB68591CB9601B781846904741
:10BBB0007B6901337B617A697B689A42F0DB064BD3
:10BBC0009B6898474FF4967000F037FA0346184682
:10BBD0001837BD4680BD00BF642A002080B584B000
:10BBE00000AF786039600123FB601C4B1B68002BA1
:10BBF00001D1FB682DE0FFF783FE642000F01DFA01
:10BC0000164B5B689847154B1B6920209847134BD0
:10BC10001B697A68120CD2B2104698470F4B1B6909
:10BC20007A6892B2120A92B2D2B2104698470B4B7F
:10BC30001B697A68D2B210469847084B9B689847B0
:10BC40003B68002B04D04FF4967000F0D5F9F860F3
:10BC5000FB6818461037BD4680BD00BF642A00202F
:10BC600080B586B000AFF860B9607A60FB68DBB27F
:10BC70007B617B69002B02D14FF480737B617B6910
:10BC80001A46B968F868FFF753FF38613B69002B23
:10BC900018D1FA687B691344FB60BA687B69134466
:10BCA000BB607A687B69D31A7B607B68FF2B03DDFE
:10BCB0004FF480737B61E2E77B68002B04DD7B68D7
:10BCC0007B61DCE700BF00E000BF3B691846183726
:10BCD000BD4680BD80B5ADF5815D82B000AF07F196
:10BCE000280343F81C0C07F1280343F8201C07F134
:10BCF000280343F8242C07F1280353F81C3C23F4B1
:10BD00007F6323F00F0307F5805202F118021360DE
:10BD1000002307F5805202F11C02136007F128038B
:10BD200007F12802114653F8243C07F5805202F12E
:10BD30001802126851F81C1CAD4819F0EDF93BE1EE
:10BD4000002307F58152136007F12803183B4FF4D5
:10BD50008052194607F5805303F118031868FFF75E
:10BD600053FE4FF4805307F5805202F11402136022
:10BD700007F1280353F81C2C07F5805303F118032F
:10BD80001B68D21A07F1280353F8243C134407F523
:10BD9000805202F1140212689A4213D907F1280363
:10BDA00053F81C2C07F5805303F118031B68D21AB3
:10BDB00007F1280353F8243C134407F5805202F19D
:10BDC0001402136007F1280307F5805202F11802EC
:10BDD000126853F81C3CD31A07F5805202F1140282
:10BDE0001268134407F5805202F11002136007F144
:10BDF000280353F81C2C07F5805303F118031B6824
:10BE0000D31A07F5815202F10402136034E007F1FE
:10BE100028031A4607F5815303F104031B681344F2
:10BE2000183B1A7807F5815303F104031B6807F1E7
:10BE3000280151F8201C0B441B781340DAB207F597
:10BE4000815303F104031B6807F1280151F8201CFA
:10BE50000B441B789A4204D0012307F581521360EA
:10BE600016E007F5815303F104031B68013307F55E
:10BE7000815202F10402136007F5815303F10403B8
:10BE80001B6807F5805202F1140212689A42BED86C
:10BE900007F581531B68002B38D0012107F580532B
:10BEA00003F118031868FFF799FE07F1280353F808
:10BEB0001C2C07F5805303F118031B68D21A07F1F5
:10BEC0002803183B134407F12802114607F5805256
:10BED00002F11002126851F8201C184618F09CFC60
:10BEE00007F12803183B4FF48052194607F5805399
:10BEF00003F118031868FFF7B3FE07F5805303F149
:10BF00001C0318603B4819F0A3F916E007F58053AD
:10BF100003F110031B6807F12802114607F12802FC
:10BF200010461A4651F8201C50F81C0CFFF798FEDA
:10BF300007F5805303F11C03186007F5805303F1E4
:10BF40001C031B68002B46D107F1280353F8242C4F
:10BF500007F5805303F110031B68D31A07F1280279
:10BF600042F8243C07F12803194607F1280353F847
:10BF7000202C07F5805303F110031B68134441F88C
:10BF8000203C07F12803194607F1280353F81C2C1D
:10BF900007F5805303F110031B68134441F81C3C60
:10BFA00007F5805303F118031B6803F5805307F569
:10BFB000805202F11802136007F1280353F81C3C69
:10BFC000B3F1007F08D207F1280353F8243C002B7B
:10BFD0003FF7B6AE00E000BF07F5805303F11C0346
:10BFE0001B68184607F581570837BD4680BD00BF5E
:10BFF000548803087888030880B584B000AF78605F
:10C000004FF0FF33BB600023FB600DE0FFF7ECFC5B
:10C010000346002B02D10023BB6009E00120FBF79F
:10C0200009F8FB680133FB60FA687B689A42EDD33C
:10C03000BB6818461037BD4680BD80B584B000AFE0
:10C0400078604FF0FF33BB600023FB600DE0FFF72B
:10C05000CBFC0346002B02D10023BB6009E00A2081
:10C06000FAF7D2FFFB680133FB60FA687B689A42FB
:10C07000EDD3BB6818461037BD4680BD80B584B08F
:10C0800000AF786039603B68BB600020FAF768F861
:10C09000334819F0DDF87B68002B03D1314819F0E3
:10C0A000D7F81AE07B68012B03D12F4819F0D0F89C
:10C0B00013E07B68022B03D12C4819F0C9F80CE07F
:10C0C0007B68032B03D12A4819F0C2F805E07B688E
:10C0D000042B02D1274819F0BBF8274819F0B8F80B
:10C0E000BB681B681946254819F016F8BB685B68E1
:10C0F0001946234819F010F8BB689B681946214877
:10C1000019F00AF8BB68DB6819461F4819F004F8F3
:10C11000BB681B6919461D4818F0FEFFBB685B69C8
:10C1200019461B4818F0F8FFBB689B691946194867
:10C1300018F0F2FFBB68DB691946174818F0ECFFEE
:10C140000023FB6008E03220FAF774FF6420FAF75E
:10C1500071FFFB680133FB60FB68092BF3DD97E798
:10C160009C890308CC890308E4890308FC89030837
:10C17000148A03082C8A03083C8A03084C8A0308A3
:10C180005C8A03086C8A03087C8A03088C8A03088B
:10C190009C8A0308B08A0308C48A030880B48DB05F
:10C1A00000AF786039607B68002B02D03B68002BC1
:10C1B00002D14FF0FF3300E10023FB62F2E0FB6AA3
:10C1C0007A681A4407F114031068516803C307F131
:10C1D0000C0307F1140292E8030083E80300002334
:10C1E000BB6211E0784ABB6A134408331B78013BF9
:10C1F00007F10C01BA6A0A44127830333B4403F861
:10C200001C2CBB6A0133BB62BB6A072BEADD00232F
:10C210003B620023BB621DE00123FB7700237B62AE
:10C2200012E007F11402BB6A13441A78FB7F134033
:10C23000DBB2002B02D03B6A01333B62FB7F5B0029
:10C24000FB777B6A01337B627B6A072BE9DDBB6A84
:10C250000133BB62BB6A072BDEDD3B6A03F00103DF
:10C26000002B3DD00023BB6235E0FB7EFB77002333
:10C270007B622AE007F114027B6A13441B78BB77C8
:10C2800007F114027B6A13441B785B08D9B207F1EB
:10C2900014027B6A13440A461A70FB7F03F0010301
:10C2A000002B0DD007F114027B6A13441B7863F056
:10C2B0007F03D9B207F114027B6A13440A461A704D
:10C2C000BB7FFB777B6A01337B627B6A072BD1DD07
:10C2D000BB6A0133BB62BA6A3B6A9A42C5DB3BE088
:10C2E0000023BB6234E03B7DFB7707237B6229E0C0
:10C2F00007F114027B6A13441B78BB7707F1140221
:10C300007B6A13441B785B00D9B207F114027B6A85
:10C3100013440A461A7097F91F30002B0DDA07F103
:10C3200014027B6A13441B7843F00103D9B207F16E
:10C3300014027B6A13440A461A70BB7FFB777B6A40
:10C34000013B7B627B6A002BD2DABB6A0133BB62A2
:10C35000BA6A3B6A9A42C6DB0023BB6213E007F16C
:10C360001402BB6A13441A781749BB6A0B441B7842
:10C370005340D9B207F11402BB6A13440A461A703B
:10C38000BB6A0133BB62BB6A072BE8DDFB6A7A68D4
:10C3900013441A4607F1140303CB10605160FB6A83
:10C3A0000833FB62FA6A3B689A4205DA3A68FB6A2C
:10C3B000D31A072B3FF703AF002318463437BD4687
:10C3C0005DF8047B704700BF6C00002080B500AFB3
:10C3D000104B00221A610F4B00225A610D4B0022B4
:10C3E0009A610C4B0022DA610B4B00225A600A4B17
:10C3F00000229A60084B4FF0FF32DA60064B4FF094
:10C40000FF321A61044B00225A6100F071FA00BF3A
:10C4100080BD00BF6C0000207C2F002080B58AB05A
:10C4200000AFF860B9607A603B60FB68002B09DB05
:10C43000BB68002B06D07B68802B09D07B68B3F5E6
:10C44000806F05D0764818F003FF4FF0FF33E2E02D
:10C450003B68002B62D1FB68002B5FD1714B5B689E
:10C46000B3F5806F5AD23B68002B52D1FB68002B8A
:10C470004FD16D4818F0ECFE08226C49B86818F0EE
:10C48000BBF90346002B3ED1BB680833082268493C
:10C49000184618F0B1F90346002B34D1614B012244
:10C4A0009A60604B4FF0FF32DA605E4B4FF0FF3224
:10C4B0001A61BB681B695D4A1361BB685B695B4AB3
:10C4C0005361BB689B69594A9361BB68DB69574AF2
:10C4D000D3611C23FB61FB6919465448FCF79CFAA5
:10C4E000B861524BDB69BA699A4206D14F4B1B695E
:10C4F0001A464C4B5A6100238DE04E4818F0A8FEB6
:10C500006FF0010387E04C4818F0A2FE4FF0FF33B4
:10C5100081E04A4818F09CFE00237CE0484B7B6198
:10C520007A693B6813447B61FB68013B7A6802FBD4
:10C5300003F31A467B6913447B617B683B61394B8B
:10C540005A687B681344374A5360364B9B68002B0C
:10C5500053D0344B5B697A689A4208DA7B683B6255
:10C56000304B5A697B68D31A2E4A536105E02D4B34
:10C570005B693B622B4B00225A6100237B620EE019
:10C58000284B18697B6ABA6813441B781946FCF774
:10C590002BFA0346234A13617B6A01337B627A6A72
:10C5A0003B6A9A42ECDB396AB868FFF7F7FD002373
:10C5B0007B620EE01B4BD8687B6ABA6813441B7819
:10C5C0001946FCF711FA0346164AD3607B6A013319
:10C5D0007B627A6A3B6A9A42ECDB3B6A7B6207E0E9
:10C5E0007B6ABA681344FF221A707B6A01337B624C
:10C5F0007A6A7B689A42F3DB01E07B683B623A69C6
:10C600007969104818F088FD3B691A46B96878695D
:10C61000FFF726FB3B6A18462837BD4680BD00BFA2
:10C62000D48A03087C2F0020EC8A03086C000020C9
:10C6300074000020008B0308188B0308308B03085C
:10C640000000F901448B030880B5ADF5836D00AFA0
:10C6500007F58363A3F21443186007F58363A3F51A
:10C660008363196007F58363A3F583631B68C7F8C9
:10C6700008344FF0FF33C7F814344CE0D7F80834CF
:10C68000B3F5806F0ADD4FF48063C7F80C34D7F838
:10C690000834A3F58063C7F8083406E0D7F80834F7
:10C6A000C7F80C340023C7F8083407F1080107F570
:10C6B0008363A3F214434FF480621868FFF7A4F970
:10C6C0000023C7F8103414E007F58363A3F58262F2
:10C6D000D7F8103413441B78DBB21946D7F814048A
:10C6E000FCF782F9C7F81404D7F810340133C7F8FF
:10C6F0001034D7F81024D7F80C349A42E4DB07F54D
:10C700008363A3F2144307F58362A2F21442126812
:10C7100002F580621A6007F58363A3F583631B68E3
:10C7200003F1FC7303F5803307F58362A2F2144230
:10C7300012689A42A2D3D7F81434184607F58367D3
:10C74000BD4680BD80B584B000AF3A4B9B68002BDE
:10C7500004D1394818F07CFD002367E01C23BB603E
:10C76000BB6819463548FCF757F978604FF0FF333E
:10C77000FB607968324818F0CFFC304BDB69194612
:10C78000304818F0C9FC2D4B5B6919462E4818F04B
:10C79000C3FC284BDB6819462C4818F0BDFC274B1E
:10C7A0009B6919462A4818F0B7FC224B1B691946A9
:10C7B000284818F0B1FC214B1B691946264818F08F
:10C7C000ABFC1C4B5B691946244818F0A5FC1B4BBD
:10C7D000DB697A689A4225D1184B5A69154BDB6898
:10C7E0009A421FD1154B9A69124B1B699A4219D173
:10C7F000124B1B6919461A48FFF726FF78600F4B4A
:10C800005B691A467968174818F086FC0B4B5B6920
:10C810007A689A4202D10023FB6006E0124818F0C1
:10C8200017FD02E0114818F013FDFB681846103799
:10C83000BD4680BD7C2F0020708B03086C0000205B
:10C84000848B0308A48B0308C48B0308E48B0308C0
:10C85000048C0308248C0308488C0308688C0308A4
:10C860000000F9018C8C0308B88C0308D88C0308ED
:10C8700080B58AB002AF7860FFF764FF0346002BF3
:10C8800029D14FF48033FB614FF48033BB61154BEA
:10C890001B697B61134B1B6903F2FF73DB0A3B616E
:10C8A0003B69DB023B610F4B5B69FB60FB680193FB
:10C8B0003B6900937B69BA69F9690B4818F02CFC55
:10C8C000FB6800933B697A69B969F86900F044F83C
:10C8D000FAF78EFB02E0054818F0BAFC00BF2037DB
:10C8E000BD4680BD6C000020F08C0308448D030819
:10C8F00080B584B000AF0023BB60154818F0A8FCD9
:10C900004FF0FC73FB6016E04FF48051F868FFF7BE
:10C91000C7F878607B68002B09D00121F868FFF721
:10C920005DF92E20F9F7ACFCBB680133BB60FB68F6
:10C9300003F58053FB60FB68B3F1007FE4D3B96873
:10C94000044818F0E9FB00BF1037BD4680BD00BFAA
:10C95000708F0308948F030890B5ADF21C4D00AFA3
:10C9600007F58364A4F20C44206007F58360A0F50A
:10C970008260016007F58361A1F214410A6007F546
:10C980008362A2F58362136007F114034FF480629F
:10C99000FF21184617F04EFF07F11403354A1C46D5
:10C9A00013460FCB07C4238002341B0C237007F5FA
:10C9B0008363A3F2044307F58362A2F20C42126878
:10C9C000C3F8802007F58363A3F2044307F583626D
:10C9D000A2F582621268C3F8842007F58363A3F28C
:10C9E000044307F58362A2F214421268C3F8882058
:10C9F00007F58363A3F2044307F58362A2F583621C
:10CA00001268C3F88C2007F58363A3F20443D7F8B8
:10CA10002824C3F8902007F114034FF47F711846BF
:10CA2000FBF7FAFF024607F58363A3F20443C3F85A
:10CA3000FC23114818F00CFC01214FF0FC70FFF7AB
:10CA4000CDF807F11403C7F81434D7F814344FF4B1
:10CA5000806219464FF0FC70FFF702F9074818F0A2
:10CA6000F7FB6420FAF7E6FA00BF07F21C47BD4661
:10CA700090BD00BF108E0308BC8F0308D08F030841
:10CA800080B483B000AF78607B681B6843F001021C
:10CA90007B681A6000BF0C37BD465DF8047B7047A9
:10CAA00080B483B000AF78607B681B6823F001021C
:10CAB0007B681A6000BF0C37BD465DF8047B704789
:10CAC00080B483B000AF786039607B683A68DA621E
:10CAD00000BF0C37BD465DF8047B704780B483B05F
:10CAE00000AF78607B686FF001021A6100BF0C37FD
:10CAF000BD465DF8047B704780B483B000AF7860BA
:10CB00007B681B6903F00103012B01D1012300E0C5
:10CB1000002318460C37BD465DF8047B704780B48F
:10CB200083B000AF78607B68DB6843F001027B680C
:10CB3000DA6000BF0C37BD465DF8047B704780B4F7
:10CB400083B000AF78607B68DB6823F001027B680C
:10CB5000DA6000BF0C37BD465DF8047B704700000B
:10CB600080B582B000AF786039607B68012B03D05C
:10CB70003B681B68012B02D11E4B1B6898477B68E2
:10CB8000022B04D03B6804331B68012B02D11A4BE3
:10CB90001B6898477B68032B04D03B6808331B68ED
:10CBA000012B02D1154B1B6898477B68042B04D0DE
:10CBB0003B680C331B68012B02D1114B1B68984753
:10CBC0007B68052B04D03B6810331B68012B02D116
:10CBD0000C4B1B6898477B68062B04D03B681433CA
:10CBE0001B68012B02D1084B1B68984700BF083710
:10CBF000BD4680BD6C0400207C0400208C04002015
:10CC00009C040020AC040020BC04002080B582B04D
:10CC100000AF786039607B68012B03D03B681B68EC
:10CC2000012B02D11E4B1B6898477B68022B04D056
:10CC30003B6804331B68012B02D11A4B1B689847D1
:10CC40007B68032B04D03B6808331B68012B02D19F
:10CC5000154B1B6898477B68042B04D03B680C334A
:10CC60001B68012B02D1114B1B6898477B68052B71
:10CC700004D03B6810331B68012B02D10C4B1B689E
:10CC800098477B68062B04D03B6814331B68012B44
:10CC900002D1084B1B68984700BF0837BD4680BDCE
:10CCA000700400208004002090040020A0040020D4
:10CCB000B0040020C004002080B582B000AF7860CE
:10CCC00039607B68012B03D03B681B68012B02D1C4
:10CCD0001E4B1B6898477B68022B04D03B680433CB
:10CCE0001B68012B02D11A4B1B6898477B68032BEA
:10CCF00004D03B6808331B68012B02D1154B1B681D
:10CD000098477B68042B04D03B680C331B68012BCD
:10CD100002D1114B1B6898477B68052B04D03B68F8
:10CD200010331B68012B02D10C4B1B6898477B68A2
:10CD3000062B04D03B6814331B68012B02D1084B2F
:10CD40001B68984700BF0837BD4680BD74040020AB
:10CD50008404002094040020A4040020B4040020D3
:10CD6000C404002080B582B000AF786039607B6871
:10CD7000012B03D03B681B68012B02D11E4B1B68A3
:10CD800098477B68022B04D03B6804331B68012B57
:10CD900002D11A4B1B6898477B68032B04D03B6871
:10CDA00008331B68012B02D1154B1B6898477B6821
:10CDB000042B04D03B680C331B68012B02D1114BB0
:10CDC0001B6898477B68052B04D03B6810331B68B1
:10CDD000012B02D10C4B1B6898477B68062B04D0B3
:10CDE0003B6814331B68012B02D1084B1B68984722
:10CDF00000BF0837BD4680BD7804002088040020AD
:10CE000098040020A8040020B8040020C8040020D2
:10CE100080B485B000AFF860B9607A603B60094AC1
:10CE2000FB681360084ABB681360084A7B6813609C
:10CE3000074A3B68136000BF1437BD465DF8047BAA
:10CE4000704700BF6C0400207004002074040020B0
:10CE50007804002080B500AF0948FFF73FFE08487E
:10CE6000FFF76DFE0648FFF71BFE802200210548F4
:10CE700017F0E0FC034B01221A6000BF80BD00BF29
:10CE800000400140942F002080B500AF5148FFF7CB
:10CE900033FE0346002B00F09A804E48FFF71EFE3B
:10CEA0004D4BDA6A4C4B1B6B9A4203D24A4B9B693F
:10CEB000002B1CDC49490120FFF7A8FE474901204F
:10CEC000FFF750FF4348FFF7EBFD434B9B69002BF7
:10CED0007CDD414B00229A613F4B0022DA633E4BDE
:10CEE000DB6F002B72D03C4BDB6F98476EE03A4B08
:10CEF0001B6A3B4A92FBF3F3DA0F13445B109BB2BD
:10CF000019463448FFF7DCFD334B9B6B002B25D1D2
:10CF1000314B01229A63304BDB6A01332E4AD362D4
:10CF20002D4B5A692C4BDB6913442B4A53612A4B16
:10CF30001B68002B0DD1284BDB69012B04D127493D
:10CF40000120FFF70DFE1DE024490120FFF7B4FE8C
:10CF500018E022490120FFF703FE13E01E4B0022D8
:10CF60009A631D4B1B68002B08D11C490120FFF759
:10CF70004DFE1A490120FFF7F5FE03E01749012095
:10CF8000FFF744FE144B9B69012B0DD1124BDA6A5B
:10CF9000114B1B6B5B089A4206D30F4B03229A611D
:10CFA0000D4BDB6A0C4A53630B4B9B69022B0ED172
:10CFB000094BDA6A084B5B6B9A4208D3064B032293
:10CFC0009A61054BDB68044A536200E000BF00BF72
:10CFD00080BD00BF00400140942F0020DC2F0020C6
:10CFE000C027090080B500AF8A4B9B69002B40F336
:10CFF0000E81884BDB6B002B00F00981854B1B6F8A
:10D00000002B5CD1834B1B6C002B58D0814B5B6C8D
:10D010000133804A53647F4B5A6C7E4B1B6C9A429F
:10D020004DD37C4B00225A647A4B1B6E002B19D0D7
:10D03000784B9B69012B07D0764B9B69022B03D061
:10D04000744B9B69032B0DD1724B1B6E714A926E10
:10D050007049C96E104698470346002B02D06D4BAD
:10D0600004229A616B4B5B6E002B21D0694B9B694C
:10D07000012B0BD0674B9B69022B07D0654B9B693B
:10D08000032B03D0634B9B69042B11D1614B5B6E67
:10D09000604A926E5F49C96E104698470346002B5E
:10D0A00006D05C4B1B695B4A53625A4B05229A615E
:10D0B000584B5B6F002B02D0564B5B6F9847554B1C
:10D0C0009B69012B31D1534B9B6A1A46514B5B6ACA
:10D0D00013441A464F4B9A624E4B9B6A42F20F72B0
:10D0E00093420CDD4B4B1B6A01334A4A1362494B96
:10D0F0009B6AA3F51C53103B464A9362ECE700BFC2
:10D10000444B1B6A434A926893420EDB414B022216
:10D110009A61404B9B681A463E4B1A623D4B1A6B14
:10D120003C4BDB6AD31A3B4A53633A4B9B69032B54
:10D1300028D1384B9B6A1A46364B5B6AD31A1A467B
:10D14000344B9A62334B9B6A002B10DA314B1B6ACB
:10D15000002B0CDD2F4B1B6A013B2E4A13622D4B1B
:10D160009B6A03F51C5310332A4A9362EAE7294B62
:10D170001B6A284A5268934204DC264B5B681A46B5
:10D18000244B1A62234B9B69042B03D0214B9B69D0
:10D19000052B3DD11F4B9B6A1A461E4B5B6AD31A67
:10D1A0001A461C4B9A621B4B9B6A002B10DA194BD8
:10D1B0001B6A002B0CDD174B1B6A013B154A1362DF
:10D1C000144B9B6A03F51C531033124A9362EAE72F
:10D1D000104B1B6A0F4A5268934219DC0E4901201A
:10D1E000FFF714FD0C490120FFF7BCFD0B48FFF7CA
:10D1F00057FC084B00229A61064B0022DA63054B6C
:10D20000DB6F002B04D0034BDB6F984700E000BFBF
:10D2100080BD00BF942F0020DC2F00200040014083
:10D2200080B485B000AFF860B9607A603B60094AAD
:10D23000FB681360084ABB681360084A7B68136088
:10D24000074A3B68136000BF1437BD465DF8047B96
:10D25000704700BF7C04002080040020840400206C
:10D260008804002080B500AF0948FFF737FC084864
:10D27000FFF765FC0648FFF713FC802200210548F4
:10D2800017F0D8FA034B01221A6000BF80BD00BF1F
:10D29000004401401430002080B500AF5148FFF732
:10D2A0002BFC0346002B00F09A804E48FFF716FC3B
:10D2B0004D4BDA6A4C4B1B6B9A4203D24A4B9B692B
:10D2C000002B1CDC49490220FFF7A0FC4749022043
:10D2D000FFF748FD4348FFF7E3FB434B9B69002BF7
:10D2E0007CDD414B00229A613F4B0022DA633E4BCA
:10D2F000DB6F002B72D03C4BDB6F98476EE03A4BF4
:10D300001B6A3B4A92FBF3F3DA0F13445B109BB2A8
:10D3100019463448FFF7D4FB334B9B6B002B25D1C8
:10D32000314B01229A63304BDB6A01332E4AD362C0
:10D330002D4B5A692C4BDB6913442B4A53612A4B02
:10D340001B68002B0DD1284BDB69012B04D1274929
:10D350000220FFF705FC1DE024490220FFF7ACFC8A
:10D3600018E022490220FFF7FBFB13E01E4B0022CE
:10D370009A631D4B1B68002B08D11C490220FFF744
:10D3800045FC1A490220FFF7EDFC03E01749022093
:10D39000FFF73CFC144B9B69012B0DD1124BDA6A51
:10D3A000114B1B6B5B089A4206D30F4B03229A6109
:10D3B0000D4BDB6A0C4A53630B4B9B69022B0ED15E
:10D3C000094BDA6A084B5B6B9A4208D3064B03227F
:10D3D0009A61054BDB68044A536200E000BF00BF5E
:10D3E00080BD00BF00440140143000205C300020AC
:10D3F000C027090080B500AF8A4B9B69002B40F322
:10D400000E81884BDB6B002B00F00981854B1B6F75
:10D41000002B5CD1834B1B6C002B58D0814B5B6C79
:10D420000133804A53647F4B5A6C7E4B1B6C9A428B
:10D430004DD37C4B00225A647A4B1B6E002B19D0C3
:10D44000784B9B69012B07D0764B9B69022B03D04D
:10D45000744B9B69032B0DD1724B1B6E714A926EFC
:10D460007049C96E104698470346002B02D06D4B99
:10D4700004229A616B4B5B6E002B21D0694B9B6938
:10D48000012B0BD0674B9B69022B07D0654B9B6927
:10D49000032B03D0634B9B69042B11D1614B5B6E53
:10D4A000604A926E5F49C96E104698470346002B4A
:10D4B00006D05C4B1B695B4A53625A4B05229A614A
:10D4C000584B5B6F002B02D0564B5B6F9847554B08
:10D4D0009B69012B31D1534B9B6A1A46514B5B6AB6
:10D4E00013441A464F4B9A624E4B9B6A42F20F729C
:10D4F00093420CDD4B4B1B6A01334A4A1362494B82
:10D500009B6AA3F51C53103B464A9362ECE700BFAD
:10D51000444B1B6A434A926893420EDB414B022202
:10D520009A61404B9B681A463E4B1A623D4B1A6B00
:10D530003C4BDB6AD31A3B4A53633A4B9B69032B40
:10D5400028D1384B9B6A1A46364B5B6AD31A1A4667
:10D55000344B9A62334B9B6A002B10DA314B1B6AB7
:10D56000002B0CDD2F4B1B6A013B2E4A13622D4B07
:10D570009B6A03F51C5310332A4A9362EAE7294B4E
:10D580001B6A284A5268934204DC264B5B681A46A1
:10D59000244B1A62234B9B69042B03D0214B9B69BC
:10D5A000052B3DD11F4B9B6A1A461E4B5B6AD31A53
:10D5B0001A461C4B9A621B4B9B6A002B10DA194BC4
:10D5C0001B6A002B0CDD174B1B6A013B154A1362CB
:10D5D000144B9B6A03F51C531033124A9362EAE71B
:10D5E000104B1B6A0F4A5268934219DC0E49022005
:10D5F000FFF70CFB0C490220FFF7B4FB0B48FFF7C9
:10D600004FFA084B00229A61064B0022DA63054B61
:10D61000DB6F002B04D0034BDB6F984700E000BFAB
:10D6200080BD00BF143000205C3000200044014069
:10D6300080B485B000AFF860B9607A603B60094A99
:10D64000FB681360084ABB681360084A7B68136074
:10D65000074A3B68136000BF1437BD465DF8047B82
:10D66000704700BF8C040020900400209404002028
:10D670009804002080B500AF0948FFF72FFA08484A
:10D68000FFF75DFA0648FFF70BFA802200210548F4
:10D6900017F0D0F8034B01221A6000BF80BD00BF15
:10D6A000004801409430002080B500AF5148FFF79A
:10D6B00023FA0346002B00F09A804E48FFF70EFA3B
:10D6C0004D4BDA6A4C4B1B6B9A4203D24A4B9B6917
:10D6D000002B1CDC49490320FFF798FA4749032037
:10D6E000FFF740FB4348FFF7DBF9434B9B69002BF7
:10D6F0007CDD414B00229A613F4B0022DA633E4BB6
:10D70000DB6F002B72D03C4BDB6F98476EE03A4BDF
:10D710001B6A3B4A92FBF3F3DA0F13445B109BB294
:10D7200019463448FFF7CCF9334B9B6B002B25D1BE
:10D73000314B01229A63304BDB6A01332E4AD362AC
:10D740002D4B5A692C4BDB6913442B4A53612A4BEE
:10D750001B68002B0DD1284BDB69012B04D1274915
:10D760000320FFF7FDF91DE024490320FFF7A4FA89
:10D7700018E022490320FFF7F3F913E01E4B0022C3
:10D780009A631D4B1B68002B08D11C490320FFF72F
:10D790003DFA1A490320FFF7E5FA03E01749032091
:10D7A000FFF734FA144B9B69012B0DD1124BDA6A47
:10D7B000114B1B6B5B089A4206D30F4B03229A61F5
:10D7C0000D4BDB6A0C4A53630B4B9B69022B0ED14A
:10D7D000094BDA6A084B5B6B9A4208D3064B03226B
:10D7E0009A61054BDB68044A536200E000BF00BF4A
:10D7F00080BD00BF0048014094300020DC30002094
:10D80000C027090080B500AF8A4B9B69002B40F30D
:10D810000E81884BDB6B002B00F00981854B1B6F61
:10D82000002B5CD1834B1B6C002B58D0814B5B6C65
:10D830000133804A53647F4B5A6C7E4B1B6C9A4277
:10D840004DD37C4B00225A647A4B1B6E002B19D0AF
:10D85000784B9B69012B07D0764B9B69022B03D039
:10D86000744B9B69032B0DD1724B1B6E714A926EE8
:10D870007049C96E104698470346002B02D06D4B85
:10D8800004229A616B4B5B6E002B21D0694B9B6924
:10D89000012B0BD0674B9B69022B07D0654B9B6913
:10D8A000032B03D0634B9B69042B11D1614B5B6E3F
:10D8B000604A926E5F49C96E104698470346002B36
:10D8C00006D05C4B1B695B4A53625A4B05229A6136
:10D8D000584B5B6F002B02D0564B5B6F9847554BF4
:10D8E0009B69012B31D1534B9B6A1A46514B5B6AA2
:10D8F00013441A464F4B9A624E4B9B6A42F20F7288
:10D9000093420CDD4B4B1B6A01334A4A1362494B6D
:10D910009B6AA3F51C53103B464A9362ECE700BF99
:10D92000444B1B6A434A926893420EDB414B0222EE
:10D930009A61404B9B681A463E4B1A623D4B1A6BEC
:10D940003C4BDB6AD31A3B4A53633A4B9B69032B2C
:10D9500028D1384B9B6A1A46364B5B6AD31A1A4653
:10D96000344B9A62334B9B6A002B10DA314B1B6AA3
:10D97000002B0CDD2F4B1B6A013B2E4A13622D4BF3
:10D980009B6A03F51C5310332A4A9362EAE7294B3A
:10D990001B6A284A5268934204DC264B5B681A468D
:10D9A000244B1A62234B9B69042B03D0214B9B69A8
:10D9B000052B3DD11F4B9B6A1A461E4B5B6AD31A3F
:10D9C0001A461C4B9A621B4B9B6A002B10DA194BB0
:10D9D0001B6A002B0CDD174B1B6A013B154A1362B7
:10D9E000144B9B6A03F51C531033124A9362EAE707
:10D9F000104B1B6A0F4A5268934219DC0E490320F0
:10DA0000FFF704F90C490320FFF7ACF90B48FFF7C7
:10DA100047F8084B00229A61064B0022DA63054B57
:10DA2000DB6F002B04D0034BDB6F984700E000BF97
:10DA300080BD00BF94300020DC3000200048014051
:10DA400080B485B000AFF860B9607A603B60094A85
:10DA5000FB681360084ABB681360084A7B68136060
:10DA6000074A3B68136000BF1437BD465DF8047B6E
:10DA7000704700BF9C040020A0040020A4040020E4
:10DA8000A804002080B500AF0948FFF727F8084830
:10DA9000FFF755F80648FFF703F8802200210548F4
:10DAA00016F0C8FE034B01221A6000BF80BD00BF04
:10DAB000001800401431002080B500AF5148FFF736
:10DAC0001BF80346002B00F09A804E48FFF706F83B
:10DAD0004D4BDA6A4C4B1B6B9A4203D24A4B9B6903
:10DAE000002B1CDC49490420FFF790F8474904202B
:10DAF000FFF738F94348FEF7D3FF434B9B69002BF0
:10DB00007CDD414B00229A613F4B0022DA633E4BA1
:10DB1000DB6F002B72D03C4BDB6F98476EE03A4BCB
:10DB20001B6A3B4A92FBF3F3DA0F13445B109BB280
:10DB300019463448FEF7C4FF334B9B6B002B25D1AD
:10DB4000314B01229A63304BDB6A01332E4AD36298
:10DB50002D4B5A692C4BDB6913442B4A53612A4BDA
:10DB60001B68002B0DD1284BDB69012B04D1274901
:10DB70000420FEF7F5FF1DE024490420FFF79CF880
:10DB800018E022490420FEF7EBFF13E01E4B0022B1
:10DB90009A631D4B1B68002B08D11C490420FFF71A
:10DBA00035F81A490420FFF7DDF803E0174904208F
:10DBB000FFF72CF8144B9B69012B0DD1124BDA6A3D
:10DBC000114B1B6B5B089A4206D30F4B03229A61E1
:10DBD0000D4BDB6A0C4A53630B4B9B69022B0ED136
:10DBE000094BDA6A084B5B6B9A4208D3064B032257
:10DBF0009A61054BDB68044A536200E000BF00BF36
:10DC000080BD00BF00180040143100205C310020AE
:10DC1000C027090080B500AF8A4B9B69002B40F3F9
:10DC20000E81884BDB6B002B00F00981854B1B6F4D
:10DC3000002B5CD1834B1B6C002B58D0814B5B6C51
:10DC40000133804A53647F4B5A6C7E4B1B6C9A4263
:10DC50004DD37C4B00225A647A4B1B6E002B19D09B
:10DC6000784B9B69012B07D0764B9B69022B03D025
:10DC7000744B9B69032B0DD1724B1B6E714A926ED4
:10DC80007049C96E104698470346002B02D06D4B71
:10DC900004229A616B4B5B6E002B21D0694B9B6910
:10DCA000012B0BD0674B9B69022B07D0654B9B69FF
:10DCB000032B03D0634B9B69042B11D1614B5B6E2B
:10DCC000604A926E5F49C96E104698470346002B22
:10DCD00006D05C4B1B695B4A53625A4B05229A6122
:10DCE000584B5B6F002B02D0564B5B6F9847554BE0
:10DCF0009B69012B31D1534B9B6A1A46514B5B6A8E
:10DD000013441A464F4B9A624E4B9B6A42F20F7273
:10DD100093420CDD4B4B1B6A01334A4A1362494B59
:10DD20009B6AA3F51C53103B464A9362ECE700BF85
:10DD3000444B1B6A434A926893420EDB414B0222DA
:10DD40009A61404B9B681A463E4B1A623D4B1A6BD8
:10DD50003C4BDB6AD31A3B4A53633A4B9B69032B18
:10DD600028D1384B9B6A1A46364B5B6AD31A1A463F
:10DD7000344B9A62334B9B6A002B10DA314B1B6A8F
:10DD8000002B0CDD2F4B1B6A013B2E4A13622D4BDF
:10DD90009B6A03F51C5310332A4A9362EAE7294B26
:10DDA0001B6A284A5268934204DC264B5B681A4679
:10DDB000244B1A62234B9B69042B03D0214B9B6994
:10DDC000052B3DD11F4B9B6A1A461E4B5B6AD31A2B
:10DDD0001A461C4B9A621B4B9B6A002B10DA194B9C
:10DDE0001B6A002B0CDD174B1B6A013B154A1362A3
:10DDF000144B9B6A03F51C531033124A9362EAE7F3
:10DE0000104B1B6A0F4A5268934219DC0E490420DA
:10DE1000FEF7FCFE0C490420FEF7A4FF0B48FEF7BA
:10DE20003FFE084B00229A61064B0022DA63054B45
:10DE3000DB6F002B04D0034BDB6F984700E000BF83
:10DE400080BD00BF143100205C310020001800406C
:10DE500080B485B000AFF860B9607A603B60094A71
:10DE6000FB681360084ABB681360084A7B6813604C
:10DE7000074A3B68136000BF1437BD465DF8047B5A
:10DE8000704700BFAC040020B0040020B4040020A0
:10DE9000B804002080B500AF0948FEF71FFE08480F
:10DEA000FEF74DFE0648FEF7FBFD802200210548E7
:10DEB00016F0C0FC034B01221A6000BF80BD00BFFA
:10DEC000001C00409431002080B500AF5148FEF79F
:10DED00013FE0346002B00F09A804E48FEF7FEFD2D
:10DEE0004D4BDA6A4C4B1B6B9A4203D24A4B9B69EF
:10DEF000002B1CDC49490520FEF788FE4749052018
:10DF0000FEF730FF4348FEF7CBFD434B9B69002BE8
:10DF10007CDD414B00229A613F4B0022DA633E4B8D
:10DF2000DB6F002B72D03C4BDB6F98476EE03A4BB7
:10DF30001B6A3B4A92FBF3F3DA0F13445B109BB26C
:10DF400019463448FEF7BCFD334B9B6B002B25D1A3
:10DF5000314B01229A63304BDB6A01332E4AD36284
:10DF60002D4B5A692C4BDB6913442B4A53612A4BC6
:10DF70001B68002B0DD1284BDB69012B04D12749ED
:10DF80000520FEF7EDFD1DE024490520FEF794FE77
:10DF900018E022490520FEF7E3FD13E01E4B0022A6
:10DFA0009A631D4B1B68002B08D11C490520FEF706
:10DFB0002DFE1A490520FEF7D5FE03E0174905207E
:10DFC000FEF724FE144B9B69012B0DD1124BDA6A2C
:10DFD000114B1B6B5B089A4206D30F4B03229A61CD
:10DFE0000D4BDB6A0C4A53630B4B9B69022B0ED122
:10DFF000094BDA6A084B5B6B9A4208D3064B032243
:10E000009A61054BDB68044A536200E000BF00BF21
:10E0100080BD00BF001C004094310020DC31002096
:10E02000C027090080B500AF8A4B9B69002B40F3E5
:10E030000E81884BDB6B002B00F00981854B1B6F39
:10E04000002B5CD1834B1B6C002B58D0814B5B6C3D
:10E050000133804A53647F4B5A6C7E4B1B6C9A424F
:10E060004DD37C4B00225A647A4B1B6E002B19D087
:10E07000784B9B69012B07D0764B9B69022B03D011
:10E08000744B9B69032B0DD1724B1B6E714A926EC0
:10E090007049C96E104698470346002B02D06D4B5D
:10E0A00004229A616B4B5B6E002B21D0694B9B69FC
:10E0B000012B0BD0674B9B69022B07D0654B9B69EB
:10E0C000032B03D0634B9B69042B11D1614B5B6E17
:10E0D000604A926E5F49C96E104698470346002B0E
:10E0E00006D05C4B1B695B4A53625A4B05229A610E
:10E0F000584B5B6F002B02D0564B5B6F9847554BCC
:10E100009B69012B31D1534B9B6A1A46514B5B6A79
:10E1100013441A464F4B9A624E4B9B6A42F20F725F
:10E1200093420CDD4B4B1B6A01334A4A1362494B45
:10E130009B6AA3F51C53103B464A9362ECE700BF71
:10E14000444B1B6A434A926893420EDB414B0222C6
:10E150009A61404B9B681A463E4B1A623D4B1A6BC4
:10E160003C4BDB6AD31A3B4A53633A4B9B69032B04
:10E1700028D1384B9B6A1A46364B5B6AD31A1A462B
:10E18000344B9A62334B9B6A002B10DA314B1B6A7B
:10E19000002B0CDD2F4B1B6A013B2E4A13622D4BCB
:10E1A0009B6A03F51C5310332A4A9362EAE7294B12
:10E1B0001B6A284A5268934204DC264B5B681A4665
:10E1C000244B1A62234B9B69042B03D0214B9B6980
:10E1D000052B3DD11F4B9B6A1A461E4B5B6AD31A17
:10E1E0001A461C4B9A621B4B9B6A002B10DA194B88
:10E1F0001B6A002B0CDD174B1B6A013B154A13628F
:10E20000144B9B6A03F51C531033124A9362EAE7DE
:10E21000104B1B6A0F4A5268934219DC0E490520C5
:10E22000FEF7F4FC0C490520FEF79CFD0B48FEF7B9
:10E2300037FC084B00229A61064B0022DA63054B3B
:10E24000DB6F002B04D0034BDB6F984700E000BF6F
:10E2500080BD00BF94310020DC310020001C004054
:10E2600080B485B000AFF860B9607A603B60094A5D
:10E27000FB681360084ABB681360084A7B68136038
:10E28000074A3B68136000BF1437BD465DF8047B46
:10E29000704700BFBC040020C0040020C40400205C
:10E2A000C804002080B500AF0948FEF717FC0848F5
:10E2B000FEF745FC0648FEF7F3FB802200210548E7
:10E2C00016F0B8FA034B01221A6000BF80BD00BFF0
:10E2D000002000401432002080B500AF5148FEF706
:10E2E0000BFC0346002B00F09A804E48FEF7F6FB2D
:10E2F0004D4BDA6A4C4B1B6B9A4203D24A4B9B69DB
:10E30000002B1CDC49490620FEF780FC474906200B
:10E31000FEF728FD4348FEF7C3FB434B9B69002BE8
:10E320007CDD414B00229A613F4B0022DA633E4B79
:10E33000DB6F002B72D03C4BDB6F98476EE03A4BA3
:10E340001B6A3B4A92FBF3F3DA0F13445B109BB258
:10E3500019463448FEF7B4FB334B9B6B002B25D199
:10E36000314B01229A63304BDB6A01332E4AD36270
:10E370002D4B5A692C4BDB6913442B4A53612A4BB2
:10E380001B68002B0DD1284BDB69012B04D12749D9
:10E390000620FEF7E5FB1DE024490620FEF78CFC75
:10E3A00018E022490620FEF7DBFB13E01E4B00229B
:10E3B0009A631D4B1B68002B08D11C490620FEF7F1
:10E3C00025FC1A490620FEF7CDFC03E0174906207C
:10E3D000FEF71CFC144B9B69012B0DD1124BDA6A22
:10E3E000114B1B6B5B089A4206D30F4B03229A61B9
:10E3F0000D4BDB6A0C4A53630B4B9B69022B0ED10E
:10E40000094BDA6A084B5B6B9A4208D3064B03222E
:10E410009A61054BDB68044A536200E000BF00BF0D
:10E4200080BD00BF00200040143200205C3200207C
:10E43000C027090080B500AF8A4B9B69002B40F3D1
:10E440000E81884BDB6B002B00F00981854B1B6F25
:10E45000002B5CD1834B1B6C002B58D0814B5B6C29
:10E460000133804A53647F4B5A6C7E4B1B6C9A423B
:10E470004DD37C4B00225A647A4B1B6E002B19D073
:10E48000784B9B69012B07D0764B9B69022B03D0FD
:10E49000744B9B69032B0DD1724B1B6E714A926EAC
:10E4A0007049C96E104698470346002B02D06D4B49
:10E4B00004229A616B4B5B6E002B21D0694B9B69E8
:10E4C000012B0BD0674B9B69022B07D0654B9B69D7
:10E4D000032B03D0634B9B69042B11D1614B5B6E03
:10E4E000604A926E5F49C96E104698470346002BFA
:10E4F00006D05C4B1B695B4A53625A4B05229A61FA
:10E50000584B5B6F002B02D0564B5B6F9847554BB7
:10E510009B69012B31D1534B9B6A1A46514B5B6A65
:10E5200013441A464F4B9A624E4B9B6A42F20F724B
:10E5300093420CDD4B4B1B6A01334A4A1362494B31
:10E540009B6AA3F51C53103B464A9362ECE700BF5D
:10E55000444B1B6A434A926893420EDB414B0222B2
:10E560009A61404B9B681A463E4B1A623D4B1A6BB0
:10E570003C4BDB6AD31A3B4A53633A4B9B69032BF0
:10E5800028D1384B9B6A1A46364B5B6AD31A1A4617
:10E59000344B9A62334B9B6A002B10DA314B1B6A67
:10E5A000002B0CDD2F4B1B6A013B2E4A13622D4BB7
:10E5B0009B6A03F51C5310332A4A9362EAE7294BFE
:10E5C0001B6A284A5268934204DC264B5B681A4651
:10E5D000244B1A62234B9B69042B03D0214B9B696C
:10E5E000052B3DD11F4B9B6A1A461E4B5B6AD31A03
:10E5F0001A461C4B9A621B4B9B6A002B10DA194B74
:10E600001B6A002B0CDD174B1B6A013B154A13627A
:10E61000144B9B6A03F51C531033124A9362EAE7CA
:10E62000104B1B6A0F4A5268934219DC0E490620B0
:10E63000FEF7ECFA0C490620FEF794FB0B48FEF7B8
:10E640002FFA084B00229A61064B0022DA63054B31
:10E65000DB6F002B04D0034BDB6F984700E000BF5B
:10E6600080BD00BF143200205C320020002000403A
:10E6700080B500AF0548FEF731FA0448FEF74FFABF
:10E680000248FEF7FDF900BF80BD00BF0004014055
:10E6900080B500AF0B48FEF72FFA0346002B0ED0D3
:10E6A0000848FEF71BFAFEF79DFCFEF7A3FEFFF7F6
:10E6B000A9F8FFF7AFFAFFF7B5FCFFF7BBFE00BF05
:10E6C00080BD00BF0004014080B500AFFFF7D0FF60
:10E6D000FEF7C0FBFEF7C6FDFEF7CCFFFFF7D2F951
:10E6E000FFF7D8FBFFF7DEFD00BF80BD80B582B02D
:10E6F00000AF786040F21F420021786816F09AF867
:10E7000000BF0837BD4680BD80B588B000AFF86057
:10E710000B467A60FB72FB68B3F5005F0AD37B6837
:10E72000D3F819301A46F968294816F0F5FC4FF06D
:10E73000FF3348E0FB68DB087B617B69B3F5806FE2
:10E740000BD37B68B3F81D309BB21A467969214818
:10E7500016F0E2FC4FF0FF3335E0FB6803F00703EF
:10E76000BB610123FB7705E0BB69013BBB61FB7F1C
:10E770005B00FB77BB69002BF6D1FB7A002B13D132
:10E780007A687B6913441F331B785AB297F91F309C
:10E79000DB435BB213405BB2D9B27A687B69134446
:10E7A0001F330A461A700DE07A687B6913441F33E1
:10E7B0001A78FB7F1343D9B27A687B6913441F33FD
:10E7C0000A461A70002318462037BD4680BD00BF98
:10E7D000E48F03081490030880B487B000AF78601A
:10E7E0007B68D3F81930DB08FB607B68D3F81930FD
:10E7F00003F00703BB6000233B610BE07A683B69D1
:10E8000013441F331B78FF2B01D0002322E03B6908
:10E8100001333B613A69FB689A42EFD30123FB75F0
:10E8200000233B6111E07A68FB6813441F331A78B8
:10E83000FB7D1340DBB2002B01D100230AE0FB7DFE
:10E840005B00FB753B6901333B613A69BB689A42E7
:10E85000E9D3012318461C37BD465DF8047B704799
:10E8600080B500AF0CF08AFBF9F734FCF9F78AFAAF
:10E87000FAF70AFAF6F7A4FE0AF0F6FE13F046F8E5
:10E880000CF082FB10F0CAF813F0ECFE0EF050FF13
:10E890000A4816F0DDFCFAF703F909F097FC00F0DE
:10E8A0000FF8F9F7EBFCF9F73DF810F02DFBF7F74F
:10E8B00013F909F047FD13F007FFF2E7349103085D
:10E8C00080B582B000AF002228494FF4FA70F9F702
:10E8D00037FC45F2AA5009F09BFD45F2AA5000F022
:10E8E000CDFA2348F7F7D6F8F8F7C0FBF9F7C6FCDE
:10E8F000F9F718F810F008FB13F0E6FE09F022FD16
:10E900000AF0DAFE0346FB80FB881B0A9BB2022B4F
:10E9100007D018233B6038680AF0EEFB154816F064
:10E9200097FC0AF0E3FE0346FB80FB88002B07D12F
:10E9300009233B6038680AF0DFFB0F4816F088FCBB
:10E94000F7F746F80346002B04D00A233B603868EB
:10E950000AF0D2FBF7F7AEF800F0BAF8074816F065
:10E9600077FC00BF0837BD4680BD00BF2DA9020857
:10E970009D8302086C910308849103089C9103080D
:10E9800080B582B002AF782200212D4815F052FFE9
:10E9900008F05EF82B4808F025FD2B4809F006FC2E
:10E9A0002A4B2B4AC3F87424284B2A4AC3F87824EC
:10E9B000294A00213C20F9F7C3FB00230193274B90
:10E9C00000930023002200212548F6F731FE254A56
:10E9D00025492648F8F736FF254A23492548F8F700
:10E9E00031FF254A25492648F8F72CFF254A2649B4
:10E9F0002648F8F727FF264A26492748F8F722FF36
:10EA0000264A27492748F8F71DFF274A274928485B
:10EA1000F8F718FF274A28492848F8F713FF284A2B
:10EA200028492948F8F70EFF084BDB6919462748A3
:10EA300016F072FB054B00229A6100BFBD4680BDF7
:10EA40009C370020A4D10308E4D20308303800200A
:10EA500099EB010871EC0108DDEC010865EE010895
:10EA6000A5AA0208F5610208B0910308C491030841
:10EA70007D610208CC910308E9630208D091030884
:10EA8000E09103082D640208E8910308F891030857
:10EA9000396A0208049203080C9203087D63020895
:10EAA0001492030824920308A16702083092030815
:10EAB00040920308616802084C92030854920308CC
:10EAC000896902085C9203086C9203087492030837
:10EAD00080B500AFC82000F004F800F039FC00BF9A
:10EAE00080BD80B590B000AF786007F10C03342290
:10EAF0000021184615F09EFE48F239033B820023A0
:10EB00007B8240F20113BB824FF40073FB8248F218
:10EB100039033B8300237B8340F20113BB834FF413
:10EB20000073FB8348F239033B8400237B8440F26B
:10EB30000113BB844FF40073FB8448F239033B8517
:10EB400000237B8540F20113BB854FF40073FB85E6
:10EB500048F239033B8600237B8640F20113BB86D3
:10EB60004FF40073FB8648F201033B8701237B8748
:10EB700040F20113BB874FF40073FB870123FB6056
:10EB800007F10C0318460CF013FB7868F8F752FAFB
:10EB900000BF4037BD4680BD80B500AF00F002F831
:10EBA00000BF80BD98B500AF002012F011FD0346F4
:10EBB000012B51D1294816F04BFB0021002012F007
:10EBC000F7FC274B1B6823F48063254A1360254814
:10EBD00016F03EFB244B5B69DA6A214BD3F83031E7
:10EBE0009A420FD1204B5B691B8E9CB212F070FDD4
:10EBF000034623449AB21A4BD3F818311B0C9BB22C
:10EC00009A4224D0164BD3F818319BB2144AC2F85A
:10EC10001831154B5B691B8E9BB21C4612F058FDD8
:10EC2000034623441A040E4BD3F8183113430C4AFD
:10EC3000C2F818310C4B5B69DB6A094AC2F8303103
:10EC400009F0DCFB094816F003FB0AF093FB04F023
:10EC5000D7F801200AF098FA00BF98BD88920308FF
:10EC60003038002098920308D8490020B492030855
:10EC700080B582B000AF00237B60094B1B6803F4B2
:10EC80000073002B08D100F00DF878607B68002B32
:10EC900002D078680AF030FA00BF0837BD4680BD60
:10ECA0003038002080B582B000AF00237B607B68E5
:10ECB000002B0ED10BF058FF0346002B02D10BF0B6
:10ECC000C1F906E00BF042FF0346002B01D10BF027
:10ECD000CFF97B6818460837BD4680BD80B500AFC8
:10ECE00001200AF051FA002014F02EFB00BF80BD75
:10ECF00080B582B000AF0BF037F90BF061F90CF082
:10ED000026F90BF005F90BF087F90BF0D5F8002385
:10ED10007B607B6818460837BD4680BD80B582B0F1
:10ED200000AF00237B600BF01FFF0346002B04D0D5
:10ED30000BF00CFF0346002B02D00BF083F906E02A
:10ED40000BF004FF0346002B01D10BF091F97B6817
:10ED500018460837BD4680BD80B582B000AF034677
:10ED6000FB803E4B1B68D3F84433012B71D13C4BE5
:10ED700093F85130012B6CD10BF004FF0346002BAC
:10ED80000AD1374B0A2283F84920354BDA6CFB88CD
:10ED9000D31A334AD36418E00BF0F4FE0346002B79
:10EDA00013D02F4B93F849300A2B0ED12C4B002255
:10EDB00083F84920294B1B68D3F848331A46284B5F
:10EDC000DA64274B022283F850200BF0DBFE034667
:10EDD000002B0AD0224B0A2283F84A20204BDA6CFF
:10EDE000FB88D31A1E4AD36418E00BF0CBFE03460F
:10EDF000002B13D11A4B93F84A300A2B0ED1184B23
:10EE0000002283F84A20154B1B68D3F848331A4672
:10EE1000134BDA64124B022283F85020104BDB6C48
:10EE2000002B03DC0E4B002283F850200C4B93F890
:10EE30005030002B0DD14FF441700AF05DF9084BB2
:10EE40000122DA65064B022283F850204FF48073CA
:10EE500000E0002318460837BD4680BDE40C0020C2
:10EE60009C37002080B500AF034816F0F1F906F09A
:10EE7000DFFE0023184680BDD892030880B588B015
:10EE800000AF78607B6803F4AA43B3F5AA4F49D179
:10EE90002A4816F0DDF92A4816F03EF907F1080372
:10EEA00018220021184615F0C5FC264B1B68D3F824
:10EEB000C830BB60234B1B68D3F8CC30FB60214BC0
:10EEC0001B68D3F8D0303B611E4B1B68D3F8D83099
:10EED00042F2107202FB03F31B4A82FB03129213ED
:10EEE000DB17D31A7B61174B1B68D3F8C830BB61A3
:10EEF000144B1B68D3F8C830FB6107F108031846B0
:10EF000000F028F80F4B1B68D3F820230F4BD3F8E1
:10EF1000FC339A4206D00B4B1B68D3F820330B4AC4
:10EF2000C2F8FC337B6803F0AA03AA2B02D108487D
:10EF300016F08EF900BF2037BD4680BDF49203085D
:10EF400010930308E40C00206B29827430380020F1
:10EF50001C93030880B584B000AF78607B68002BF9
:10EF60000FD10D4816F074F9182200210B4815F046
:10EF700061FC0B4B0022C3F80822094B0022C3F8A6
:10EF80000C220AF02DFA074816F062F9064816F02E
:10EF90005FF90023FB6017E038930308403A002034
:10EFA000303800204C93030868930308FB68591C11
:10EFB000AC4AFB689B0013445B681A46AA4816F0EB
:10EFC000ABF8FB680133FB60FB68052BEEDDA74B5C
:10EFD000D3F80C3245F2AA52934231D1A34BD3F865
:10EFE000083203F00103002B2AD07B681B681A4605
:10EFF0009F49A04816F090F89C4BD3F81032194660
:10F000009D4816F089F87B681A68984BD3F810323F
:10F01000D31ABB60934B5B68BA681344BB60B96892
:10F02000964816F079F88F4B5B68BA681946944891
:10F0300016F072F8B96800200CF08EF80AF0D0F9DA
:10F040008A4BD3F80C3245F2AA52934233D1874B04
:10F05000D3F8083203F00203002B2CD07B68043372
:10F060001B681A468749834816F056F87F4BD3F839
:10F0700014321946804816F04FF87B6804331A683A
:10F080007A4BD3F81432D31ABB60764B9B68BA68BC
:10F090001344BB60B968794816F03EF8714B9B6821
:10F0A000BA681946764816F037F8B96801200CF0AE
:10F0B00053F80AF095F96D4BD3F80C3245F2AA5289
:10F0C000934233D1694BD3F8083203F00403002B89
:10F0D0002CD07B6808331B681A466B49654816F0CC
:10F0E0001BF8624BD3F818321946634816F014F82F
:10F0F0007B6808331A685D4BD3F81832D31ABB60AB
:10F10000584BDB68BA681344BB60B9685B4816F0BB
:10F1100003F8544BDB68BA681946594815F0FCFFF0
:10F12000B96802200CF018F80AF05AF94F4BD3F8DE
:10F130000C3245F2AA52934233D14C4BD3F80832E9
:10F1400003F00803002B2CD07B680C331B681A4695
:10F150004E49484815F0E0FF444BD3F81C3219469D
:10F16000454815F0D9FF7B680C331A683F4BD3F83C
:10F170001C32D31ABB603B4B1B69BA681344BB609B
:10F18000B9683E4815F0C8FF364B1B69BA68194686
:10F190003B4815F0C1FFB96803200BF0DDFF0AF012
:10F1A0001FF9324BD3F80C3245F2AA52934233D1B5
:10F1B0002E4BD3F8083203F02003002B2CD07B68B1
:10F1C00014331B681A4632492A4815F0A5FF274B0D
:10F1D000D3F824321946284815F09EFF7B68143373
:10F1E0001A68224BD3F82432D31ABB601D4B9B699B
:10F1F000BA681344BB60B968204815F08DFF194BFD
:10F200009B69BA6819461E4815F086FFB968052043
:10F210000BF0A2FF0AF0E4F8144BD3F80C3245F2DD
:10F22000AA5293424ED1114BD3F8083203F0100387
:10F23000002B47D07B6810331B681A4615490D48D0
:10F2400015F06AFF094BD3F8203219460A4815F029
:10F2500063FF7B6810331A68044BD3F82032D31A4B
:10F26000BB6019E0BC4900208493030830380020BB
:10F270009493030898930308B0930308CC9303086E
:10F28000E0930308FC930308009403080894030820
:10F2900010940308189403081F4B5B69BA68134461
:10F2A000BB60B9681D4815F037FF1B4B5B69BA6836
:10F2B00019461B4815F030FFB96804200BF04CFFCD
:10F2C0000AF08EF87B68002B09D01822796815485F
:10F2D00015F0A2FA144B45F2AA52C3F80C221348B7
:10F2E00015F0B6FF0023FB600DE0FB68591C0A4ACD
:10F2F000FB689B0013445B681A460D4815F00CFF31
:10F30000FB680133FB60FB68052BEEDD00BF00BF2F
:10F310001037BD4680BD00BFBC490020CC93030818
:10F32000E0930308403A002030380020209403087E
:10F330008493030880B500AF18220349034815F0F1
:10F340006BFA00BF80BD00BFC049002050380020CC
:10F3500080B400AF0E4B1B68D3F828310D4A136000
:10F360000B4B1B68D3F830310A4A9360084B1B687B
:10F37000D3F82C31074A5360054B1B68D3F834315E
:10F38000044AD36000BFBD465DF8047B704700BFF0
:10F39000E40C00201438002080B400AF0D4B1B6833
:10F3A00045F2AA5293420ED10B4BD3F8083203F028
:10F3B0000103002B07D0074B5A68084B5B689A4241
:10F3C00001DD002300E001231846BD465DF8047B03
:10F3D000704700BFBC49002030380020143800209E
:10F3E00080B400AF0D4B1B6845F2AA5293420ED178
:10F3F0000B4BD3F8083203F00103002B07D0074B67
:10F400005A68084B1B689A4201DA002300E0012386
:10F410001846BD465DF8047B704700BFBC4900201C
:10F42000303800201438002080B584B000AF7860F8
:10F430000023FB6013F06AFF0346012B02D14FF457
:10F440008073FB60FB6818461037BD4680BD000026
:10F4500080B59CB000AF7860396000237B6601F016
:10F460000FFE78667B6E002B04D0786E09F044FEA8
:10F470007B6E76E007F10C0358220021184615F048
:10F48000D9F90123BB810023FB8148F239033B8278
:10F4900000237B820123BB827B68344A02FB03F397
:10F4A000BB614FF47A73BB63314B1B68D3F8903167
:10F4B000FB663B68012B05DC2D4B1B68D3F8A431A0
:10F4C000BB6610E03B68022B05D1294B1B68D3F8C3
:10F4D000A831BB6607E03B68022B04DD244B1B68A8
:10F4E000D3F8AC31BB66FA6EBB6E9A4201DDBB6EDF
:10F4F000FB66FB6E642202FB03F3FB63BB6E6422BC
:10F5000002FB03F33B641A4B1B68D3F89C31194A86
:10F51000B2FBF3F37B64164B1B68D3F8A031154A9A
:10F52000B2FBF3F3BB64144BFB64144B3B65002349
:10F530007B65134BBB65134B1B6843F04003114ABB
:10F54000136007F10C03184610F062FD78660D4B4E
:10F550001B6823F040030B4A1360786E09F0CCFD62
:10F560007B6E18467037BD4680BD00BF400D03005E
:10F57000E40C002080FC0A002DF6010843F6010887
:10F5800029F401083038002080B584B000AF7860DD
:10F5900039607B687B810FF0F3FCF860FB68002B1F
:10F5A00001D0FB681AE0B7F90A30002B07DDFFF73E
:10F5B000F3FE0346002B10D12323FB600DE0B7F9C7
:10F5C0000A30002B07DAFFF70BFF0346002B04D1AC
:10F5D0002423FB6001E00023FB60FB681846103722
:10F5E000BD4680BD80B584B000AF786039600FF053
:10F5F000D3FCF860FB6818461037BD4680BD80B567
:10F6000084B000AF786039600FF0D2FCF86009F088
:10F61000FDFEF7F7D5FB0346002B02D04FF48073B5
:10F62000FB60FB6818461037BD4680BD80B582B0D0
:10F6300000AF7860FFF7B0FE034618460837BD46B6
:10F6400080BD80B582B000AF7860FFF7C9FE034689
:10F6500018460837BD4680BD80B5B6B000AF7860AB
:10F6600039600023A7F8D4307B68002B01D1002338
:10F67000D2E03B68002B22D1694B1B68D3F8903154
:10F68000642202FB03F3BB60654B1B68D3F898311F
:10F69000642202FB03F3FB60614B1B68D3F89C31CF
:10F6A000604AB2FBF3F33B615D4B1B68D3F8A031BA
:10F6B0005C4AB2FBF3F37B6107F108033B607B68B4
:10F6C000002B04DA4FF6FF73A7F8D63009E07B6809
:10F6D000002B03DD0123A7F8D63002E00023A7F8B2
:10F6E000D63007F11803B4220021184615F0A2F80D
:10F6F0000123BB610023FB61B7F8D430DB00D833B2
:10F700003B4448F2390223F8B82CB7F8D430DB0078
:10F71000D8333B44002223F8B62CBB699BB203F0DC
:10F720000F039AB2B7F8D43042F4807292B2DB0081
:10F73000D8333B4423F8B42CB7F8D430DB00D833AB
:10F740003B444FF4007223F8B22CB7F8D4300E3398
:10F750009B00D8333B447A6843F8C02C0023BB6637
:10F760007B68002BB8BF5B42FB664FF47A733B6744
:10F770003B681B687B673B681B68BB673B685B68D3
:10F78000FB673B681B68C7F880303B689B68C7F81D
:10F7900084303B689B68C7F888303B68DB68C7F8F3
:10F7A0008C300023C7F890301F4BC7F898301F4BA0
:10F7B000C7F89C300023C7F8A0300023C7F8A43056
:10F7C0000023C7F8A8300023C7F8AC30BB69C7F8DE
:10F7D000B030174BC7F8C030164BC7F8BC30164BCB
:10F7E000C7F8B830B7F9D6309BB2C7F8C430BB6998
:10F7F000C7F8C83007F1180318460BF0E1FEC7F848
:10F80000D000D7F894301946D7F8D00010F02EFD6C
:10F81000C7F8CC00D7F8CC301846D837BD4680BDE5
:10F82000E40C002080FC0A009D8302083194020849
:10F8300089F50108E5F50108FFF5010880B582B0FA
:10F8400000AF0023FB710BF0F5F80346002B04D149
:10F85000FB79002B01D1002300E001231846083773
:10F86000BD4680BD80B5A0B000AF0123BB670023BB
:10F87000FB67934BD3F8083223F00103904AC2F898
:10F88000083209F0ADFD07F1140364220021184687
:10F8900014F0D0FF0123BB820023FB8248F239031E
:10F8A0003B8300237B830123BB83BB6F854A02FB21
:10F8B00003F33B62BB6F844A02FB03F37B62834B1F
:10F8C0001B68D3F89031642202FB03F37B647F4B07
:10F8D0001B68D3F89431642202FB03F3BB647B4BB7
:10F8E0001B68D3F89C317A4AB2FBF3F3FB64774B85
:10F8F0001B68D3F8A031764AB2FBF3F33B65754B36
:10F90000BB65754B3B66754B7B660023BB66744BD2
:10F910003B676B4B1B6843F04003694A136007F178
:10F920001403184610F000F9F867642008F036FD5B
:10F93000FB6F40F20112934240F08880FFF77EFF98
:10F940000346002B40F08280604B1B68D3F8903157
:10F95000642202FB03F37B605C4B1B68D3F8943199
:10F96000642202FB03F3BB60584B1B68D3F89C3145
:10F97000574AB2FBF3F3FB60544B1B68D3F8A0313A
:10F98000534AB2FBF3F33B61BB6F4F4A02FB03F3F5
:10F990003A1D11461846FFF75FFE0123BB82002384
:10F9A000FB8248F239033B8300237B830123BB8323
:10F9B000BB6F4FF47A6202FB03F33B62BB6F424AB8
:10F9C00002FB03F37B6264237B644FF47A73BB64B2
:10F9D000444BFB644FF4E1533B653E4BBB653E4BF0
:10F9E0003B663E4B7B660023BB663D4B3B6707F1A6
:10F9F0001403184610F098F8F867642008F0CEFC5D
:10FA0000FB6F40F20112934213D1FFF717FF034639
:10FA1000002B0ED12A4BD3F8083243F00103284AB9
:10FA2000C2F80832304815F013FC40F20113FB67AE
:10FA300018E0234BD3F8083223F00103204AC2F820
:10FA40000832F96F294815F067FB0BE01C4BD3F81F
:10FA5000083223F001031A4AC2F80832F96F23482A
:10FA600015F05AFB164B1B6823F04003144A136031
:10FA70001F4B5B68124AD2F8102219461D4815F038
:10FA80004BFB124B1B68D3F8C8300D4AC2F810323A
:10FA90000B4BD3F81032194600200BF05DFB09F038
:10FAA0009FFC134B5B681946134815F035FBF86F44
:10FAB00009F022FBFB6F18468037BD4680BD00BFB2
:10FAC00030380020400D030030F8FFFFE40C002028
:10FAD00080FC0A003DF8010899F30108E1F30108F0
:10FAE00059F601084019010064940308789403084A
:10FAF000BC49002094940308B894030880B400AF74
:10FB00000D4B1B6845F2AA5293420ED10B4BD3F812
:10FB1000083203F00203002B07D0074B9A68084B0A
:10FB2000DB689A4201DD002300E001231846BD4650
:10FB30005DF8047B704700BFBC49002030380020CE
:10FB40001438002080B400AF0D4B1B6845F2AA5258
:10FB500093420ED10B4BD3F8083203F00203002B73
:10FB600007D0074B9A68084B9B689A4201DA00233A
:10FB700000E001231846BD465DF8047B704700BFD6
:10FB8000BC490020303800201438002080B582B0F5
:10FB900000AF7860FFF7B2FF034618460837BD464E
:10FBA00080BD80B582B000AF7860FFF7CBFF034621
:10FBB00018460837BD4680BD80B485B000AF786078
:10FBC0000C4B1B6845F2AA52934209D10A4BD3F859
:10FBD000083203F00203002B02D00023FB6001E097
:10FBE0002123FB60FB6818461437BD465DF8047B93
:10FBF000704700BFBC4900203038002080B584B079
:10FC000000AF78600023FB6013F080FB0346012BFC
:10FC100002D14FF48073FB60FB6818461037BD4675
:10FC200080BD000080B59CB000AF786039600023D3
:10FC30007B6601F025FA78667B6E002B04D0786E27
:10FC400009F05AFA7B6E76E007F10C035822002186
:10FC5000184614F0EFFD0123BB810123FB8148F21C
:10FC600039033B8200237B820123BB827B68344AB9
:10FC700002FB03F3BB614FF47A73BB63314B1B6828
:10FC8000D3F89031FB663B68012B05DC2D4B1B68DC
:10FC9000D3F8A431BB6610E03B68022B05D1294B99
:10FCA0001B68D3F8A831BB6607E03B68022B04DD74
:10FCB000244B1B68D3F8AC31BB66FA6EBB6E9A421C
:10FCC00001DDBB6EFB66FB6E642202FB03F3FB638C
:10FCD000BB6E642202FB03F33B641A4B1B68D3F830
:10FCE0009C31194AB2FBF3F37B64164B1B68D3F8C3
:10FCF000A031154AB2FBF3F3BB64144BFB64144B05
:10FD00003B65144B7B65144BBB65144B1B6843F080
:10FD10004003124A136007F10C03184610F078F9FB
:10FD200078660E4B1B6823F040030C4A1360786E14
:10FD300009F0E2F97B6E18467037BD4680BD00BF02
:10FD4000400D0300E40C002080FC0A008DFB01083C
:10FD5000A3FB0108B9FB0108FDFB010830380020B6
:10FD600080B584B000AF786039607B687B810FF02C
:10FD700007F9F860FB68002B01D0FB681FE0B7F9BA
:10FD80000A30002B07DDFFF7B9FE0346002B10D128
:10FD90002523FB600DE0B7F90A30002B07DAFFF7E7
:10FDA000D1FE0346002B04D12623FB6001E0002393
:10FDB000FB60FB68002B01D0FB6800E0FB68184685
:10FDC0001037BD4680BD80B584B000AF7860396023
:10FDD0000FF0E2F8F860FB6818461037BD4680BDAA
:10FDE00080B584B000AF786039600FF0E1F8F8605A
:10FDF000FEF758FFF860FB68002B01D0FB6800E0BD
:10FE0000FB6818461037BD4680BD000080B5B6B00F
:10FE100000AF786039600123A7F8D4307B68002BED
:10FE200001D10023D2E03B68002B22D1694B1B6833
:10FE3000D3F89031642202FB03F3BB60654B1B686F
:10FE4000D3F89831642202FB03F3FB60614B1B681B
:10FE5000D3F89C31604AB2FBF3F33B615D4B1B6806
:10FE6000D3F8A0315C4AB2FBF3F37B6107F10803DE
:10FE70003B607B68002B04DA4FF6FF73A7F8D6309F
:10FE800009E07B68002B03DD0123A7F8D63002E0F0
:10FE90000023A7F8D63007F11803B4220021184632
:10FEA00014F0C8FC0123BB610023FB61B7F8D43018
:10FEB000DB00D8333B4448F2390223F8B82CB7F8BA
:10FEC000D430DB00D8333B44002223F8B62CBB6986
:10FED0009BB203F00F039AB2B7F8D43042F48072A9
:10FEE00092B2DB00D8333B4423F8B42CB7F8D430BB
:10FEF000DB00D8333B444FF4007223F8B22CB7F840
:10FF0000D4300E339B00D8333B447A6843F8C02C7E
:10FF10000023BB667B68002BB8BF5B42FB664FF4D7
:10FF20007A733B673B681B687B673B681B68BB67F2
:10FF30003B685B68FB673B681B68C7F880303B68C1
:10FF40009B68C7F884303B689B68C7F888303B687B
:10FF5000DB68C7F88C300023C7F890301F4BC7F818
:10FF600098301F4BC7F89C300023C7F8A0300023FF
:10FF7000C7F8A4300023C7F8A8300023C7F8AC3076
:10FF8000BB69C7F8B030174BC7F8C030164BC7F87D
:10FF9000BC30164BC7F8B830B7F9D6309BB2C7F8AB
:10FFA000C430BB69C7F8C83007F1180318460BF016
:10FFB00007FBC7F8D000D7F894301946D7F8D0001F
:10FFC00010F054F9C7F8CC00D7F8CC301846D83721
:10FFD000BD4680BDE40C002080FC0A009D83020821
:10FFE0003194020861FD0108C7FD0108E1FD010827
:10FFF00080B582B000AF0023FB710AF029FD0346F3
:020000040802F0
:10000000002B04D1FB79002B01D1002300E0012358
:1000100018460837BD4680BD80B5A0B000AF7860F7
:100020000023FB67934BD3F8083223F00203914A75
:10003000C2F8083209F0D4F907F11803642200214C
:10004000184614F0F7FB01233B8301237B8348F21E
:100050003903BB830023FB8301233B847B68864AEF
:1000600002FB03F37B627B68844A02FB03F3BB62FF
:10007000834B1B68D3F89031642202FB03F3BB640B
:100080007F4B1B68D3F89431642202FB03F3FB64BB
:100090007B4B1B68D3F89C317A4AB2FBF3F33B6588
:1000A000774B1B68D3F8A031764AB2FBF3F37B653C
:1000B000754BFB65754B7B66754BBB660023FB661A
:1000C000744B7B676B4B1B6843F04003694A1360BA
:1000D00007F1180318460FF027FDF867642008F0B1
:1000E0005DF9FB6F40F20112934240F08980FFF707
:1000F0007FFF0346002B40F08380614B1B68D3F8E1
:100100009031642202FB03F3BB605D4B1B68D3F8A4
:100110009431642202FB03F3FB60594B1B68D3F854
:100120009C31584AB2FBF3F33B61554B1B68D3F843
:10013000A031544AB2FBF3F37B617B684F4A02FB68
:1001400003F307F1080211461846FFF75FFE01238B
:100150003B8301237B8348F23903BB830023FB836A
:1001600001233B847B684FF47A6202FB03F37B62DA
:100170007B68424A02FB03F3BB626423BB644FF417
:100180007A73FB64444B3B654FF4E1537B653E4B14
:10019000FB653E4B7B663E4BBB660023FB663D4BDF
:1001A0007B6707F1180318460FF0BEFCF867642060
:1001B00008F0F4F8FB6F40F20112934213D1FFF7FD
:1001C00017FF0346002B0ED12A4BD3F8083243F019
:1001D0000203284AC2F80832304815F039F840F2D4
:1001E0000113FB6718E0234BD3F8083223F0020316
:1001F000204AC2F80832F96F294814F08DFF0BE04D
:100200001C4BD3F8083223F002031A4AC2F8083212
:10021000F96F234814F080FF164B1B6823F040034E
:10022000144A13601F4B9B68124AD2F814221946D5
:100230001D4814F071FF124B1B68D3F8CC300D4AE7
:10024000C2F814320B4BD3F81432194601200AF0CD
:1002500083FF09F0C5F8134B9B681946134814F047
:100260005BFFF86F08F048FFFB6F18468037BD460C
:1002700080BD00BF30380020400D030030F8FFFF84
:10028000E40C002080FC0A00F1FF0108FDFA0108DF
:1002900045FB01080DFE0108401901006C9503089B
:1002A00080950308BC4900209C95030854950308D9
:1002B00080B586B000AF786039607868F0F762F991
:1002C00002460B46C7E904237868F0F75BF902465B
:1002D0000B46D7E90401F0F7BFF902460B46C7E920
:1002E00004233868F0F74EF902460B46C7E90223AB
:1002F0003868F0F747F902460B46D7E90201F0F7F4
:10030000ABF902460B46C7E90223D7E90223D7E936
:100310000401EFF7EBFF02460B4643EC172BB0EE60
:10032000470AF0EE670A17F0E1FA51EC100B4FF0B4
:100330000002074BEFF7DAFF02460B46104619465C
:10034000F0F762FC034618461837BD4680BD00BF73
:100350000000E03F80B584B000AF786039607B6812
:100360007B817B681B0C3B810EF00AFEF860FB680A
:10037000002B01D0FB6839E0B7F90A30002B07DD0C
:10038000FFF70AF80346002B10D12323FB600DE092
:10039000B7F90A30002B07DAFFF722F80346002BE3
:1003A00004D12423FB6001E00023FB60FB68002BE9
:1003B00001D0FB681AE0B7F90830002B07DDFFF722
:1003C0009DFB0346002B10D12523FB600DE0B7F900
:1003D0000830002B07DAFFF7B5FB0346002B04D1EA
:1003E0002623FB6001E00023FB60FB681846103702
:1003F000BD4680BD80B584B000AF786039600EF036
:10040000CBFDF860FB6818461037BD4680BD80B54F
:1004100084B000AF786039600EF0CAFDF860FEF776
:1004200041FCF860FB68002B01D0FB6800E0FB6832
:1004300018461037BD4680BD80B5BAB000AFF86031
:10044000B9607A600023A7F8E2300123A7F8E03012
:10045000FB68002B04D1BB68002B01D1002325E1F0
:100460007B68002B22D1934B1B68D3F89031642218
:1004700002FB03F37B618F4B1B68D3F89831642236
:1004800002FB03F3BB618B4B1B68D3F89C318A4A98
:10049000B2FBF3F3FB61874B1B68D3F8A031864AAC
:1004A000B2FBF3F33B6207F114037B60FB68002BA4
:1004B00004DA4FF6FF73A7F8E63009E0FB68002B7B
:1004C00003DD0123A7F8E63002E00023A7F8E630B9
:1004D000BB68002B04DA4FF6FF73A7F8E43009E09D
:1004E000BB68002B03DD0123A7F8E43002E0002302
:1004F000A7F8E43007F12403B4220021184614F0D1
:1005000099F901237B620023BB62B7F8E230DB007C
:10051000E8333B4448F2390223F8BC2CB7F8E23008
:10052000DB00E8333B44002223F8BA2C7B6A9BB201
:1005300003F00F039AB2B7F8E23042F4807292B23D
:10054000DB00E8333B4423F8B82CB7F8E230DB009B
:10055000E8333B444FF4007223F8B62CB7F8E2308E
:100560000E339B00E8333B44FA6843F8C42CB7F8D9
:10057000E030DB00E8333B4448F2390223F8BC2C7E
:10058000B7F8E030DB00E8333B44002223F8BA2C14
:100590007B6A9BB203F00F039AB2B7F8E03042F4E3
:1005A000807292B2DB00E8333B4423F8B82CB7F8F2
:1005B000E030DB00E8333B444FF4007223F8B62C04
:1005C000B7F8E0300E339B00E8333B44BA6843F899
:1005D000C42C00237B67BB6883EAE372A2EBE3725F
:1005E000FB68002BB8BF5B429342B8BF1346BB67A2
:1005F0004FF47A73FB677B681B68C7F880307B68B1
:100600001B68C7F884307B685B68C7F888307B68F4
:100610001B68C7F88C307B689B68C7F890307B6894
:100620009B68C7F894307B68DB68C7F89830002374
:10063000C7F89C30214BC7F8A430214BC7F8A8302D
:100640000023C7F8AC300023C7F8B0300023C7F848
:10065000B4300023C7F8B8307B6AC7F8BC30194BF8
:10066000C7F8CC30184BC7F8C830184BC7F8C4309F
:10067000B7F9E4301A04B7F9E6309BB21343C7F870
:10068000D0307B6AC7F8D43007F1240318460AF04B
:1006900097FFC7F8DC00D7F8A0301946D7F8DC0080
:1006A0000FF0E4FDC7F8D800D7F8D8301846E8377F
:1006B000BD4680BDE40C002080FC0A009D8302083A
:1006C0003194020855030208F50302080F040208DA
:1006D00080B588B000AFF860B9607A604C4B0022FA
:1006E000C3F804244A4B1B6843F04003484A136094
:1006F0000023FB61F86908F0FFFC08F071FE454B30
:100700001B6845F2AA5293426DD1414BD3F808328F
:1007100003F00303032B66D13F4B1B68D3F828314A
:10072000FA689A4214DB3C4B1B68D3F82C31FA6808
:100730009A420DDC384B1B68D3F83031BA689A42C4
:1007400006DB354B1B68D3F83431BA689A4207DDB3
:10075000BA68F968314814F0DFFC2223FB6144E0F9
:1007600008F03EFE2B4B5B68FA68D31ABB61294B3D
:100770009B68BA68D31A7B61294814F069FD254B40
:100780005B681946274814F0C7FC224B9B68194642
:10079000254814F0C1FC1F4BDB681946234814F0B0
:1007A000BBFC7A687969B869FFF746FEF8612048B2
:1007B00014F04EFD174B5B6819461A4814F0ACFC58
:1007C000144B9B681946184814F0A6FC114BDB68C3
:1007D0001946164814F0A0FC0E4B1B691946154823
:1007E00014F09AFC01E02123FB61094B0122C3F8BC
:1007F0000424074B1B6823F04003054A1360F86983
:1008000008F07AFCFB6918462037BD4680BD00BF62
:1008100030380020BC490020E40C0020C0950308BB
:10082000F0950308009603080C9603081896030831
:10083000249603083496030880B483B000AF786030
:10084000084BDA68084B1B68D3F84C319A4201DD3B
:10085000002300E0012318460C37BD465DF8047BF9
:10086000704700BFBC490020E40C002080B483B076
:1008700000AF7860084BDA68084B1B68D3F8483142
:100880009A4201DA002300E0012318460C37BD46E6
:100890005DF8047B704700BFBC490020E40C0020D9
:1008A00080B485B000AF78600C4B1B6845F2AA524B
:1008B000934209D10A4BD3F8083203F00403002B0A
:1008C00002D00023FB6001E02123FB60FB68184697
:1008D0001437BD465DF8047B704700BFBC4900205B
:1008E0003038002080B584B000AF78600023FB6012
:1008F00012F00CFD0346012B02D14FF48073FB6014
:10090000FB6818461037BD4680BD000080B59AB020
:1009100000AF7860396007F10803582200211846BB
:1009200013F088FF01233B8102237B8148F23903C6
:10093000BB810023FB8100233B827B6847F230525E
:1009400002FB03F37B614FF47A737B63234B1B68D9
:10095000D3F8E4317B667A6E3B689A4201DD3B68EE
:100960007B667B6E642202FB03F3BB633B686422FD
:1009700002FB03F3FB63194B1B68D3F8F831184AE9
:10098000B2FBF3F33B64154B1B68D3F8FC31144AFC
:10099000B2FBF3F37B64134BBB64134BFB64134B4D
:1009A0003B65134B7B65134B1B6843F04003114AB7
:1009B000136007F1080318460FF02AFB38660D4B49
:1009C0001B6823F040030B4A1360386E08F094FB59
:1009D0003B6E18466837BD4680BD00BFE40C002062
:1009E00080FC0A00390802086D080208A108020804
:1009F000E50802083038002080B584B000AF786088
:100A000039600EF0BDFAF860FB68002B01D0FB687E
:100A100000E0FB6818461037BD4680BD80B584B045
:100A200000AF786039600EF0B7FAF860FB681846DE
:100A30001037BD4680BD000080B584B000AF78603F
:100A400039600AF03DF80346002B07D10E4814F038
:100A5000FFFB4FF48073FB60FB6810E00EF0A8FA18
:100A6000F860FB68002B01D0FB6808E0FEF71AF97C
:100A7000F860FB68002B01D0FB6800E0FB681846BB
:100A80001037BD4680BD00BF4096030880B584B0D6
:100A900000AF786039600AF013F80346002B07D1E5
:100AA000144814F0D5FB4FF48073FB60FB681DE025
:100AB0000EF07EFAF860FB68002B01D0FB6815E0B1
:100AC000FEF7F0F8F860FB68002B01D0FB680DE042
:100AD000094B1B68D3F89831084AA2FB0323DB08B3
:100AE0009BB21846FEF738F9F860FB6818461037D5
:100AF000BD4680BD40960308E40C0020CDCCCCCC94
:100B000080B5B6B000AF786039600223A7F8D63060
:100B10007B68002B01D10023BEE03B68002B22D173
:100B20005F4B1B68D3F8E431642202FB03F3BB6024
:100B30005B4B1B68D3F8EC31642202FB03F3FB60D0
:100B4000574B1B68D3F8F831564AB2FBF3F33B61BD
:100B5000534B1B68D3F8FC31524AB2FBF3F37B6171
:100B600007F108033B6007F11803B422002118467F
:100B700013F060FE0123BB610023FB61B7F8D630A0
:100B8000DB00D8333B4448F2390223F8B82CB7F8DD
:100B9000D630DB00D8333B44002223F8B62CBB69A7
:100BA0009BB203F00F039AB2B7F8D63042F48072CA
:100BB00092B2DB00D8333B4423F8B42CB7F8D630DC
:100BC000DB00D8333B444FF4007223F8B22CB7F863
:100BD000D6300E339B00D8333B447A6843F8C02CA0
:100BE0000023BB667B68002BB8BF5B42FB664FF4FB
:100BF0007A733B673B681B687B673B681B68BB6716
:100C00003B685B68FB673B681B68C7F880303B68E4
:100C10009B68C7F884303B689B68C7F888303B689E
:100C2000DB68C7F88C300023C7F890301E4BC7F83C
:100C300098301E4BC7F89C300023C7F8A030002323
:100C4000C7F8A4300023C7F8A8300023C7F8AC3099
:100C50000023C7F8B030164BC7F8C030154BC7F8A3
:100C6000BC30154BC7F8B8300023C7F8C430BB6997
:100C7000C7F8C83007F1180318460AF0A1FCC7F8F6
:100C8000D000D7F894301946D7F8D0000FF0EEFA1C
:100C9000C7F8CC00D7F8CC301846D837BD4680BD51
:100CA000E40C002080FC0A009D83020831940208B5
:100CB000F90902081D0A0208390A020880B59CB029
:100CC00000AF78605A4BD3F8083223F00403584A37
:100CD000C2F8083208F084FB07F1080364220021FF
:100CE000184613F0A7FD01233B8102237B8148F2C4
:100CF0003903BB810023FB8100233B827B6842F2E6
:100D0000107202FB03F37B617B684A4A02FB03F328
:100D1000BB61494B1B68D3F8E431642202FB03F347
:100D2000BB63454B1B68D3F8E831642202FB03F335
:100D3000FB63414B1B68D3F8F831404AB2FBF3F335
:100D40003B643D4B1B68D3F8FC313C4AB2FBF3F3E8
:100D50007B640023BB643A4BFB6400237B65002368
:100D6000BB650023FB65374B7B66314B1B6843F04B
:100D700040032F4A136007F1080318460EF0D4FE13
:100D8000F8662B4B1B6823F04003294A136064204C
:100D900007F004FBFB6E40F20112934213D109F0FD
:100DA00065FE0346002B0ED1214BD3F8083243F0E9
:100DB00004031F4AC2F80832234814F049FA40F2EB
:100DC0000113FB660DE01A4BD3F8083223F004033D
:100DD000174AC2F80832F96E1C4814F09DF9202316
:100DE000FB661B4BDB68124AD2F8182219461948D9
:100DF00014F092F9104B1B68D3F8D0300C4AC2F8AB
:100E000018320B4BD3F81832194602200AF0A4F915
:100E100008F0E6FA0E4BDB6819460F4814F07CF92F
:100E2000F86E08F069F9FB6E18467037BD4680BD54
:100E30003038002018FCFFFFE40C002080FC0A0082
:100E40006DAA0208010B0208589603086C96030865
:100E5000BC49002088960308BC96030880B584B07E
:100E600000AF786039600023FB60264B1B6843F0BD
:100E70004003244A1360244B1B6845F2AA52934254
:100E80002ED1204BD3F8083203F00403002B27D0D7
:100E90001E4B1B68D3F848317A689A4206DB1B4B1D
:100EA0001B68D3F84C317A689A4209DD164BDB682F
:100EB0007A681946164814F02FF92223FB6012E0D5
:100EC00008F08EFA104BDB687A68D31ABB60BB68F7
:100ED000002B08D03968B868FFF712FEF86002E00E
:100EE0002123FB6000E000BF064B1B6823F040039A
:100EF000044A1360F86808F0FFF8FB6818461037DA
:100F0000BD4680BD30380020BC490020E40C0020E4
:100F1000E496030880B584B000AF786039600023A0
:100F2000FB60284B1B6843F04003264A136008F01F
:100F3000C3FF254B1B6845F2AA5293422ED1214B89
:100F4000D3F8083203F00403002B27D01F4B1B6893
:100F5000D3F848317A689A4206DB1C4B1B68D3F8F9
:100F60004C317A689A4209DD174BDB687A6819467A
:100F7000174814F0D1F82223FB6012E008F030FA91
:100F8000114BDB687A68D31ABB60BB68002B08D0B2
:100F90003968B868FFF7B4FDF86002E02123FB6010
:100FA00000E000BF08F072FF064B1B6823F040030F
:100FB000044A1360F86808F09FF8FB681846103779
:100FC000BD4680BD30380020BC490020E40C002024
:100FD000E496030880B584B000AF78600023FB601E
:100FE000244BD3F8003245F2AA5293420CD1224B43
:100FF0001B6845F2AA52934206D11E4BD3F8083221
:1010000003F00403002B03D10120FFF757FEF86023
:10101000FB6840F20112934202D0FB68002B24D1FE
:10102000144BD3F8003245F2AA5293421BD1124B13
:101030001B6845F2AA52934212D10E4BD3F80832E4
:1010400003F00403002B0BD00C4B1B68D3F85C227D
:101050007B68134400211846FFF75CFFF86004E04A
:101060005523FB6001E01623FB60FB681846103730
:10107000BD4680BD30380020BC490020E40C002073
:1010800080B582B000AF00237B60244BD3F80032E0
:1010900045F2AA5293420CD1214B1B6845F2AA5249
:1010A000934206D11D4BD3F8083203F00403002B02
:1010B00003D10120FFF702FE78607B6840F2011245
:1010C000934202D07B68002B22D1144BD3F800321C
:1010D00045F2AA52934219D1114B1B6845F2AA520C
:1010E000934210D10D4BD3F8083203F00403002BC8
:1010F00009D00C4B1B68D3F85C3200211846FFF76F
:10110000ADFE786004E055237B6001E016237B6030
:101110007B6818460837BD4680BD00BF30380020C8
:10112000BC490020E40C002080B598B000AF7E4B95
:10113000D3F8083223F008037B4AC2F808320023B0
:10114000FB65FFF79DFFF865FB6D002B04D0F86D84
:1011500007F0D2FFFB6DE3E008F042F93B1D582297
:101160000021184613F066FB0123BB800323FB809C
:1011700048F239033B8100237B810123BB8142F28A
:1011800010733B61694B1B68D3F8003242F2107256
:1011900002FB03F3DB08664AA2FB03239B087B6187
:1011A000624B1B68D3F8043242F2107202FB03F365
:1011B000DB085F4AA2FB03239B08BB615B4B1B68F8
:1011C000D3F80C3242F2107202FB03F3DB08584AE8
:1011D000A2FB03239B08574AB2FBF3F3FB61534B7B
:1011E0001B68D3F8103242F2107202FB03F3DB08E3
:1011F0004F4AA2FB03239B084E4AB2FBF3F33B6228
:101200000023BB640023FB6400233B654A4B3B6423
:101210000023BB65444B1B6843F04003424A136004
:101220003B1D18460DF070FFF8653F4B1B6823F01F
:1012300040033D4A1360642007F0B0F8FB6DB3F53E
:10124000807F15D13B6C984703461A46BB6D9A4286
:101250000ED1354BD3F8083243F00803324AC2F8B6
:101260000832364813F0F4FF40F20113FB650BE03F
:101270002D4BD3F8083223F008032B4AC2F808326A
:10128000F96D2F4813F048FFFB6D40F201129342B5
:101290003AD1254BD3F8083203F00803002B33D0A2
:1012A00009F0F2FB0346002B2ED1264B1B691E4A88
:1012B000D2F81C221946244813F02EFF1B4B1B6842
:1012C000D3F8D83042F2107202FB03F31F4A82FBBC
:1012D00003129213DB17D31A134AC2F81C32124BB3
:1012E000D3F81C321946032009F036FF08F078F8CD
:1012F000144B1B691946164813F00EFF002140F6E7
:10130000C41000F09BF907E0074BD3F8083223F034
:101310000803054AC2F80832F86D07F0EDFEFB6DD0
:1013200018466037BD4680BD30380020E40C0020F0
:10133000176CC11600A24A0489AA0208189703086C
:101340002C970308BC490020489703086B29827436
:101350007097030880B584B000AF78600023FB600D
:1013600011F0D4FF0346012B02D14FF48073FB60D0
:10137000FB6818461037BD4680BD000080B59AB0A6
:1013800000AF786039603B68002B02DC01233B60D2
:1013900005E03B684B4A934201DD4A4B3B6000232A
:1013A0003B660020FFF716FE38663B6E002B04D02C
:1013B000386E07F0A1FE3B6E80E007F1080358226B
:1013C0000021184613F036FA01233B8103237B8169
:1013D00048F23903BB810023FB8101233B823A4B56
:1013E0007B617B697A6802FB03F37B6142F21073D5
:1013F0007B63364B1B68D3F800327B667A6E3B68A2
:101400009A4201DD3B687B667B6E42F2107202FB02
:1014100003F32F4A82FB03121A441212DB17D31A6A
:10142000BB633B6842F2107202FB03F3284A82FB63
:1014300003121A441212DB17D31AFB63234B1B68E7
:10144000D3F80C3242F2107202FB03F3DB08214A9C
:10145000A2FB03239B08204AB2FBF3F33B641B4B24
:101460001B68D3F8103242F2107202FB03F3DB0860
:10147000184AA2FB03239B08174AB2FBF3F37B64D1
:101480000023BB640023FB6400233B65134B7B6597
:10149000134B1B6843F04003114A136007F1080324
:1014A00018460EF0B5FD38660D4B1B6823F040035F
:1014B0000B4A1360386E07F01FFE3B6E1846683704
:1014C000BD4680BDA086010000E1F505E40C0020CA
:1014D000B7600BB6176CC11600A24A045513020878
:1014E0003038002090B5A7B000AF786039607B68D5
:1014F000002B01D1002396E00023C7F8903007F1BC
:101500001C0374220021184613F094F90123BB83B5
:101510000023BB667B68002BB8BF5B42FB660023E1
:101520003B670023FB8303233B6248F23903BB8400
:101530007B68BB620023C7F8883042F210737B6778
:101540000123C7F8943010E0D7F8942013465B00CD
:1015500013449B0098333B44783B4FF0FF321A60B2
:10156000D7F894300133C7F89430D7F89430052B6E
:10157000EADD3B68002B45D12D4B1B68D3F80032C8
:1015800042F2107202FB03F3DB082A4AA2FB032398
:101590009B08FB60264B1B68D3F8083242F210729E
:1015A00002FB03F3DB08234AA2FB03239B083B61F6
:1015B0001F4B1B68D3F80C3242F2107202FB03F38C
:1015C000DB081C4AA2FB03239B081B4AB2FBF3F374
:1015D0007B61174B1B68D3F8103242F2107202FB8A
:1015E00003F3DB08134AA2FB03239B08124AB2FB56
:1015F000F3F3BB6107F1780407F10C030FCB84E828
:101600000F0007E03B6807F17804186859689A688A
:10161000DB680FC407F11C0318460EF0C7F8C7F8C3
:101620009000D7F8903018469C37BD4690BD00BF5B
:10163000E40C0020176CC11600A24A0480B586B0E5
:1016400000AF78603960224B0022C3F80424204B9D
:101650001B6843F040031E4A136000237B617869D6
:1016600007F04AFD1B4B1B6845F2AA5293421BD15F
:10167000174BD3F8083203F00803002B14D007F0FF
:10168000AFFE144B1B693B617A683B69D31AFB6060
:1016900007F10C0318460EF0C1FDFB680021184647
:1016A000FFF720FF786101E021237B61084B0122D5
:1016B000C3F80424064B1B6823F04003044A13605C
:1016C000786907F019FD7B6918461837BD4680BD5B
:1016D00030380020BC49002080B584B000AF78606D
:1016E0000023FB6011F012FE0346012B02D14FF4E0
:1016F0008073FB60FB6818461037BD4680BD000054
:1017000080B59CB000AF7860396000237B6607F13C
:101710000C0358220021184613F08CF80123BB81DA
:101720000423FB8148F239033B8200237B8201239F
:10173000BB827B68314A02FB03F3BB614FF47A73CF
:10174000BB632F4B1B68D3F8B431FB663B68012B9E
:1017500005DC2B4B1B68D3F8B831BB6610E03B6847
:10176000022B05D1264B1B68D3F8BC31BB6607E0C2
:101770003B68022B04DD224B1B68D3F8C031BB66EB
:10178000FA6EBB6E9A4201DDBB6EFB66FB6E642295
:1017900002FB03F3FB63BB6E642202FB03F33B64B7
:1017A000174B1B68D3F8C831164AB2FBF3F37B64BE
:1017B000134B1B68D3F8CC31124AB2FBF3F3BB6472
:1017C00000237B65104BBB65104B1B6843F0400347
:1017D0000E4A136007F10C0318460EF019FC7866E8
:1017E0000A4B1B6823F04003084A1360786E07F029
:1017F00083FC7B6E18467037BD4680BDE0930400C5
:10180000E40C002080FC0A00D916020830380020C1
:1018100080B5B6B000AF786039600423A7F8D43043
:101820007B68002B01D10023D2E03B68002B22D142
:10183000694B1B68D3F8B431642202FB03F3BB602D
:10184000654B1B68D3F8D031642202FB03F3FB60C5
:10185000614B1B68D3F8C831604AB2FBF3F33B61BC
:101860005D4B1B68D3F8CC315C4AB2FBF3F37B6170
:1018700007F108033B607B68002B04DA4FF6FF7327
:10188000A7F8D63009E07B68002B03DD0123A7F819
:10189000D63002E00023A7F8D63007F11803B422AF
:1018A0000021184612F0C6FF0123BB610023FB6133
:1018B000B7F8D430DB00D8333B4448F2390223F880
:1018C000B82CB7F8D430DB00D8333B44002223F8DF
:1018D000B62CBB699BB203F00F039AB2B7F8D430B1
:1018E00042F4807292B2DB00D8333B4423F8B42C2C
:1018F000B7F8D430DB00D8333B444FF4007223F800
:10190000B22CB7F8D4300E339B00D8333B447A68FE
:1019100043F8C02C0023BB667B68002BB8BF5B423A
:10192000FB664FF47A733B673B681B687B673B68D9
:101930001B68BB673B685B68FB673B681B68C7F855
:1019400080303B689B68C7F884303B689B68C7F869
:1019500088303B68DB68C7F88C300023C7F89030CC
:101960001F4BC7F898301F4BC7F89C300023C7F8AF
:10197000A0300023C7F8A4300023C7F8A830002304
:10198000C7F8AC30BB69C7F8B030174BC7F8C030E8
:10199000164BC7F8BC30164BC7F8B830B7F9D6307D
:1019A0009BB2C7F8C430BB69C7F8C83007F1180349
:1019B000184609F005FEC7F8D000D7F8943019464C
:1019C000D7F8D0000EF052FCC7F8CC00D7F8CC30D6
:1019D0001846D837BD4680BDE40C002080FC0A00C4
:1019E0009D8302083194020889F50108E5F5010894
:1019F000FFF501080000000080B582B000AF7860FC
:101A00007868EEF7BFFD0AA3D3E90023EEF724FEC2
:101A100002460B4610461946EFF7CEF803467B60A8
:101A20007B6818460837BD4680BD00BFAFF3008015
:101A300060E5D022DBF9204080B584B000AF78604B
:101A40000023FB6011F062FC0346012B02D14FF42E
:101A50008073FB60FB6818461037BD4680BD0000F0
:101A600080B59CB000AF7860396000237B6607F1D9
:101A70000C0358220021184612F0DCFE0123BB8122
:101A80000523FB8148F201033B8201237B82012372
:101A9000BB827B68314A02FB03F3BB614FF47A736C
:101AA000BB632F4B1B68D3F8B431FB663B68012B3B
:101AB00005DC2B4B1B68D3F8B831BB6610E03B68E4
:101AC000022B05D1264B1B68D3F8BC31BB6607E05F
:101AD0003B68022B04DD224B1B68D3F8C031BB6688
:101AE000FA6EBB6E9A4201DDBB6EFB66FB6E642232
:101AF00002FB03F3FB63BB6E642202FB03F33B6454
:101B0000174B1B68D3F8C831164AB2FBF3F37B645A
:101B1000134B1B68D3F8CC31124AB2FBF3F3BB640E
:101B200000237B65104BBB65104B1B6843F04003E3
:101B30000E4A136007F10C0318460EF069FA786636
:101B40000A4B1B6823F04003084A1360786E07F0C5
:101B5000D3FA7B6E18467037BD4680BDE093040013
:101B6000E40C002080FC0A00391A020830380020FA
:101B700080B5B6B000AF786039600523A7F8D430DF
:101B80007B68002B01D10023D2E03B68002B22D1DF
:101B9000694B1B68D3F8B431642202FB03F3BB60CA
:101BA000654B1B68D3F8D031642202FB03F3FB6062
:101BB000614B1B68D3F8C831604AB2FBF3F33B6159
:101BC0005D4B1B68D3F8CC315C4AB2FBF3F37B610D
:101BD00007F108033B607B68002B04DA4FF6FF73C4
:101BE000A7F8D63009E07B68002B03DD0123A7F8B6
:101BF000D63002E00023A7F8D63007F11803B4224C
:101C00000021184612F016FE0123BB610023FB6180
